:1000000000800020BD01000059D3000011D3000082
:1000100011D3000011D3000011D3000011D3000050
:1000200011D3000011D3000011D3000059D30000F8
:1000300059D3000011D30000D9C90000DDCA000067
:1000400059D3000059D3000059D3000059D3000000
:1000500059D3000059D3000059D3000059D30000F0
:1000600059D3000059D3000059D3000059D30000E0
:1000700059D3000059D3000059D3000059D30000D0
:1000800059D3000059D3000059D3000059D30000C0
:1000900059D3000059D3000059D3000059D30000B0
:1000A00015AF000021AF000059D3000059D3000064
:1000B00059D3000059D3000059D3000059D3000090
:1000C00059D3000059D3000059D3000059D3000080
:1000D00059D3000059D3000059D3000059D3000070
:1000E00059D3000059D3000059D3000059D3000060
:1000F00059D30000C5F3000059D30000F1F400000B
:1001000059D3000031DD000059D3000059D300005D
:1001100059D3000059D3000059D3000059D300002F
:1001200059D3000059D3000059D3000059D300001F
:1001300059D3000059D3000059D3000059D300000F
:1001400059D3000059D3000059D3000059D30000FF
:10015000C9CB0000DDCB0000F1CB000005CC0000D6
:1001600059D300004DE0000059D3000059D30000DE
:1001700059D3000059D3000059D3000059D30000CF
:1001800059D3000059D3000059D3000059D30000BF
:1001900059D3000059D3000059D3000059D30000AF
:1001A00059D3000059D3000059D3000059D300009F
:1001B00059D3000059D3000059D30000564B4CF2DC
:1001C000205210B51A804DF628121A8000BF00BFC9
:1001D0000DF0C6F8514B4FF010621A60504A9A6009
:1001E000504ADA60504A136813F4807304D14F49BF
:1001F0000B604FF4A85313604D4B1A78110703D5C9
:100200001A7842F008021A704A4B4B492A221A7097
:100210004A4A4B4B8B4204D252F8040F43F8040B6A
:10022000F8E7484B484900228B4202D243F8042B9E
:10023000FAE74649464A002352F8230041F82300D2
:1002400001336F2BF8D1434B434A802103F8011B44
:100250009342FBD1414B3D4A1A60414B8A221A70AE
:10026000A3F5805324225A70A0221A709A7992071B
:10027000FCD59A79D406FCD43A4A937903F00C035E
:10028000082B384BF9D103221A7140225A719A79FE
:100290009006FCD5334A9179324B4906FBD5324A58
:1002A000324911600221516020221A709A7902F0BD
:1002B0000C020C2AFAD12E4B2E4A1A602E4B2F4AD2
:1002C0001A6000225A60072243F8042C2C4AC3F813
:1002D0000C2D62B60DF0F4FB144B1B68DA0705D544
:1002E00028480DF0C1F9284B284A1A60284B1B7882
:1002F0005B0609D5244C254B22689A4204D121483B
:100300000DF0B2F90023236010F0AAFB0DF02EF8D7
:100310000CF05CFFFEE700BF0E200540308004407B
:10032000823F04000100002B10D0034014D0034092
:1003300002D0074000E00740D49BFF1FF4430100B8
:100340004088FF1FD49BFF1FE8A3FF1F0082FF1FF1
:100350000000000000E400E05FE400E008ED00E0E1
:100360000050064000400640448004400000030165
:1003700004800440C010050014E000E0FF76010096
:1003800000002020236F4F5F1CE00340A5C3945A58
:1003900000F00740FFFFFFFFFFFFFFFFFFFFFFFF32
:1003A000FFFFFFFFFFFFFFFFFFFFFFFFFFFFFFFF5D
:1003B000FFFFFFFFFFFFFFFFFFFFFFFFFFFFFFFF4D
:1003C000FFFFFFFFFFFFFFFFFFFFFFFFFFFFFFFF3D
:1003D000FFFFFFFFFFFFFFFFFFFFFFFFFFFFFFFF2D
:1003E000FFFFFFFFFFFFFFFFFFFFFFFFFFFFFFFF1D
:1003F000FFFFFFFFFFFFFFFFFFFFFFFFFFFFFFFF0D
:10040000FFFFFFFFFFFFFFFFFFFFFFFFDEF9FFFF23
:1004100010B5054C237833B9044B13B10448AFF33E
:1004200000800123237010BDD49BFF1F000000003B
:10043000F8430100084B10B51BB108490848AFF359
:1004400000800848036803B910BD074B002BFBD0A0
:10045000BDE81040184700BF00000000D89BFF1FF8
:10046000F8430100D49BFF1F0000000038B504468C
:10047000104621700A491D4610F0D4F801464FF08D
:100480007E5010F083F9074910F0CCF8E560606009
:10049000256165610DF0A4FAE061204638BD00BF1A
:1004A000DB0FC9400024744938B50446104621705A
:1004B00009491D4610F0B6F801464FF07E5010F085
:1004C00065F9064910F0AEF8E56060602561656188
:1004D0000DF086FAE06138BDDB0FC9400024744995
:1004E00038B503780446032B20D8DFE803F01A1848
:1004F0001002C16840690FF08BFF0D490546606826
:1005000010F044F90146284610F040F938BD08497A
:10051000406810F03BF9E16810F084F838BDC0681D
:1005200038BDC16840690FF073FF38BD002038BD89
:100530000024744970B504460E460DF051FA054684
:10054000E069281A10F01AF8E3682361E561666132
:10055000A0610146606810F019F90146A0601048DA
:1005600010F014F90FF0EAFB0FF08AF80FF0FCFE20
:10057000054601464FF07E500FF04AFF616910F0CA
:1005800051F821690646284610F04CF801463046DD
:100590000FF040FFE0602046BDE87040FFF7A0BFCD
:1005A000000080BF08B50E200CF0EAFC114B1B8840
:1005B000012B19D0104B1B88984213DB40F6FF71BA
:1005C0008842D4BFC3EB0001C3EB0101C1EB013191
:1005D000C3F57F630F33282091FBF3F1BDE808409A
:1005E0000DF054B80021F3E70146BDE8084014209F
:1005F0000DF04CB8209EFF1FB49CFF1F10B50446A1
:100600000CF0C0FA204610BD70B44C88A04220D92E
:1006100001230133DBB21CB2660031F8144084427E
:100620001D46F6D3A04211D005F10045013D965B71
:1006300031F8151032F81530401AF21A00FB02F0AA
:10064000641A90FBF4F4E01870BC7047905B70BCC7
:10065000704702260125E5E700280CDA064A4342E6
:1006600082FB0320DA17C2EB600000EB4000A3EB33
:100670008000C0F10C007047ABAAAA2A38B5234B02
:100680001B78002B2CD015200CF07AFC204B186026
:10069000204B1B88984203DA1F4C237863BB38BD7C
:1006A0001E4A1488A042A4EB0302A8BF20467F2A5A
:1006B0001CDDC01AC001541C90FBF4F4002CEBD0DC
:1006C000154B1A780AB901221A70154D2B689C42F5
:1006D00004D0144BE1B2187808F0EEFC2C6038BD61
:1006E00011200DF091FB0A4B1860D1E7C01AC0EB46
:1006F000C01090FBF2F4E1E70A4B0021187808F0F3
:10070000DBFC0023064A2370136038BD329EFF1FB6
:10071000009CFF1F769CFF1FA49EFF1F4C9EFF1F87
:10072000A09EFF1F4C9CFF1F38B50F200DF06CFBE7
:100730001B4A1C4B12881860C0F53B600830904281
:1007400020DB194B1B889842A3EB0204A8BF184674
:10075000801A7F2CC6BFC0010134C0EBC01090FBD3
:10076000F4F47CB1114B1A780AB901221A70104DB9
:100770002B689C4204D00F4BE1B2187808F09CFC27
:100780002C6038BD094C237803B938BD094B0021D2
:10079000187808F091FC0023054A2370136038BDD7
:1007A000B89CFF1FC89DFF1F389EFF1F5C9EFF1F48
:1007B000809CFF1F6E9CFF1FF0B40E8886420DD2F6
:1007C00003F10043013B31F81350854202D9F0BCDC
:1007D000FFF71ABF32F81300F0BC70471088F0BC66
:1007E000704700BF094B1B880C2B09D8084A80B200
:1007F00052F8232028B143F6FE73984203D9108C97
:100800007047108870470349FFF7FEBE269CFF1F04
:10081000601E0100FC1F01004B4B4C4A2DE9F047C4
:100820001E8814684A4BB442B3F80080494B33DB4E
:100830004445A8BF4446A6421C60C8BF00202DDD29
:10084000C6EB0807B7F5804F33DB80037B1C90FBBA
:10085000F3F0FFF7C7FF404A404B15881B88C0F3F1
:10086000C61909FB05F57F2D8246A8BF7F252BB34E
:10087000A64253DC4445D4BFC6EB0404C6EB0804CF
:100880009F42CCBF03FB04445C43354BC8BF0137D8
:1008900094FBF7F71F6013E034461E60C6EB0807B1
:1008A000A045D4BFC6EB0800C6EB0400B7F5804FE7
:1008B000CBDAC0EB803090FBF7F0CAE7284A136030
:1008C000284C2368994508D0274B1B88002B34D12E
:1008D000264B1B886BBBC4F80090254C23689A45B7
:1008E00006D0214B1B885A1F032A19D9C4F800A02F
:1008F000204C23689D420FD01F4B188848B11A4BDB
:100900001E4A1B88D35C834203D0C0B2E9B208F010
:10091000D3FB2560BDE8F087BDE8F0870024AFE792
:10092000164AD05C2030C0B20AF07F0108F0C4FB48
:10093000DCE7484608F034FCCDE7104A4946D05C75
:1009400008F0BAFBC4E700BFB49CFF1F1C9EFF1F4A
:100950007C9EFF1FF89BFF1F089CFF1F0A9CFF1F28
:10096000849EFF1F689CFF1F029EFF1FAA9CFF1F03
:10097000209CFF1FAC9CFF1F129EFF1F9889FF1F2A
:100980002DE9F04F17208BB00DF03EFADFF870B371
:10099000DFF870A3CBF8000016200DF035FABA4B43
:1009A000CAF800001B880C2B00F05E82B74EB84AD4
:1009B0003188B84B52F8214000221A70B64BB74A22
:1009C0001B88B7491288013B012A31F9133005937E
:1009D00000F0AE81B34B0193B34B0293B34FDFF8FA
:1009E000288300230093B24B1B88012B00F0F48175
:1009F000DFF81893AF4B0393D9F80050AE4B049334
:100A00000023AE4A1288013A032A00F24982DFE845
:100A100012F0A500ED000400C900284605930FF070
:100A2000ADFDA7490FF0FEFD059B054618460FF0EA
:100A3000A5FDA4490FF0F6FD014628460FF0EAFC9B
:100A40000FF0B6FF0546C9F8005038680FF096FD64
:100A50009B490FF0E7FD814600980FF08FFD994903
:100A60000FF0E0FD014648460FF0D4FC0FF0A0FF68
:100A70003860954A954B17881988954BDBF800200C
:100A80001B88DFF88CE2C7EB050C3D44039FC7F8D9
:100A900000C0471A084404990D6001990F6002993B
:100AA000BEF8007008609A4280F2E7800025C3EB30
:100AB000070E7445DAF8000080F2D380611C98427A
:100AC00005FB01F50EF1010E95FBFEF5C0F25F830B
:100AD0008742A8BF0746FF1A01FB07F494FBFEF408
:100AE0009A4200F3A780984200F3A480794C2068D2
:100AF0000FF044FD78490FF095FD78490FF08AFC1E
:100B00000FF056FFA0F5FF531C3B082B98BF4FF486
:100B10000050D8F80030184400282060C0F29F80B0
:100B2000B0F5804F80F2F6806D4B1B781BB1B0F5AD
:100B3000005F40F0F7806B4D2B78002B40F0AB81CD
:100B4000694D20682B68634C984204D080B208F04D
:100B500091FB23682B600BB0BDE8F08F284605930E
:100B60000FF00CFD61490FF05DFD059B0546184631
:100B70000FF004FD5E490FF055FD014628460FF0C9
:100B800049FC0FF015FF0546C9F8005038680FF012
:100B9000F5FC56490FF046FD814600980FF0EEFC3B
:100BA00053495DE7284605930FF0E8FC4A490FF0EA
:100BB00039FD059B054618460FF0E0FC4D490FF046
:100BC00031FD014628460FF025FC0FF0F1FE0546E9
:100BD000C9F8005038680FF0D1FC3F490FF022FDF2
:100BE000814600980FF0CAFC424939E72846059330
:100BF0000FF0C4FC40490FF015FD059B0546184653
:100C00000FF0BCFC3D490FF00DFD014628460FF0EA
:100C100001FC0FF0CDFE0546C9F8005038680FF012
:100C2000ADFC35490FF0FEFC814600980FF0A6FCA4
:100C3000324915E73388002B3FF458AF2B1B002BAC
:100C4000B8BF5B42092B00F32D81D8F80030214C4E
:100C50004FF40050184400282060BFF661AF002216
:100C60005AE0984205FB04F5B8BF002195FBFEF55C
:100C700080F2848291FBFEF432E7BA42D4BFC3EB28
:100C80000205C3EB070512E74E9EFF1F5C9CFF1F8A
:100C90005889FF1FFE9BFF1F2089FF1F229EFF1FF9
:100CA00068220100509CFF1F909CFF1FF09BFF1FBC
:100CB000B09DFF1F409EFF1FB49DFF1F2E89FF1F89
:100CC000CDCC4C3FCDCC4C3EA489FF1F2C89FF1FBF
:100CD000189EFF1F8C89FF1F9A99193FCDCC4C4558
:100CE000569FFF1FA99CFF1F2489FF1F3333733FAB
:100CF000CDCC4C3DCDCCCC3E6666663FCDCCCC3D1C
:100D0000589CFF1F1C9CFF1F589EFF1F3C9EFF1FEF
:100D1000389CFF1F43F6FF72C04B22601B78002BEC
:100D20003FF409AF05F094FBBD4B01221A7007E7B1
:100D3000BC4BBD4A1B88BD491278013B31F91350A9
:100D4000002A40F0C78011200DF05EF80090B84BEB
:100D50000193D3F80080009B984540F3C080B54BC9
:100D6000B54F1B88B54A012B3B68B2F80090B44AD6
:100D700002922046A3EB050500F0E2800FF0FEFB97
:100D8000029A52F829100FF04DFC014600200FF096
:100D90003FFB0FF00DFE009BC8EB05029D42B8BF64
:100DA0001D469042C8EB050580F2DE8000FB05552C
:100DB000013295FBF2F5A34BDFF8B4820293D8F829
:100DC00000302B4403EBD3735B10C8F800309E4B0C
:100DD0001B88012B7FF40CAE9C4B03931D460F2008
:100DE0000DF012F82A6804929042034680F2CC80FB
:100DF000904A1288012A00F03F81904A0790128899
:100E00008F4D069220460FF0B9FB069ADFF86492E8
:100E100055F82210D9F800500FF004FC01460020CC
:100E20000FF0F6FA059BEA1A05920FF0C1FD059A3C
:100E3000079B04999A42C1EB020EB8BF1A4670454F
:100E400080F24481521A00FB02220EF1010192FB52
:100E5000F1F2D8F800107E4804900A4402EBD272F6
:100E60005210C8F80020CCE57A4B1B78002B3FF4D9
:100E70009DAD794E794A3188794B52F82100012293
:100E80001A700FF07BFB4FF07C510FF0CBFB0FF093
:100E90008FFD044692E505F0D7FA00232B704FE64C
:100EA0003868E6E505F500500130001B0FF066FBE1
:100EB0006C496D4C0FF0B6FB054620680FF05EFBE9
:100EC0006A490FF0AFFB014628460FF0A3FA0FF076
:100ED0006FFD1EE615200CF053F8009037E7594BD4
:100EE0000293D3F80080009B984542DA514B524F51
:100EF0001B88524A012B3B68B2F80090504A03927B
:100F000020461D4400F0E9800FF038FB039A52F8A8
:100F100029100FF087FB0FF04BFD009B9D42C8EBA3
:100F20000502A8BF1D46C8EB05059042BABF00FBED
:100F300005550132454395FBF2F5DFF834813EE774
:100F40000FF01CFB029A52F829100FF06BFB0FF008
:100F50002FFD009BC8EB05029D42B8BF1D46824293
:100F6000C8EB05053FF722AF00FB05F595FBF2F551
:100F700021E7DFF8FC80304FD8F8003003EBD37363
:100F80005B10C8F800302EE5314A049212680692D0
:100F9000904237DD274A1288012A00F0BC80274A98
:100FA00009901188264A0891204607920FF0E6FA28
:100FB000079A0899DFF8BC9052F82110D9F8005030
:100FC0000FF030FB059B2B4405930FF0F1FC0599C6
:100FD000099B069A9942C2EB010EA8BF19467045BB
:100FE00080F2BE80891A00FB01110EF1010291FB13
:100FF000F2F2D8F800100A4402EBD2725210C8F88C
:101000000020FEE4D8F80020DFF8689002EBD272EE
:101010005210D9F80050C8F80020F2E4569FFF1F84
:10102000A99CFF1FA889FF1F329EFF1FB41F01004C
:10103000509CFF1F969CFF1FF09BFF1F409CFF1FB3
:1010400080220100909CFF1FB09DFF1F409EFF1F4C
:10105000B49DFF1F009EFF1F5C9CFF1F5889FF1F50
:10106000FE9BFF1FCDCCCC3E8C89FF1F9A99193F68
:10107000589EFF1F3C9EFF1F464A08901188464A13
:101080000791204606920FF079FA069A0799DFF841
:101090000C9152F82110D9F800500FF0C3FA059BBB
:1010A000E91A05910FF084FC0599089B049A99426E
:1010B000C2EB010EB8BF1946704558DA891A00FB19
:1010C00001110EF1010291FBF2F2C2E60499521AEB
:1010D00000FB02F292FBFEF2BBE60FF04FFA039A1E
:1010E00052F829100FF09EFA014600200FF090F9F7
:1010F0000FF05EFC009A9542C8EB0503A8BF1546A9
:10110000C8EB05059842BABF00FB055501334543BE
:1011100095FBF3F511E71F491F4A089020460D88FB
:1011200007920FF02BFA079ADFF8709052F825100B
:10113000D9F800500FF076FA014600200FF068F958
:10114000059B2B4405930FF033FC0599089B069AE9
:101150009942C2EB010EA8BF19467045FFF642AF97
:10116000069A891A00FB01F191FBFEF241E7049A0D
:10117000891A00FB01F191FBFEF26AE6B842D4BF86
:10118000C3EB0001C3EB070104FB01F172E51F464D
:10119000A1E400BF409CFF1F802201003C9EFF1F76
:1011A00008B5244B1B88FBB1234B1B78FBB1234BA9
:1011B0001B78E3B1224B1B78CBB1224B1B78B3B128
:1011C000214B22481A78C2B9214A22490088128844
:1011D00009680244B1EB620F09DD01221A70642034
:1011E000BDE8084005F048B9174A117801B908BDB3
:1011F0001370BDE8084008F007B8154A1649008882
:10120000128809680244B1EB620FF0DD00221A7007
:1012100007F0FAFF642005F02FF9642005F02CF99F
:10122000642005F029F94FF41670BDE808400CF071
:10123000F9BB00BFC09DFF1FA89EFF1F769EFF1F2A
:10124000779EFF1F789EFF1F249CFF1F389CFF1F67
:10125000189EFF1F589CFF1F1C9CFF1F38B5114C88
:10126000232025780BF08CFE0F4A42F82500131F2F
:1012700002F1C400002253F8041F83420A44FAD149
:1012800023780A4907480A4C0133DBB2322B81FB31
:10129000025108BF0023D217C2EB21120370226053
:1012A00038BD00BF0C9CFF1FC49CFF1F1F85EB5166
:1012B000149EFF1F2DE9F04FB84CB94D2068B94F6F
:1012C00083B00FF05BF9B8490FF0ACF90646102077
:1012D0000CF09AFD0FF052F9B4490FF0A3F9314622
:1012E0000FF098F80FF064FB2988206088423B8853
:1012F00043DA9E465B1A7F2B4FF0000247DDD20196
:101300005E1C92FBF6F2AA4EDFF8C882B6F800C067
:10131000C8F80020BCF1190F00F0DF80BCF11A0FF3
:1013200000F01781BCF11E0F00F020810126B146AC
:10133000A04A1288002A00F09D808842C0F20781EE
:101340007045D4BFC1EB0000C1EB0E009A42BABF9A
:1013500002FB00000133504390FBF3F3964A136005
:10136000964B1888C0B9964A1288AAB9954B197835
:1013700001B11A7003B0BDE8F08F9842D4BFC1EB41
:101380000002C1EB03029E465B1A7F2BB7DCC2EB67
:10139000C21292FBF3F2B6E72988D4F800E0DFF836
:1013A0000082DFF8F8A171456CDCDFF818C29CF808
:1013B0000020002A2ED14FF0010B04288CF800B039
:1013C00028D1002E40F094817D4B18880028D1D080
:1013D000B9F1000FCED023682C883A88A34280F25E
:1013E00065810023141B7E2C774DD5BFC3EB83137F
:1013F000C3EBC3135B00013493FBF4F42B6801349B
:10140000A34203D0C0B2E1B207F056FE2C6003B095
:10141000BDE8F08F012800F0F680022800F0EB8094
:101420000328D1D1694B1B88092BCDD0002ECBD0FE
:1014300023682E883A88B34280F27B810023961B72
:101440007E2EDFF88CA1D5BFC3EB8313C3EBC31390
:101450005B00013693FBF6F6DAF800300136B34252
:1014600003D0F1B24A2007F027FECAF80060ABE7CC
:1014700016469146BCF11E0F7FF472AF0022DFF8D2
:1014800058817EE04F4B1A78002A3FF473AF002456
:1014900001281C7000F0A480022840F00E81002E6C
:1014A00000F0A3804A4D2B68002B00F09E800420A2
:1014B000214607F001FE424B2C60188800283FF4BB
:1014C00059AFB9F1000F3FF455AFC0B2002107F09A
:1014D000F3FD3D4B00221A604CE7DFF8FC8098F8E2
:1014E0000020C2B1DFF8D890B9F800A0BAF1000F1F
:1014F00011D0DFF8E89099F800B0934578D05FFA02
:101500008AF07F2107F0D8FD98F80030B6F800C0C7
:1015100089F8003010E0DFF8C49099F800A09245F7
:1015200066D0274B0021187807F0C6FD98F80030E8
:10153000B6F800C089F800301E4B1A88002A97D0F0
:10154000BCF11E0F40F006810026B14619E00020D4
:10155000FCE6DFF8848098F80020002A0BBF012603
:1015600000264FF000094FF00109E1E6DFF868803E
:10157000104B98F800601A88B6FA86F676094FF094
:10158000000998F80030002B3FF4E8AE2988B7F83E
:1015900000E02068C1EB0E03CFE600BF489CFF1FB0
:1015A000C69DFF1FC29DFF1F9A99193FCDCCCC3E0F
:1015B0004E9EFF1F889EFF1FBC9CFF1F569CFF1F57
:1015C000609EFF1F559EFF1F2C9CFF1F029EFF1F4A
:1015D000C09CFF1F349EFF1F009EFF1F109CFF1F1B
:1015E0001EB1614D2B68002B7BD1604B188865E7DD
:1015F0000026B1469CE6002E3FF4E6AEDFF868A177
:10160000DAF800202EE0002E3FF4DEAEB7F80080BE
:10161000F045D4BFC1EB0802C1EB0E02C1EB0808D4
:10162000B8F17E0FDFF840A1D5BFC2EB8212C2EB4A
:10163000C212520008F1010892FBF8F8DAF8002013
:1016400008F10108424506D05FFA88F101200093B5
:1016500007F032FD009B1888CAF8008002287FF44A
:10166000DFAE42462168B5F800803888414559DA36
:101670000021C8EB0008B8F17E0FD3BFC1EB811188
:10168000C1EBC11108F10108490091FBF8F808F11C
:101690000108904506D05FFA88F10420009307F016
:1016A0000BFD009B1888CAF80080B9E69342D4BFAE
:1016B000C4EB0303C4EB020394E6032827D12C4BAD
:1016C0001B88092B91D0002E8FD0274D2B68002B23
:1016D0008BD04A20214607F0EFFC244B2C60188861
:1016E000ECE6214607F0E8FC204B2C601888E5E684
:1016F00040207F218DE80C0007F0DEFC019B009A62
:10170000188858451CD002287FF48AAE76E7042852
:101710007FF46BAF002E3FF468AF2146402007F006
:10172000CBFC62E78142D4BFC8EB0101C8EB0001EA
:101730009FE79342D4BFC6EB0303C6EB02037EE6EA
:10174000B8F80010DAF800E0B7F800808E45FFF630
:1017500065AF5DE72988B7F800E020680026C1EB97
:101760000E03B146E9E500BFC09CFF1F609EFF1F4E
:10177000029EFF1F08B5114B1B88022B09D0052BB9
:1017800007D0032B15D0042B0BD00D4B01221A7060
:1017900008BD7F21412007F08FFC094B01221A7000
:1017A00008BD7F21092007F087FC054B01221A7034
:1017B00008BD4021092007F07FFCE6E7BA9CFF1F27
:1017C000789CFF1F38B5074B074D1B88052B044637
:1017D00006D02B68834203D0C1B2052007F06CFC11
:1017E0002C6038BDBA9CFF1F649EFF1F38B5124D98
:1017F000124C2B88052B12D022684AB9022B0ED02E
:10180000033B012B13D90E4A00231370236038BD0C
:101810000021052007F050FC2B88022B04D1002169
:10182000412007F049FCEEE7052BE9D1F7E700215D
:10183000092007F041FCE6E7BA9CFF1F649EFF1FEA
:10184000789CFF1F464B1B881D2B70B541D0454D22
:101850000024454B1B88022B16D0444B1B88022BBF
:1018600054D02888424B002C1B780ADB8442A8BF46
:10187000044634B1002B3AD02046BDE87040FFF753
:10188000A1BF002B2FD170BD3A4B1B78002B37D056
:1018900015200BF075FB384B1860384A1288002A67
:1018A000DBD0374A186811888142D6DC354B2A884C
:1018B0001B888342A3EB0106A8BF03465B1AB24212
:1018C000BABF02FB03330136534393FBF6F31C44C8
:1018D000C3E72A4B1C888CB12B4B224D1C78002C63
:1018E000B7D02C88B5E7BDE87040FFF77FBFFFF7A2
:1018F00041FF2046BDE87040FFF764BF194DA8E7DF
:1019000011200CF081FA1C4B1860C6E70F200CF078
:101910007BFA1A4B1D4A1B881060002BA1D01C4A71
:10192000C0F53B63118808338B429ADB194A28883B
:1019300012889342A2EB0105A8BF1346A842A3EB6D
:10194000010306DA00FB0333013593FBF5F31C4476
:1019500088E700FB03F292FBF5F31C4482E700BF2B
:101960004E9EFF1F529EFF1F229EFF1FB09DFF1F16
:10197000789CFF1F329EFF1F009CFF1FBA9CFF1F19
:10198000769CFF1F4C9EFF1F009EFF1FC89DFF1FE0
:10199000B89CFF1F389EFF1F38B510200CF034FA9A
:1019A000C830B0F5FA7FC0F2EE80B0F57A6F01462C
:1019B000A8BF4FF47A6101F51673B3F57A6FA8BF2B
:1019C0004FF47A639BB289B28E4A8F4C11802220E9
:1019D000238007F0F5FC21888C4D8D4C242007F0E6
:1019E000EFFC0E200BF0CCFA40F6FF71C8308842B5
:1019F000A8BF084620EAE07000F5FA6283B28A4286
:101A0000A8BF0A460220194622802B8007F0D8FC86
:101A10002188042007F0D4FC17200CF0F5F90446C7
:101A200016200CF0F1F9A042B8BF204600F1C80121
:101A3000B1F5FA7FC0F2A280B1F57A6FA8BF4FF47A
:101A40007A6101F54873B3F57A6FA8BF4FF47A63F2
:101A50009BB289B26F4A704C11800A20238007F034
:101A6000AFFC21880C2007F0ABFC0F200CF0CCF968
:101A7000C0F53F610431B1F5AF6F7CDBB1F5FA6FB2
:101A8000A8BF4FF4FA6189B2644BC0F54360B0F56A
:101A9000AF6F19806CDBB0F5FA6FA8BF4FF4FA6036
:101AA00083B25F4CA420238007F08AFCA620218803
:101AB00007F086FC0B200BF07FFF002868D0112078
:101AC0000CF0A2F900F1C801B1F52F7F6EDA40F2F7
:101AD00014534FF42F71534A1180534C0620238026
:101AE00007F06EFC2188082007F06AFC00244FF400
:101AF000AF75E1B24D4809F081FA01348542A8BFC3
:101B000005460C2CF5D101200CF07EF9044600208E
:101B10000CF07AF9323CA0F1320345496FF495702C
:101B200000FB03F300FB04F081FB034281FB004157
:101B3000DB17C017C3EB6223C0EB612003F5AF7264
:101B400000F5AF739342A8BF13469D42A8BF1D4640
:101B5000A5F11401312938DC40F26C73322135488B
:101B6000354A018013602A20BDE8384007F028BCC0
:101B70004FF4AF6395E74FF4AF6185E740F214533C
:101B80004FF4FA7166E740F24C434FF4FA711BE7E9
:101B900015200BF0F5F900F59671B1F52F7F96DB66
:101BA00041F25C2399421FDD194694E741F25C2320
:101BB0009942F9DC1B4A00F5487089B2B0F52F7FD5
:101BC000118019DA4FF42F7387E740F23A72A5F5C6
:101BD000B9751A4B02FB05F583FB0523ED17A5EB41
:101BE000631389B23233BAE70E4A00F5617089B2E5
:101BF000B0F52F7F1180E5DB8342A8BF03469BB27F
:101C00006BE700BFC69DFF1FC29DFF1FB49CFF1F57
:101C10007C9EFF1F189EFF1F389CFF1FB89CFF1F54
:101C2000389EFF1F769CFF1F4C9EFF1FA89CFF1F26
:101C300067BBCF46749EFF1F9489FF1FB5814E1B63
:101C40002DE9F84F0C200BF067F90C200BF01CFE6F
:101C5000A74914200BF028FEA649A74808F060FE0B
:101C6000022103200BF0B6FE022104200BF0B2FE8D
:101C7000022105200BF0AEFE022106200BF0AAFE89
:101C800001210A200BF0A6FE012109200BF0A2FE83
:101C900001210D200BF09EFE012128200BF09AFE61
:101CA000012114200BF096FE02210B200BF092FE76
:101CB00001210C200BF08EFE0C2000210BF076FE93
:101CC00004200BF079FE002836D005200BF074FEBE
:101CD00000283BD00023894D06202B700BF06CFEB2
:101CE000B0FA80F35B090024854A137005F054FFB5
:101CF0002B78EBB9204607F08DFB824B82491B887D
:101D0000824D0988824A2970A3F5AF7140F23A7377
:101D100003FB01F382FB0312DB177E4E7E48A3EB2D
:101D2000621332335A21336009F0A4F9A8B9FEE7EF
:101D3000BDE8F84F08F004BD06200BF03DFE00287A
:101D4000C3D16E4D034628700124CDE703200BF06C
:101D500033FEB0FA80F35B09BDE7704A7048126841
:101D6000DFF804B200230121FEF79EFB0B200BF0ED
:101D700023FE011E0CBF012300238BF8003002D18B
:101D800011200BF027FEDFF8A491664FDFF8DC810D
:101D9000654E0023C9F800303B60C8F800304FF0B2
:101DA000040A14E00BF0ECF83B68184438600AF0C1
:101DB000010080F0010004F04FFB3388002B14BFBA
:101DC0004B20DC200BF02EFEBAF1010A1BD00F20B5
:101DD0000CF01AF8D8F8003003440E20C8F8003090
:101DE0000BF0CEF8D9F800309BF800200344C9F876
:101DF00000301520002AD5D111200CF005F83B68E1
:101E000018443860D3E7D8F80030D9F800204749A3
:101E10003868DFF85CE1DFF85CC1002BB8BF033342
:101E2000002AB8BF033292100A604149414A09882A
:101E300012880028B8BF03309B10801038605F1AEA
:101E40001944CEF80070CCF80010DFF82CE13A4FBE
:101E50003A49C8F80030C2EB000C0244CEF800C08A
:101E60003A600B600CB1FFF797FD33885BB94FF414
:101E7000FA7004F001FB04F0EBFA06F0C1F94FF43C
:101E8000AF600BF0CFFD2E4B012404201C600BF043
:101E900093FD10B92B4B28701C702B4B1B881C2BEF
:101EA0001CD02A4C04F1C80523200BF069F844F833
:101EB000040F01200BF0B6FDA542F5D1244A254BB5
:101EC0001078187007F0B0F904F0BEFA45F6BF526A
:101ED00021492248BDE8F84F0AF00ABE204B188875
:101EE0000028DED01F4BC0B2197807F0E5F8D8E71C
:101EF000001B374640420F00E090FF1F2A9CFF1F47
:101F0000B89DFF1F749EFF1F509EFF1F8C9CFF1FDC
:101F1000B5814E1B9489FF1FA89CFF1F2889FF1FB6
:101F2000E09DFF1FF09BFF1F0E9EFF1F049CFF1FE5
:101F3000A489FF1F2C89FF1F909CFF1F909EFF1FED
:101F4000489EFF1F149CFF1F4E9EFF1FC09CFF1F3B
:101F5000CC9DFF1FAE9DFF1FA50500006C9EFF1FBF
:101F6000949CFF1F449CFF1F329EFF1F3C9EFF1F3F
:101F7000409EFF1FB49DFF1F509CFF1F2DE9F04F97
:101F80008BB007ADC04F2C460AAE611BC9B2BF482B
:101F900009F034F83B88834294BF0020012004F804
:101FA000010BA642F1D1BA48BA4A9DF81C70BA4951
:101FB00007709DF81E00B94D10709DF820209DF807
:101FC0002430B74EB74C0A709DF8221029700025B6
:101FD0003370257073B9002940F01A81B2491AB1E3
:101FE0000B78002B40F00882002800F0DB810223F0
:101FF000237005E0002A40F0BB800523AA49237026
:10200000DFF8F8B2DFF8F8829DF81D209DF8210076
:10201000DFF8F092DFF8F0A2A44DA54FA54E0B70AB
:102020009DF81FC09DF823109DF827309DF826E0ED
:102030008BF8002088F800009DF8252029700120E9
:102040003A70337089F800C08AF800E00BF0DCFECB
:10205000994A9A4B11688842CCBF012200221A701B
:1020600040F38A80964B1B88182B00F28580954A96
:10207000B2F800E00C3B0093BEF1000F40F0858009
:10208000914A9BF800C092F800B098F8008099F847
:1020900000209AF8009094F800A02C78ABEB4C0B41
:1020A000C2EB0B0BA8EB880EDE44C9EB897BC9EBB6
:1020B0008B09DFF81CB2F14497F800E0BBF800B0E0
:1020C00009EB44093478CE4404FB0BEE4FF00C09C5
:1020D0007E4C19FB0AEEC4F800E0B8F1000F0BD0FB
:1020E00036784EB17A4E3688042E0CBF0EF1020EB1
:1020F0000EF1040EC4F800E0764E774CDFF80CB217
:102100003688DBF800B02488DFF804A2DFF80492F8
:10211000BAF800A0B9F80090009BC6EBC6065E4472
:10212000033CDFF8F4B104EB4404DBF800B00EEB41
:1021300084045444C9EBC909DFF8E0A1D944DFF8AD
:10214000E0B15AF826605BF829900C3C1C44A319B6
:102150004B44BCF1000F29D02C783CB3002A5BD152
:10216000B8FA88F85D4C4FEA581884F8008024E0EB
:10217000062323704C4943E7524AB2F800E000239B
:102180000093BEF1000F3FF47BAFBEF1010F47D0CB
:10219000BEF1020F00F0C8804C4C9BF800C099F8CB
:1021A000002098F80080D4F800E096E74B4C00251A
:1021B00025700AB13A781ABB0022494C8842227035
:1021C0004849C4BF484AC2F800E00A68934213D0A5
:1021D000464A474C106805900598206012680692A0
:1021E000444C069A24880B60121AA24284BF424AC9
:1021F00013600BB0BDE8F08F3D483C4A0068EDE746
:10220000BCF1000FD8D1B8F1000FD5D10122D4E72D
:10221000042323702449F3E6304A00241470CBE7EA
:10222000294A9BF800C092F800E098F8008099F8DD
:10223000002094F800B09AF800902C780194AEEB4E
:102240004C0EC2EB0E0EA8EB88047444C9EBC9090E
:10225000D944A31EDFF878A0DFF8C8E0019C97F806
:1022600000B05EF829E0BAF800A096F8009003EB01
:1022700044045C4409FB0A4909F11809134CCE4493
:10228000C4F800E029E700BF749EFF1FA89CFF1F51
:10229000769EFF1F779EFF1F789EFF1F799EFF1F70
:1022A0007A9EFF1FBA9DFF1FC49DFF1FA99EFF1F9F
:1022B000AA9EFF1F549EFF1F9489FF1F009EFF1FB1
:1022C0004E9EFF1FFC9BFF1FA689FF1F089EFF1F3E
:1022D000649CFF1F449EFF1F269EFF1F8A9EFF1FB8
:1022E0008B9EFF1F709CFF1F949EFF1F949FFF1FDC
:1022F000609CFF1F5E9EFF1F9C9EFF1FA59EFF1FF1
:10230000A79EFF1FA69EFF1FA89EFF1FBC9CFF1F2E
:102310000E9CFF1F7A9CFF1F849EFF1F442001001C
:10232000201B010030220100374A9BF800C092F8C0
:1023300000B0247899F8002098F800800394ABEB63
:102340004C049AF80090314B95F800A0CDF804A009
:10235000A8EB880BA41A5C444FF0050B1BFB094B40
:10236000039C97F800A0CDF808A0C9EBC909B3F801
:1023700000A009EB0403BDF80490029C0BF1050BCF
:102380001EFB09BE96F800B0DFF8A490A6440BFB34
:102390000AEE59F823901E4C0EF10C0ECE44C4F8F0
:1023A00000E09AE65FBB0B78012B2BD9194A23700A
:1023B0001288002A3FF424AE174A1288013A92B2DA
:1023C000062A3FF61DAE154A1278002A3FF418AED1
:1023D000134A1268012A7FF413AE1248124A0068A9
:1023E000124E82FB0025C217C2EB650202EB4202CD
:1023F000A0EB8202328003E60323237000E6012370
:102400002370FDE53B46FBE5A689FF1F649CFF1F8B
:10241000089EFF1F309EFF1FCE9DFF1FB69CFF1F13
:10242000489EFF1F9C9EFF1FABAAAA2A0C9EFF1F5F
:10243000C82301002DE9F04F3A4B1B788BB0002BDD
:102440006BD10E200AF09CFD0EF098F8014636483C
:10245000364E374DFEF76EF83348FEF741F80EF072
:10246000A7FA80F30C003060FFF788FD2C68012C80
:102470007AD0022C00F0B182032C00F0C3832D4EE1
:102480002D4C33682D4A2E4E0993099B31681288D2
:102490002360591A013A9142274F00F29982294E3E
:1024A00032689A1A0D2A00F28282274E32689A1AEE
:1024B000132A00F27782254E32689A1A252A1AD9F1
:1024C000234B1B88002B40F05D81224B1B78002B97
:1024D00040F05881FEF7C2FE1F4B1B881B3B9BB28E
:1024E000022B04D81D4B1B78002B40F04E8103F0CB
:1024F000D5FF236833601A4D2A689B1A502B00F2CF
:102500000D82184B1B88012B00F0258206F068FE17
:1025100006F096FC0BB0BDE8F08F07F099FF0BB00A
:10252000BDE8F08F2A9CFF1FE09DFF1F1C9EFF1F30
:10253000489EFF1F949FFF1FDC9DFF1F9089FF1F78
:10254000B09CFF1F9C9CFF1F849CFF1F889CFF1F4B
:10255000C09DFF1F249CFF1F4E9EFF1F009EFF1F5C
:10256000D09DFF1F209EFF1FDFF82093A04AB9F8DF
:1025700000001378834204D0C3B21846137006F0EB
:102580006BFDDFF804839B4AB8F80030117899425C
:1025900004D0994F3978002940F0F286974A336881
:1025A0001288974E9A42C0F2FA80964A1278002A10
:1025B00040F0F580DFF8D8A2BAF8003023B9924B8A
:1025C0001B88002B00F00685904A914B11881B88D0
:1025D000904A0B4412685B1093428F4A126880F253
:1025E000A88400219342B4BF01230B4604910093B9
:1025F000ACBF4FF0010B8B4605910E200AF0C0FCDA
:10260000864B874A1B68176803930133A7F252323F
:10261000002B8446029240F3DA86802BA8BF8023E9
:10262000804A814912780191002A00F0C28009781D
:10263000914200F0BE80B8F80010DFF84CE29942F9
:1026400001F0F7806C49AEF80030784B4FF0010E86
:1026500081F800E01978DFF83CE2019B8EF8001069
:102660001A70009B002B00F01781BAF80030002B85
:1026700000F012816E4B1B685A1C002A40F3AB8697
:10268000802A00F3A7866B4C6B496C482488098824
:1026900000682144B0EB610FC1F24083A3F148020E
:1026A0000F2A02D8473BA9F800300E200AF068FC38
:1026B0006FF454731F44874202DC614B00221A708E
:1026C00000200BF0A1FB5F4A5F4B11685F4C1B8839
:1026D0008842D4BF002201222270002B00F0208407
:1026E0005B4B1C78944240D088423EDD59490C78BF
:1026F000002C00F03487584991F800C0BCF1000F5D
:1027000040F02B87554F0097554F56480297534F2F
:10271000007887F800C0524F4FF0010E87F800C0D4
:1027200081F800E0002841F0DB804F49097800295A
:1027300000F0F7874D4903910C460978002940F0D5
:10274000ED874B48464F0078397001210297217080
:1027500058B1424840490090002008700099029FFB
:102760000870039901243C7008701A70414B1B8853
:10277000A3F11B02012A40F2C7851D2B00F0118630
:102780003D4C7EE6FEF70CFDA4E63C4B1B78002B8F
:102790003FF4ADAE2B68012B7FF4A9AEA9E63168FA
:1027A000374A069106983749106002220B602A606A
:1027B00000E71E49DFF8DCE0097800293FF44DAF5F
:1027C0009EF8000081423FF448AF03984B2840F345
:1027D000F7871833802BB8F80000A8BF80239842F1
:1027E0003FF43BAF2848038003480123037034E7DC
:1027F000AE9DFF1F8C9CFF1F149CFF1FB49CFF1FEE
:10280000949FFF1F249CFF1FA29CFF1F389CFF1F4B
:10281000189EFF1F589CFF1F1C9CFF1F949EFF1FAC
:10282000049CFF1F8A9EFF1F6C9CFF1F8B9EFF1F37
:10283000089EFF1FC69DFF1FC29DFF1F489CFF1FD4
:10284000B99DFF1F9489FF1FCE9DFF1F3E9CFF1F58
:10285000F49BFF1FA89EFF1F109EFF1F629EFF1F7D
:10286000B69CFF1FA99EFF1FA59EFF1FF59BFF1F84
:10287000009EFF1F4E9EFF1FDC9DFF1F549EFF1FEB
:102880007C9CFF1FD89DFF1F509EFF1FCC9DFF1FEC
:10289000749CFF1F6D9CFF1F029B9C45BFF605AFFC
:1028A0008B4B1B88002B3FF400AFBBF1000F7FF474
:1028B000E1AE884B1B881BB1059B002B7FF4DAAE81
:1028C000049B002B3FF4F1AE834B1A78002A7FF46F
:1028D000ECAEDFF8809299F8004001221A70002CCB
:1028E00040F045837D4B1B78002B02F0D8807C4B59
:1028F0001B78002B02F09B837A4B1B78002B7FF414
:10290000D4AE794B1B78002B3FF4CFAEB8F8003033
:1029100076490A3BA8F800300A70C6E605F084F94B
:10292000734B1B7873B9734B1B785BB9724B1B7875
:1029300043B9724B1B782BB9714B1B7813B903F059
:1029400083FD01E003F08CFD23682B606D4B1B8839
:10295000012B7FF4DBAD6C4A6C4B11686C481A7824
:10296000A1F118032A2101FB03F10160002A00F004
:10297000C182684C2368994200F36A8310DA664882
:102980000278002A40F09287644A1068D0F17F00F4
:1029900048BF0330801001301B1A994242F3D086A1
:1029A0002160A9E2FEF74EFF2368336083E5FDF75F
:1029B000E7FFFEF77FFC5A4B1B88032B00F02B85AB
:1029C000584B1B88032B00F02285236833606CE58D
:1029D000FDF722FF3B68336061E5534A3468118894
:1029E000A14204DB464B1B78002B00F061834F4E65
:1029F0004F48336807934F4B079A00681B88121A99
:102A00009A4200F2AD80002B00F0AA804A4B1A884F
:102A1000002A3FF4B5AE494B49481B680088A342E1
:102A2000B8BF2346994241F37281464B1960DFF8E3
:102A3000288188F80020344FFDF7EEFE38687F28A3
:102A400040F37D85404B7F3883FB0032C317C3EBD7
:102A5000620303EB4303A0EB830073303B4B019312
:102A60001B883860002B40F0D686234B00931B78E0
:102A7000002B00F0CA83364C2378002B00F0C5836E
:102A8000DFF8D890DFF8C0A04FF0000B0CE003F1A6
:102A90007300C0B298F8001006F036FB23780BF1F3
:102AA000010B5B4540F3B1833B6859F8040F1844B0
:102AB000A0F17F038AFB0321DA17C2EB610202EB6C
:102AC00042027F28A3EB8203E1DCFDF7C5FDE0E7CE
:102AD000A29CFF1FD49DFF1FB99DFF1FA59EFF1F36
:102AE000A69EFF1FA79EFF1FA89EFF1F149CFF1FEF
:102AF000B69CFF1F109EFF1F629EFF1FF59BFF1FCE
:102B0000249CFF1F209EFF1F9C9EFF1F789CFF1F81
:102B1000809EFF1FA49CFF1F689EFF1F649EFF1FD7
:102B2000229EFF1FB09DFF1FB49CFF1F949FFF1F9D
:102B30007C9CFF1FA09CFF1F129CFF1FD89DFF1FA6
:102B40007C9EFF1FF89BFF1FABAAAA2A549CFF1F65
:102B50005489FF1FBA9DFF1F989CFF1F2C89FF1FE0
:102B6000554B564A1B681088554AA342B8BF2346A6
:102B7000994200F38482534C12888342A8BF0346D3
:102B80002360002A7FF453AF9942C8BF134640F335
:102B90007D82401AB0F5804FAABF9B03C3EB8333FD
:102BA000013093FBF0F0FDF71DFEC0F3C6100DF0F1
:102BB000E5FC454B044618880DF0E0FC4349074608
:102BC00020460DF02FFD014638460DF02BFD214625
:102BD0000DF020FC4FF07E5104460DF0C1FE0028A0
:102BE00041F079803A4920460DF0D8FE002840F0A7
:102BF000718620460DF002FFC0B2DFF8F48088F83D
:102C0000000018E7334B34681988A14274DD324B59
:102C10001B78002B70D1DFF8DC9099F800007F283A
:102C200040F34086A3F155337F3803F1004383FB23
:102C30000032C317C3EB620303EB4303A0EB830033
:102C40007330264B01931B88C0B289F80000002B1B
:102C500041F03380224B00931B78002B00F0AC84B2
:102C6000204C2378002B00F0A7841F4FDFF87C80D6
:102C70004FF0000A0AE003F17300C0B206F06CFAEC
:102C800023780AF1010A534540F3968457F8043F2C
:102C900099F800001844A0F17F0388FB0321DA179C
:102CA000C2EB610202EB42027F28A3EB8203E2DC6B
:102CB000FDF7D2FCE1E700BFD89DFF1F7C9EFF1F00
:102CC000129CFF1FF89BFF1F8C9EFF1FCDCCCC3D9D
:102CD0000000FE42B49CFF1F249CFF1F549CFF1F5A
:102CE000629EFF1F5489FF1F2C89FF1FABAAAA2ACF
:102CF000989CFF1F049EFF1FB84F38687F2840F341
:102D0000CC81B74B7F3883FB0032C317C3EB620320
:102D100003EB4303A0EB83007330DFF8249399F8AF
:102D200000A0824500F01782AE4B1B88002B43D1D8
:102D3000AD4AAE4812680088914205DC8242D4BF99
:102D4000C1EB0203C1EB0003411AB1F5804FA6BFEE
:102D50009B030131C3EB833393FBF1F0FDF742FD9D
:102D6000C0F3C6100DF00AFCA14B044618880DF004
:102D700005FCA049804620460DF054FC0146404623
:102D80000DF050FC21460DF045FB4FF07E510446FE
:102D90000DF0E6FD002840F00A87974920460DF027
:102DA000FDFD002840F0938520460DF027FEC0B2BF
:102DB000DFF8908288F80000BAF17F0F40F3B88303
:102DC0008748AAF17F0A80FB0A304FEAEA73C3EB17
:102DD000600000EB4000AAEB80007330874B00934B
:102DE0001B78C0B289F80000002B40F01883844B98
:102DF00003931B78002B40F04985824B02931B788C
:102E0000002B40F07C87804B0193029B1B78FBB129
:102E10007E4B1B88012B00F0C185022B01F04D80F9
:102E2000032B01F08C81042B01F09783052B01F01B
:102E30003884062B01F0FF85072B01F0BB87082B98
:102E400002F0BA80092B02F0BF810A2B02F09283B4
:102E5000009B1B78002B00F07484019B6A4C19883E
:102E6000002900F0FB8438687F2840F365835C4BC1
:102E70007F3883FB0032C317C3EB620303EB4303CA
:102E8000A0EB830073303860002940F0AA84009BD7
:102E90001B78002B00F06B815D4C2378002B00F039
:102EA0006681DFF8A4A1DFF89C814FF0000B0CE0F5
:102EB00003F17300C0B298F8001006F025F92378EA
:102EC0000BF1010B5B4540F352813B685AF8040F4C
:102ED000434A1844A0F17F0382FB0321DA17C2EBB7
:102EE000610202EB42027F28A3EB8203E0DCFDF7E4
:102EF000B3FBDFE7474B1960474B1B68A92202FB76
:102F000003F3002BBCBF03F57F533F339B13543BAC
:102F1000194481F30C0128200AF0B8FBFFF7F6BA38
:102F2000384C3E483549364A237003700B70137095
:102F30001CE493424FF0000B80F2B2800123CDF8E5
:102F400000B0CDF814B00493FFF757BB344B1B7897
:102F5000002B7FF4AAAB039B324A243B83F3470345
:102F6000D9B25B20136006F0A7F899F80040032C53
:102F700030D1DFF8D88098F80030002B42F05D8225
:102F8000294F3B78002B42F04B82254C2378002BB5
:102F900042F03982254B1B78002B42F02782244ACD
:102FA0001380244B1B78002B42F013820D4B7F22A1
:102FB0001A8098F800306BB93B785BB923784BB92D
:102FC0001D4A7F210720138006F076F87F210B2011
:102FD00006F072F8194B1F68FFF767BB9C9EFF1F36
:102FE000ABAAAA2A129CFF1FF89BFF1F7C9EFF1F03
:102FF0008C9EFF1FCDCCCC3D0000FE42629EFF1F89
:10300000F59BFF1FB69CFF1F549CFF1FCE9DFF1F0B
:103010005489FF1FA49CFF1F8C89FF1F109EFF1F58
:10302000A89EFF1F349CFF1FA79EFF1FA69EFF1F89
:10303000AA9CFF1FA99EFF1F029EFF1F049CFF1F4B
:10304000049EFF1F989CFF1F2C89FF1FA59EFF1F3A
:10305000B64A1078002840F05783B54A1268D2F17A
:103060007F0248BF033203EBA202531CB14A236024
:103070009942B8BF1160FFF63FAF19463CE7AE4B2F
:1030800012881960002A7FF4D2AC0B469842D4BF54
:10309000C1EB0003C1EB03037BE5FDF7DDFA3CE682
:1030A0000123CDF810B0CDF800B00593FFF7A5BA15
:1030B00001232B60A14EA24CFFF7E3B9029B1B78C2
:1030C000FBB1A04B1B88012B00F0EA84022B00F01F
:1030D0007386032B01F0A980042B01F06382052B7A
:1030E00001F05683062B01F0AF84072B01F0AF856A
:1030F000082B01F01987092B02F02F800A2B02F010
:10310000C381019B1B88002B00F07483009B1B78FC
:103110003BB9039B1B7823B9029B1B78002B01F062
:103120000480894B1B78002B00F0FE8087490B78C8
:10313000082B00F2F98086483A680068854C013314
:10314000DBB25F1E101A44F827000B70824B346804
:10315000198889F800208C42784E7FF711AB3268CD
:103160007E4B0892089A764C1A60FFF78AB9039B47
:103170001B78002BA2D03B68A3F10C007F2840F302
:10318000828377488B3B80FB0320DA17C2EB600019
:1031900000EB4000A3EB800303F17300DFF8D48160
:1031A000C0B298F8001005F0AFFF009B1B78002B11
:1031B00084D0664C2378002B80D0DFF8BCA14FF080
:1031C000000B0CE003F17300C0B298F8001005F09A
:1031D0009BFF23780BF1010B5B457FF76FAF3B68DB
:1031E0005AF8040F5E4A1844A0F18B0382FB0321B6
:1031F000DA17C2EB61020C3802EB42027F28A3EB24
:103200008203DFDCFDF728FADEE74F4B1B78002B4B
:1032100040F0F6823B68534A1278002A45D0A3F169
:103220000C007F2840F33B834D4A8B3B82FB0321FC
:10323000DA17C2EB610202EB4202A3EB820303F155
:103240007300C0B298F8001005F05EFF009B1B7879
:1032500053B33E4C23783BB3DFF81C91DFF800A159
:103260004FF0000B0BE003F17300C0B298F80010B0
:1032700005F04AFF23780BF1010B5B4514DD3B6839
:1032800059F8040F1844A0F18B038AFB0321DA17C5
:10329000C2EB61020C3802EB42027F28A3EB8203EF
:1032A000E1DCFDF7D9F9E0E73B682F4A1278FAB183
:1032B000244A1288012A00F07D84022A00F07B86CD
:1032C000032A01F02F80042A01F09381052A01F0DE
:1032D000CC82062A01F0D083072A01F01384082A41
:1032E00001F0D386092A01F090870A2A02F00A81A8
:1032F000019A1288002A00F095821C4A104C137023
:1033000003232B60FFF7BDB8DFF8708098F800301A
:10331000002B40F01881164F3B78002B40F01485AD
:10332000074C3B70FFF7ADB83A680FE7689EFF1F88
:10333000649EFF1FA49CFF1FF89BFF1F949FFF1F0D
:10334000DC9DFF1FCE9DFF1F109EFF1F5489FF1F96
:10335000189CFF1F3089FF1FB49CFF1F409FFF1F59
:10336000ABAAAA2AF59BFF1FB69CFF1F049EFF1F56
:10337000109CFF1F989CFF1F2C89FF1F009EFF1FA2
:10338000DBB21846137005F075FEB04BB0491A4613
:10339000B04B184600230B703B7013700370FFF79F
:1033A000FDB8DFF8CC8298F80030002B40F0D781D0
:1033B000A94F3B78002BB3D0A84BA94C1988A22069
:1033C00005F0FEFF98F800303B70FFF75AB8012374
:1033D000FFF726B98024A349A34BA44A09881B8878
:1033E00012680B44B2EB630FBFF65FA9A04B1B78CA
:1033F000002B40F02482B8F800309E4AA3423FF4EC
:1034000054A99D4B148001221A70FFF74EB9FDF7A5
:103410008BF9FFF7DABAFDF731F9FFF7D1BA974B1D
:1034200001931B88002B42F085818A4B0393944BB8
:103430000293944C23786BB3DFF85C82DFF848A2E8
:103440004FF0000B09E003F17300C0B205F084FEF9
:1034500023780BF1010B5B451CDD58F8043F99F80C
:1034600000001844A0F17F038AFB0321DA17C2EBA6
:10347000610202EB42027F28A3EB8203E3DCFDF74B
:10348000EBF8E2E77E4B029305F066FE009B1B78AB
:10349000002BCED1039B1B78002B3FF4B6AC99F8E0
:1034A0000030A3F10C007F2840F3EA8176488B3B83
:1034B00080FB0320DA17C2EB600000EB4000A3EBB7
:1034C000800303F17300C0B205F046FE009B1B7839
:1034D000002B00F0CA816B4C2378002B01F0C582D1
:1034E000DFF8B481DFF8A0A14FF0000B0AE003F190
:1034F0007300C0B205F030FE23780BF1010B5B4581
:103500007FF783AC58F8043F99F800001844A0F105
:103510008B038AFB0321DA17C2EB61020C3802EB42
:1035200042027F28A3EB8203E1DCFDF795F8E0E798
:103530005046FDF791F851E4FDF78EF8A3E4FDF74E
:103540008BF8FFF78BBA514A1278002A40F0D581E8
:10355000414F434C3B70FEF794BF002008704C492C
:10356000087840B1394900910978002900F0B58107
:10357000009F002139704749097800297FF4DAA8B3
:10358000002C40F0CE80002840F0CB80384C2F4FEC
:1035900094F800E02F4C0394394C02942D4C2C49A4
:1035A0002070374C0097087038702070BEF1000F03
:1035B0007FF4D2A8FFF7D9B8264B1B78002B6DD02B
:1035C00099F80030A3F10C007F2840F3C8832E4AFD
:1035D0008B3B82FB0321DA17C2EB610202EB420252
:1035E000A3EB820303F17300C0B205F0B5FD009BAD
:1035F0001B78002B52D0234C2378002B4ED0264F23
:10360000DFF884804FF0000A09E003F17300C0B2D4
:1036100005F0A2FD23780AF1010A53453EDD57F873
:10362000043F99F800001844A0F18B0388FB0321A4
:10363000DA17C2EB61020C3802EB42027F28A3EBDF
:103640008203E2DCFDF708F8E1E700BF629EFF1F9E
:10365000109EFF1FF59BFF1F109CFF1F529EFF1F18
:10366000DC9DFF1FC69DFF1FC29DFF1F489CFF1FC3
:10367000009EFF1F509EFF1F149CFF1F549CFF1FA6
:10368000B69CFF1F5489FF1FABAAAA2A549EFF1F96
:10369000A99EFF1FA59EFF1F2C89FF1FA84B1B780B
:1036A000FBB1A84B1B88012B00F0D086022B00F049
:1036B000CB87032B01F04281042B01F0CD81052B38
:1036C00001F01784062B01F0D884072B01F0E78561
:1036D000082B01F07087092B01F0D5870A2B01F028
:1036E000A287019B1B88002B00F0F082964B1B7871
:1036F000002B40F0E682954B954A198834680020EB
:10370000012310602B6026E50130C0B2022886BF7D
:103710000021117010701946FFF7EEBB03980021CD
:1037200001708C49097800293FF41FA8844902914F
:103730000978002900F0AE87029800210170FFF798
:1037400014B8039B1B78002B7FF487AB029B1B787C
:10375000002B7FF482AB019B1988FFF784BB7E4A64
:103760001278002A3FF4F4AE7C4F387802F0E6FE7F
:103770007B4B1B78002B00F0B78439887E2900F240
:10378000B384784CDFF80C922368D9F800209B1A98
:103790000F2B40F29680744B01311B8889B239801F
:1037A0002BB1052B03D0C9B2052005F085FC6F4F66
:1037B000226898F80030C9F800203B70FEF761BE1F
:1037C000243B002BB8F8000040F3748498423EF488
:1037D00044AF9BB26648A8F8003001230370FEF79F
:1037E0003CBFDFF89081C0B298F8001005F08CFC67
:1037F000FFF74DBB5F4B3878197805F085FC85E401
:103800007F21402005F058FC5B495C4A3B680B6017
:1038100000211170FFE4C0B298F8001005F074FCAC
:10382000FFF723B9D8B298F8001005F06DFC3B689B
:1038300063E5534BDFF860E11978FEF70EBF4B2CC0
:1038400040F34C821834802CB8F800304D4AA8BFA1
:103850008024A3427FF4D5ADFEF727BF99F800007E
:1038600005F07AFC2188FFF7FEBA029B1B78002B3B
:103870007FF4CEAA039B1B78002B7FF4EEAA6AE7A5
:10388000FCF7EAFE1FE6FCF7E7FE87E43E4B0193F8
:103890001B88002B7FF4F6AD294B0293FFE5FCF764
:1038A000DBFECEE4FCF7D8FEFFF7CBB90132D2B293
:1038B000022A40F25A82002202701946FFF71CBB0E
:1038C000284C2A4F98F800303B70FEF7DABD7F2075
:1038D000FFF76EBA7F20FFF790B9194F1A49029788
:1038E0004FF0000C81F800C0009F02994FF0010ECC
:1038F00087F800E081F800C03DE6244F387802F0F8
:103900001DFE174B1B78002B00F0368239887E296C
:1039100000F23282134CDFF87C902368D9F8002043
:103920009B1A0F2BCDD91A4B0131188889B23980D7
:10393000002800F03D82C9B2C0B205F0BDFB36E7F9
:10394000B69CFF1FCE9DFF1F109EFF1FB49CFF1F44
:10395000F89BFF1F009EFF1F549EFF1F529EFF1FDC
:10396000AA9EFF1FDC9DFF1FBA9CFF1F109CFF1F1C
:10397000149CFF1F989CFF1F189CFF1F5489FF1F5A
:103980008B9EFF1F509EFF1F549CFF1F449CFF1FD8
:10399000949CFF1F989EFF1F6D9CFF1FDFF89CA348
:1039A00099F80000BAF80030DF4AE04CC31A82FBF5
:1039B000031ED917C1EB6E0101EB4101A3EB81039B
:1039C00003EB430354F8233018447F2840F3A684C4
:1039D0007F3882FB0032C317C3EB620303EB430360
:1039E000A0EB83007330DFF858B3C0B205F0B4FB2E
:1039F000BBF80030022B7FF62BAA99F80010BAF81A
:103A00000030C94ACB1A82FB030ED817C0EB6E00F8
:103A100000EB4000A3EB800303EB430304EB8303C1
:103A2000586808447F2840F318877F3882FB0032AB
:103A3000C317C3EB620202EB4202A0EB82007330B9
:103A4000C0B205F089FBBBF80030032B7FF600AA5B
:103A500099F80010BAF80030B34ACB1A82FB030E73
:103A6000D817C0EB6E0000EB4000A3EB800303EB24
:103A7000430304EB8304A06808447F2840F351818A
:103A80007F3882FB0032C317C3EB620202EB4202B3
:103A9000A0EB82007330C0B205F05EFBFFF7D8B92F
:103AA000DFF898A23868BAF800309F4A9F4CC31AD2
:103AB00082FB031ED917C1EB6E0101EB4101A3EBA1
:103AC000810303EB430354F8233018447F2840F369
:103AD000A0847F3882FB0032C317C3EB620303EB81
:103AE0004303A0EB83007330DFF85882DFF850B255
:103AF00098F80010C0B205F007FBBBF80030022BAD
:103B00007FF6FFAA3968BAF80030874ACB1A82FBE1
:103B1000030ED817C0EB6E0000EB4000A3EB800350
:103B200003EB430304EB8303586808447F2840F306
:103B300098867F3882FB0032C317C3EB620202EB28
:103B40004202A0EB82007330C0B298F8001005F07A
:103B5000DBFABBF80030032B7FF6D3AA3968BAF83A
:103B60000030714ACB1A82FB030ED817C0EB6E00EF
:103B700000EB4000A3EB800303EB430304EB83045F
:103B8000A06808447F2840F3F4807F3882FB00322D
:103B9000C317C3EB620202EB4202A0EB8200733058
:103BA00098F80010C0B205F0AFFAFFF7AABA0120EA
:103BB000FFF7FEB8DFF884A15B49BAF800205B4C40
:103BC0009A1A81FB020ED017C0EB6E0000EB40008A
:103BD000A2EB800202EB420254F8220018447F2834
:103BE00040F31B84A0F17F0381FB0321DA17C2EBB2
:103BF000610000EB4000A3EB80007330DFF840B1C0
:103C000098F80010C0B205F07FFABBF80030022B24
:103C100050D93968BAF80030434ACB1A82FB030EF8
:103C2000D817C0EB6E0000EB4000A3EB800303EB62
:103C3000430304EB8303586808447F2840F3E1867C
:103C40007F3882FB0032C317C3EB620202EB4202F1
:103C5000A0EB82007330C0B298F8001005F054FA5F
:103C6000BBF80030032B25D93868BAF800302E4A4B
:103C7000C31A82FB031ED917C1EB6E0101EB410190
:103C8000A3EB810303EB430304EB8304A368184411
:103C90007F2867DD7F3882FB0032C317C3EB6202E7
:103CA00002EB4202A0EB82007330C0B298F8001021
:103CB00005F02AFA3B68FFF71BBB05F04DFAFEF74B
:103CC000C9BF0021402005F0F7F914E599F800007C
:103CD00005F042FA0AE50120FEF78FBF243C002CD4
:103CE000B8F8003040F32486A3423EF4DEACA4B220
:103CF0000F4BA8F8004001221A70FEF7D6BC0D4BFE
:103D000001931B88002B7FF4BFABFFF77EB80A49F5
:103D10008342A8BF03460B60FEF789BE1446FFF737
:103D200065BBFCF799FCB6E6ABAAAA2A241F0100E2
:103D3000149CFF1F549CFF1FF89BFF1F0C9EFF1F2E
:103D4000289CFF1F989CFF1FDD4BDE4C19886A20C2
:103D500005F036FB98F800303B70FEF792BBFCF79D
:103D60007BFC41E4FCF778FC9FE702701946FFF703
:103D7000C3B8FCF771FC13E7D34B1B78002B3FF45F
:103D80009FAD3B88CE4F002B3FF49AADCD4CDFF872
:103D900048932268D9F80010521A0F2A7FF691AD85
:103DA000CA4A013B108899B2398000287FF4C3AD1C
:103DB000C8B205F0F5F9FAE4DFF820A33868BAF8DC
:103DC0000030C34AC34CC31A82FB031ED917C1EB90
:103DD0006E0101EB4101A3EB810303EB430354F8B4
:103DE000233018447F2840F328847F3882FB003238
:103DF000C317C3EB620303EB4303A0EB83007330F1
:103E0000DFF8DC82DFF8DCB298F80010C0B205F011
:103E10007BF9BBF80030022B7FF673A93968BAF83A
:103E20000030AB4ACB1A82FB030ED817C0EB6E00F2
:103E300000EB4000A3EB800303EB430304EB83039D
:103E4000586808447F2840F326867F3882FB00327A
:103E5000C317C3EB620303EB4303A0EB8300733090
:103E6000C0B298F8001005F04FF9BBF80030032BF2
:103E70007FF647A93868BAF80030954AC31A82FB22
:103E8000031ED917C1EB6E0101EB4101A3EB8103C6
:103E900003EB430304EB8304A36818447F287FF7F4
:103EA00068AF7F3882FB0032C317C3EB620303EBBA
:103EB0004303A0EB8300733072E6DFF820A299F889
:103EC0000000BAF80030824A824CC31A82FB031EFB
:103ED000D917C1EB6E0101EB4101A3EB810303EBA9
:103EE000430354F8233018447F2840F37F837F38FE
:103EF00082FB0032C317C3EB620303EB4303A0EB67
:103F000083007330DFF8DCB1C0B205F025F9BBF8EF
:103F10000030022B7EF69CAF99F80010BAF8003002
:103F20006B4ACB1A82FB030ED817C0EB6E0000EB76
:103F30004000A3EB800303EB430304EB83035868C7
:103F400008447F2840F39F857F3882FB0032C317E7
:103F5000C3EB620303EB4303A0EB83007330C0B2F7
:103F600005F0FAF8BBF80030032B7EF671AF99F834
:103F70000010BAF80030564ACB1A82FB030ED8174D
:103F8000C0EB6E0000EB4000A3EB800303EB4303A8
:103F900004EB8304A06808447F287FF7C2AE7F3813
:103FA00082FB0032C317C3EB620303EB4303A0EBB6
:103FB000830073306FE5DFF824A14549BAF800208B
:103FC000444C9A1A81FB020ED017C0EB6E0000EB36
:103FD0004000A2EB800202EB420254F82200184497
:103FE0007F2840F32E83A0F17F0381FB0321DA17A2
:103FF000C2EB610000EB4000A3EB80007330DFF800
:10400000E4B098F80010C0B205F07EF8BBF80030BC
:10401000022B7FF64FAE3968BAF800302C4ACB1A23
:1040200082FB030ED817C0EB6E0000EB4000A3EB41
:10403000800303EB430304EB8303586808447F28A1
:1040400040F325857F3882FB0032C317C3EB620340
:1040500003EB4303A0EB83007330C0B298F8001069
:1040600005F052F8BBF80030032B7FF623AE38681A
:10407000BAF80030164AC31A82FB031ED917C1EBE7
:104080006E0101EB4101A3EB810303EB430304EB5E
:104090008304A36818447F287FF764AE7F3882FBCF
:1040A0000032C317C3EB620303EB4303A0EB8300AF
:1040B0007330FAE501283EF4D0AA0123FFF78ABB4A
:1040C000449CFF1FDC9DFF1FA99EFF1F949CFF1FA8
:1040D000ABAAAA2AEC200100989EFF1F0C9EFF1F8E
:1040E000989CFF1F289CFF1FCE4B1B78002B3FF492
:1040F000E7AB3B88CC48002B3FF4E2ABCB4CDFF87E
:104100003C932268D9F80010521A0F2A7FF6D9ABD7
:10411000C74A013B128899B20180002A3FF447AB9D
:10412000052A7FF440ABFFF742BB4FF47A43013BD3
:10413000FDD199F8000005F00FF8FEF7F2BFDFF8A7
:1041400000A399F80000BAF80030BA4ABA4CC31A72
:1041500082FB031ED917C1EB6E0101EB4101A3EBFA
:10416000810303EB430354F8233018447F2840F3C2
:10417000E8817F3882FB0032C317C3EB620202EB97
:104180004202A0EB82007330DFF8B8B2C0B204F094
:10419000E3FFBBF80030022B7EF65AAE99F8000020
:1041A000BAF80030A34AC31A82FB0321DA17C2EB24
:1041B000610202EB4202A3EB820303EB430304EB35
:1041C00083035B6818447F2840F325847F380C22E2
:1041D00090FBF2F302FB13007330C0B204F0BCFF9B
:1041E000BBF80030032B7EF633AE99F80000BAF826
:1041F0000030904AC31A82FB0321DA17C2EB610236
:1042000002EB4202A3EB820303EB430304EB8304C0
:10421000A36818447F287FF784AD7F380C2290FB79
:10422000F2F302FB1300733035E4DFF814A23868B0
:10423000BAF800307F4A804CC31A82FB031ED9179C
:10424000C1EB6E0101EB4101A3EB810303EB4303DF
:1042500054F8233018447F2840F370817F3882FB64
:104260000032C317C3EB620202EB4202A0EB8200F2
:104270007330DFF8D481DFF8CCB198F80010C0B209
:1042800004F042FFBBF80030022B7EF63AAF3868EC
:10429000BAF80030674AC31A82FB0321DA17C2EB6F
:1042A000610202EB4202A3EB820303EB430304EB44
:1042B00083035B6818447F2840F3B4837F380C2263
:1042C00090FBF2F302FB13007330C0B298F80010B9
:1042D00004F01AFFBBF80030032B7EF612AF3868EB
:1042E000BAF80030534AC31A82FB0321DA17C2EB33
:1042F000610202EB4202A3EB820303EB430304EBF4
:104300008304A36818447F287FF733AD7F380C22DD
:1043100090FBF2F302FB1300733041E4FCF79CF9CD
:10432000FFF761BBDFF818A14249BAF80020424C00
:104330009A1A81FB020ED017C0EB6E0000EB400012
:10434000A2EB800202EB420254F8220018447F28BC
:1043500040F3FA80A0F17F0381FB0321DA17C2EB5F
:10436000610101EB4101A3EB81007330DFF8D4B0B0
:1043700098F80010C0B204F0C7FEBBF80030022B62
:104380007FF698AC3868BAF800302A4AC31A82FB24
:104390000321DA17C2EB610202EB4202A3EB8203B4
:1043A00003EB430304EB83035B6818447F2840F36B
:1043B0003C837F380C2290FBF2F302FB1300733036
:1043C000C0B298F8001004F09FFEBBF80030032B39
:1043D0007FF670AC3868BAF80030164AC31A82FB10
:1043E0000321DA17C2EB610202EB4202A3EB820364
:1043F00003EB430304EB8304A36818447F287FF78F
:10440000B1AC7F380C2290FBF2F302FB1300733047
:104410004BE4FCF721F9FFF767BBFCF71DF9FFF749
:10442000EDBB00BFA99EFF1F529EFF1FDC9DFF1F1B
:10443000BA9CFF1FABAAAA2A7C210100989EFF1FED
:104440000C9EFF1F289CFF1F989CFF1FDFF838A3BE
:1044500099F80000BAF80030C34AC44CC31A82FB72
:104460000317D917C1EB670101EB4101A3EB8103EE
:1044700003EB430354F8233018447F286ADD7F3868
:1044800082FB0032C317C3EB620202EB4202A0EBD5
:1044900082007330DFF8F4B2C0B204F05DFEBBF806
:1044A0000030022B7FF61DA999F80000BAF8003001
:1044B000AD4AC31A82FB0321DA17C2EB610202EB99
:1044C0004202A3EB820303EB430304EB83035B6829
:1044D00018447F2840F3AC827F380C2290FBF2F323
:1044E00002FB13007330C0B204F036FEBBF800309C
:1044F000032B7FF6F6A899F80000BAF800309A4A24
:10450000C31A82FB0321DA17C2EB610202EB4202FB
:10451000A3EB820303EB430304EB8304A368184477
:104520007F2814DD7F380C2290FBF2F302FB13008E
:104530007330C0B204F010FEFFF7D3B8FCF78CF86C
:1045400097E6FCF789F81FE6FCF786F80EE7FCF71C
:1045500083F8EEE7FCF780F89CE7DFF82CA299F8E7
:104560000000BAF80030804A814CC31A82FB031E57
:10457000D917C1EB6E0101EB4101A3EB810303EB02
:10458000430354F8233018447F28DADD7F3882FB58
:104590000032C317C3EB620303EB4303A0EB8300BA
:1045A0007330F1E5DFF8E0A13868BAF800306E4A00
:1045B0006F4CC31A82FB031ED917C1EB6E0101EBCE
:1045C0004101A3EB810303EB430354F82330184468
:1045D0007F28B3DD7F3882FB0032C317C3EB620351
:1045E00003EB4303A0EB8300733042E6FCF734F89F
:1045F00088E4DFF894A15C49BAF800205C4C9A1A70
:1046000081FB020ED017C0EB6E0000EB4000A2EB66
:10461000800202EB420254F8220018447F2893DD06
:10462000A0F17F0381FB0321DA17C2EB610000EBED
:104630004000A3EB8000733098E6FCF70DF8FFF71D
:10464000DFBBFCF709F8DAE4DFF83CA199F80000D9
:10465000BAF80030444A474CC31A82FB0317D917F3
:10466000C1EB670101EB4101A3EB810303EB4303C2
:1046700054F8233018447F287FF76CAF7F3882FBD3
:104680000032C317C3EB620303EB4303A0EB8300C9
:104690007330FFE638480090384839490390FEF7F8
:1046A0005BB8DFF8E4A099F80000BAF800302E4AB1
:1046B000344CC31A82FB0321DA17C2EB610202EB0E
:1046C0004202A3EB820303EB430354F82330184464
:1046D0007F2840F3A4817F380C2290FBF2F302FB89
:1046E00013007330DFF8A4B0C0B204F035FDBBF89E
:1046F0000030022B19D999F80000BAF800300C22CA
:10470000C11A91FBF2F302FB131302FB03435B6834
:1047100018447F2840F384847F3890FBF2F302FB37
:1047200013007330C0B204F017FDBBF80030032B48
:104730007EF68EABBAF8003099F800000C22C11A50
:1047400091FBF2F302FB131302FB0344A36818442A
:104750007F287FF7E6AA7F3890FBF2F302FB130075
:104760007330FFF798B900BFABAAAA2A241F010033
:10477000901B0100EC200100629EFF1FF59BFF1FB4
:10478000109EFF1F002401000C9EFF1F289CFF1F8E
:10479000DFF864A33868BAF80030CE4ACE4CC31AAA
:1047A00082FB0321DA17C2EB610202EB4202A3EBA8
:1047B000820303EB430354F8233018447F2840F36B
:1047C00024817F380C2290FBF2F302FB130073303C
:1047D000DFF82883DFF828B398F80010C0B204F09F
:1047E00093FCBBF80030022B1AD93868BAF80030B5
:1047F0000C22C11A91FBF2F302FB131302FB0343D9
:104800005B6818447F2840F3D4837F3890FBF2F331
:1048100002FB13007330C0B298F8001004F074FC6F
:10482000BBF80030032B7EF66CACBAF80030386869
:104830000C22C11A91FBF2F302FB131302FB034497
:10484000A36818447F287FF794AA7F3890FBF2F37F
:1048500002FB13007330FFF7A3B9FBF7FDFEFFF770
:10486000EFB8FBF7F9FEFFF76FB9DFF88CA29949B3
:10487000BAF80020984C9A1A81FB0210D117C1EBAC
:10488000600101EB4101A2EB810202EB420254F80C
:10489000220018447F2840F3BB80A0F17F030C2046
:1048A00093FBF0F200FB12307330DFF854B298F84B
:1048B0000010C0B204F028FCBBF80030022B1AD95B
:1048C0003868BAF800300C22C11A91FBF2F302FBEF
:1048D000131302FB03435B6818447F2840F39D8356
:1048E0007F3890FBF2F302FB13007330C0B298F8EC
:1048F000001004F009FCBBF80030032B7FF6DAA9A6
:10490000BAF8003038680C22C11A91FBF2F302FBAE
:10491000131302FB0344A36818447F287FF722AADD
:104920007F3890FBF2F302FB13007330FFF7BDB941
:10493000012B3DF4BAAE0124FFF7DAB9DFF8B8A1D4
:1049400099F80000BAF80030624A644CC31A82FB3E
:104950000321DA17C2EB610202EB4202A3EB8203EE
:1049600003EB430354F8233018447F2846DD7F3897
:104970000C2290FBF2F302FB13007330DFF880B1DE
:10498000C0B204F0E9FBBBF80030022B19D999F84A
:104990000000BAF800300C22C11A91FBF2F302FBBE
:1049A000131302FB03435B6818447F2840F38F8096
:1049B0007F3890FBF2F302FB13007330C0B204F0B7
:1049C000CBFBBBF80030032B7EF68BAEBAF8003081
:1049D00099F800000C22C11A91FBF2F302FB1313A9
:1049E00002FB0344A36818447F287FF7B0AD7F38EB
:1049F00090FBF2F302FB130073309AE5FBF72CFEF9
:104A0000BCE7FBF729FEFFF726B9FBF725FEDFE63B
:104A1000FBF722FE49E7FBF71FFEFFF7DEBBFBF7C4
:104A20001BFE5FE6FBF718FE4FE4FBF715FEC7E43D
:104A3000FBF712FE57E5DFF8C0A099F80000BAF8BE
:104A40000030244A264C34E6DFF8ACA03868BAF8C7
:104A50000030204A224CA2E6DFF89CA099F8000022
:104A6000BAF800301B4A1F4C70E7029B1B78002BE2
:104A70007EF4CEA9FEF7F1B9DFF87CA01549BAF8AB
:104A80000020174CF7E6FBF7E7FDFFF768BAFBF7E6
:104A9000E3FDFFF7E2BAFBF7DFFDFFF7E1B9124BE9
:104AA0001B78002B00F0D682104B1B78002B7DF476
:104AB000FCAD0F4B1B78002B3DF4F7ADB8F8003080
:104AC0000C490A33A8F800300A70FDF7EEBDFBF779
:104AD000C3FD73E7ABAAAA2A002401007C210100D0
:104AE000A8220100901B0100A69EFF1FA79EFF1F8A
:104AF000A89EFF1F149CFF1F0C9EFF1F989CFF1F6A
:104B0000289CFF1FA44C2288002A00F02383A3497D
:104B1000DFF89CB20988BBF800000331884227DD2A
:104B20009F48A0490088B1F800E0DFF87CC2181A5D
:104B30000C2190FBF1F901FB19004FF0900909FBE2
:104B40000EFE01FB00E06FF00B0E5CF8000003446A
:104B50000EFB02307F2840F3CE847F3890FBF1F3C8
:104B600001FB13007330C0B298F8001004F0CCFAC7
:104B7000BBF8002023881344022B23DD884B894A8D
:104B800038681B88B2F800C0DFF81CE2C31A0C2199
:104B900093FBF1F201FB1232902303FB0CF301FBB8
:104BA000023373445B6818447F2840F3A7857F383D
:104BB00090FBF1F301FB13007330C0B298F80010C2
:104BC00004F0A2FABBF8002023881344032B23DD52
:104BD000734B744A38681B88B2F800C0DFF8C8E12C
:104BE000C31A0C2193FBF1F201FB1232902303FB59
:104BF0000CF301FB023373449B6818447F2840F395
:104C00000B857F3890FBF1F301FB13007330C0B2CA
:104C100098F8001004F078FABBF8002023881344B9
:104C2000042B7FF747A85D4B1B88012B7FF442A81C
:104C30003A68A2F10C007F287FF794A88B3A0C20E9
:104C400092FBF0F300FB13207330FFF72EB8524CA9
:104C50002388002B40F00D83DFF854B15049514AAE
:104C60000988D7F80080B2F800E04F48C1EB080C83
:104C70000C229CFBF2F102FB11C14FF0900C0CFBDB
:104C80000EFE02FB01E16FF00B0E405880440EFB5C
:104C900003807F2840F36A84A0F17F0393FBF2F046
:104CA00002FB10307330414BC0B2197804F02CFA7B
:104CB000BBF8002023881344022B23DD384A394BEC
:104CC00011883868B3F800C0DFF8DCE0411A0C2224
:104CD00091FBF2F302FB1311902303FB0CF302FB95
:104CE000013373445B6818447F2840F3F1847F38B4
:104CF00090FBF2F302FB130073302C4BC0B2197817
:104D000004F002FABBF8002023881344032B23DDB0
:104D1000234A244B11883868B3F800C0DFF888E0D4
:104D2000411A0C2291FBF2F302FB1311902303FBB7
:104D30000CF302FB013373449B6818447F2840F353
:104D4000CF847F3890FBF2F302FB13007330174BD4
:104D5000C0B2197804F0D8F9BBF8002023881344B6
:104D6000042B7EF7CEA90D4B1B88012B7EF4C9A91D
:104D70003A68A2F10C007F2840F356818B3A0C2050
:104D800092FBF0F300FB13207330084BC0B219788C
:104D900004F0BAF9FEF7B5B99A9CFF1F429CFF1FB9
:104DA0000C9EFF1FBC9DFF1F201C0100989CFF1F35
:104DB000289CFF1FCF4C2388002B40F06582DFF832
:104DC00068B3CD49CD4A098899F80000B2F800E0EF
:104DD000DFF85883C1EB000C0C229CFBF2F102FBC4
:104DE00011C14FF0900C0CFB0EFE02FB01E16FF0C5
:104DF0000B0E58F8011008440EFB03007F2840F307
:104E00007E83A0F17F0393FBF2F002FB103073303E
:104E1000C0B204F0A1F9BBF8002023881344022B90
:104E200022DDB54AB54B118899F80000B3F800C0EF
:104E3000DFF8F8E2411A0C2291FBF2F302FB1311A6
:104E4000902303FB0CF302FB013373445B681844AB
:104E50007F2840F341847F3890FBF2F302FB13007C
:104E60007330C0B204F078F9BBF8002023881344F3
:104E7000032B22DDA04AA14B118899F80000B3F85A
:104E800000C0DFF8A8E2411A0C2291FBF2F302FB0A
:104E90001311902303FB0CF302FB013373449B6853
:104EA00018447F2840F320847F3890FBF2F302FB04
:104EB00013007330C0B204F04FF9BBF80020238810
:104EC0001344042B7DF7C4AF8D4B1B88012B7DF45D
:104ED000BFAF99F80020A2F10C007F287EF721AF28
:104EE0008B3A0C2092FBF0F300FB13207330FEF79B
:104EF000D2BDDFF804A299F80000BAF80030814C66
:104F0000C11A0C2291FBF2F302FB131302FB03F311
:104F1000E35818447F287FF771AD7F3890FBF2F398
:104F200002FB1300733029E5774B1A88182A13D037
:104F30003B681344A3F118007F2840F3C6830C207C
:104F4000973B93FBF0F200FB123303F173006F4BBE
:104F5000C0B2197804F0D8F86D4B6E491A78022A5D
:104F600094BF013200221A701A7831F81200182802
:104F700010D10424022A02F10100C2B288BF00222B
:104F800031F81200182804D1013CF3D11A70FEF751
:104F9000B8B81A703B680344A3F118007F2843DDBA
:104FA0000C20973B93FBF0F200FB123303F17300EC
:104FB000EBE6FBF751FB2EE4534B1B88182B12D06A
:104FC00099F800201344A3F118007F2840F393833D
:104FD0000C20973B93FBF0F200FB123303F17300BC
:104FE000C0B204F0B9F84A4A4A4B127833F812308A
:104FF000182B3DF42DAF99F800201344A3F11800AD
:105000007F287EF78EAE0C20973B93FBF0F200FBDF
:10501000123303F17300FEF73EBDFBF71DFB65E4A1
:10502000FBF71AFBFFF77EBBFBF716FBADE63A4B2F
:105030001B78002B7DF439AB384B1B78002B3DF4EB
:1050400034ABB8F800303649013BA8F800300A709C
:10505000FDF72BBB304B1B78002B7DF477AF2F4B2C
:105060001B78002B3DF421ABB8F800302C490133FC
:10507000A8F800300A70FDF718BBDFF87CA099F89B
:105080000000BAF80030274C3AE71F4A1288182A65
:1050900012D01344A3F118007F2840F3C1820C20E2
:1050A000973B93FBF0F200FB123303F17300C0B2A5
:1050B00098F8001004F028F8154B16491A78022ABF
:1050C00094BF013200221A701A7831F812001828A1
:1050D0002FD10424022A02F10100C2B288BF0022AB
:1050E00031F81200182823D1013CF3D11A703B6823
:1050F000FEF7FEB89A9CFF1F0C9EFF1FBC9DFF1F72
:10510000429CFF1F00240100329CFF1F989CFF1F40
:10511000999CFF1F289EFF1FA79EFF1FA89EFF1F91
:10512000149CFF1FA8220100289CFF1F201C0100C7
:105130001A703B680344A3F118007F287EF712AE73
:105140000C20973B93FBF0F200FB123303F173004A
:10515000FEF7ABBDDFF82CB3E2E4BE4B1A88182A89
:1051600013D03B681344A3F118007F2840F37A82E0
:105170000C20973B93FBF0F200FB123303F173001A
:10518000B54BC0B2197803F0BFFFB44BB4491A78DD
:10519000022A94BF013200221A701A7831F81200E4
:1051A00018287FF4F7AE0424022A02F1010294BF0A
:1051B000D2B2002231F8120018287FF4EAAE013C86
:1051C000F2D11A70FDF79DBFA24B1B88182B12D08D
:1051D00099F800201344A3F118007F2840F372824D
:1051E0000C20973B93FBF0F200FB123303F17300AA
:1051F000C0B203F0B1FF994A994B127833F81230DC
:10520000182B7FF4F8AEFDF723BE924A1288182AB5
:1052100012D01344A3F118007F2840F369820C20B8
:10522000973B93FBF0F200FB123303F17300C0B223
:1052300098F8001003F068FF884B89491A78022A11
:1052400094BF013200221A701A7831F8120018281F
:105250007FF46FAF0424022A02F1010294BFD2B29C
:10526000002231F8120018287FF462AF013CF2D11D
:105270003CE77C4ADFF80CB21288BBF8001003321E
:1052800091427FF715ADE9E4764ADFF8F8B112886C
:10529000BBF80010033291427FF7BDAD91E5724C2F
:1052A0002388002B40F0E481DFF8D8B16F4999F8EA
:1052B00000006F4A09881788DFF8B8E1411A0C220C
:1052C00091FBF2FC02FB1C114FF0900C0CFB07F75A
:1052D00002FB01716FF00B075EF80110014407FB40
:1052E00003107F2840F3C1817F3890FBF2F302FB6B
:1052F00013007330C0B203F02FFFBBF800202388E7
:105300001344022B21DD594B594A99F800001B88A0
:10531000B2F800E0574FC31A0C2193FBF1F201FBE6
:105320001232902303FB0EF301FB02333B445B6814
:1053300018447F2840F3F8817F3890FBF1F301FB9C
:1053400013007330C0B203F007FFBBF800202388BE
:105350001344032B21DD454B454A99F800001B8877
:10536000B2F800E0434FC31A0C2193FBF1F201FBAA
:105370001232902303FB0EF301FB02333B449B6884
:1053800018447F2840F3C1817F3890FBF1F301FB83
:1053900013007330C0B203F0DFFEBBF80020238897
:1053A0001344042B7EF79DA92E4B1B88012B7EF402
:1053B00098A999F80020A2F10C007F287FF7C7A8D0
:1053C0008B3A0C2092FBF0F300FB13207330FFF7B5
:1053D000B0B8294B00227F2107201A8003F06CFE11
:1053E0007F210B2003F068FEFDF7E3BD234B012274
:1053F0007F2107201A8003F05FFE7F210B2003F03E
:105400005BFEFDF7CEBD1E4B04227F2107201A80D4
:1054100003F052FE00210B2003F04EFEFDF7BABD53
:10542000174B02227F2107201A8003F045FE7F21BF
:105430000B2003F041FEFDF7A8BD114B0021072012
:105440001C8003F039FE7F210B2003F035FEFDF7B1
:1054500097BD00BF3A9CFF1F989CFF1F999CFF1FA0
:105460009C9DFF1F429CFF1F9A9CFF1F0C9EFF1FCD
:10547000BC9DFF1F201C0100129CFF1FAA9CFF1F48
:10548000029EFF1F289CFF1FAF4B1A88182A13D0BB
:105490003B681344A3F118007F2840F33F810C20A0
:1054A000973B93FBF0F200FB123303F17300A74B21
:1054B000C0B2197803F028FEA54BA6491A78022A33
:1054C00094BF013200221A701A7831F8120018289D
:1054D0007FF460AD0424022A02F1010294BFD2B22B
:1054E000002231F8120018287FF453AD013CF2D1AC
:1054F0001A70FDF706BEFBF7AFF8FFF734BBFBF7FA
:10550000ABF885E4904A1288182A12D01344A3F10C
:1055100018007F2840F3F6800C20973B93FBF0F2B5
:1055200000FB123303F17300C0B298F8001003F0CF
:10553000EBFD874B87491A78022A94BF013200227B
:105540001A701A7831F8120018287FF4F2AD04248A
:10555000022A02F1010294BFD2B2002231F81200F5
:1055600018287FF4E5AD013CF2D1BFE5FBF774F8F4
:10557000FFF799BB744B1B88182B12D099F80020A9
:105580001344A3F118007F2840F3C5800C20973BFB
:1055900093FBF0F200FB123303F17300C0B203F08F
:1055A000DBFD6B4A6B4B127833F81230182B7FF40B
:1055B00022ADFDF74DBC684B1B88182B12D099F813
:1055C00000201344A3F118007F2840F3B0800C2082
:1055D000973B93FBF0F200FB123303F17300C0B270
:1055E00003F0BAFD5A4A5D4B127833F81230182B8B
:1055F0003EF477A899F800201344A3F118007F28FF
:105600007EF7A5AF0C20973B93FBF0F200FB123323
:1056100003F17300FEF78DBFFBF71EF8FFF7F7BA33
:10562000FBF71AF843E5484B1B88182B11D099F863
:1056300000201344A3F118007F2872DD0C20973B53
:1056400093FBF0F200FB123303F17300C0B203F0DE
:1056500083FD3F4A3F4B127833F81230182BC9D1E3
:10566000FEF73FB8FAF7F8FF8AE5FAF7F5FF41E6EB
:105670003B4ADFF800B11288BBF8001003329142B8
:105680007FF73BAE12E6374B1B88182B11D099F8E9
:1056900000201344A3F118007F2839DD0C20973B2C
:1056A00093FBF0F200FB123303F17300C0B203F07E
:1056B00053FD274A2C4B127833F81230182B99D10E
:1056C000FEF70FB8FAF7C8FF92E5FAF7C5FF3EE418
:1056D000FAF7C2FFFFF711BBFAF7BEFFFFF7C1BB36
:1056E000FAF7BAFFFFF733BBFAF7B6FFFFF7E2BBF3
:1056F000FAF7B2FF9BE5FAF7AFFF71E4FAF7ACFFF8
:10570000FFF75BBAFAF7A8FF0EE7FAF7A5FF41E645
:10571000FAF7A2FFCAE7FAF79FFF3FE7FAF79CFF05
:10572000C5E6FAF799FF91E7FAF796FF0AE6FAF766
:1057300093FF54E70D4B03930D4B0293FDF7A4BE6B
:1057400023601946FDF7D8BB3C9CFF1F989CFF1FA8
:10575000999CFF1FA49DFF1F329CFF1F289EFF1FC7
:10576000429CFF1F3A9CFF1F9C9DFF1FF59BFF1F44
:10577000B69CFF1F289CFF1F38B507F09DFC0B4807
:1057800005F0D4FB00234FF07E5201210848FAF7C0
:105790006DFE084B084A0949802400251C711846F3
:1057A0001D60BDE838400BF049B900BFA89CFF1F41
:1057B000E09DFF1F6C9EFF1F1C89FF1FFD05000061
:1057C00010B50446A4206368198803F0F9FDE36866
:1057D000A6201988BDE8104003F0F2BD43682A20D6
:1057E000198803F0EDBD00BF10B5044622206368A0
:1057F000198803F0E5FDE36824201988BDE810400E
:1058000003F0DEBD10B504460A206368198803F072
:10581000D7FDE3680C201988BDE8104003F0D0BD27
:1058200010B5044606206368198803F0C9FDE368D3
:1058300008201988BDE8104003F0C2BD10B5044629
:1058400002206368198803F0BBFDE368042019880F
:10585000BDE8104003F0B4BD70B50E4C84B0122505
:105860000422012306460390029320468DE824007B
:105870001423102106F05EFD0622092302930396ED
:105880000195204600921423102106F053FD04B028
:1058900070BD00BFD89EFF1F70B5AE4CB4F900308C
:1058A000032B00F0E880002B4DD0022B6CD0052B91
:1058B00000F09880012B00F0C080042B00D070BD58
:1058C00000244FF4AF75E1B2A34805F097FB013413
:1058D0008542A8BF05460C2CF5D1012008F094FAAA
:1058E0000446002008F090FA323CA0F132039B49B4
:1058F0006FF4957000FB03F300FB04F081FB03429F
:1059000081FB0041DB17C017C3EB6223C0EB6120B2
:1059100003F5AF7200F5AF739342A8BF13469D42E3
:10592000A8BF1D46A5F11401312900F3E28040F221
:105930006C7332218A488B4A0180BDE870402A206E
:10594000136003F03DBD0E2007F01AFB40F6FF7117
:10595000C8308842A8BF084620EAE07000F5FA6225
:1059600083B28A42804D814EA8BF0A460220194662
:1059700033802A8003F024FD2988042003F020FDD1
:10598000B4F90030022B92D1172008F03DFA0546F9
:10599000162008F039FAA842B8BF284600F1C8011D
:1059A000B1F5FA7FC0F2BF80B1F57A6FA8BF4FF4AE
:1059B0007A6101F54873B3F57A6FA8BF4FF47A6343
:1059C0009BB289B26A4A6B4D11800A202B8003F08A
:1059D000F7FC29880C2003F0F3FCB4F90030052B08
:1059E0007FF468AF0F2008F00FFAC0F53F6304336F
:1059F000B3F5AF6FC0F28F80B3F5FA6FA8BF4FF465
:105A0000FA6399B25C4BC0F54360B0F5AF6F198093
:105A10007EDBB0F5FA6FA8BF4FF4FA6083B2574D42
:105A2000A4202B8003F0CCFC2988A62003F0C8FC1E
:105A3000B4F90030012B7FF440AF0B2007F0BCFF1E
:105A400000283CD0112008F0DFF900F1C801B1F5C1
:105A50002F7F3CDB41F25C23994278DC484A00F519
:105A6000487089B2B0F52F7F11806DDB8342A8BFEB
:105A700003469BB231E0102008F0C6F9C830B0F5FB
:105A8000FA7F4BDBB0F57A6F0146A8BF4FF47A611D
:105A900001F51673B3F57A6FA8BF4FF47A639BB222
:105AA00089B2384A384D118022202B8003F088FCBF
:105AB0002988242003F084FCB4F90030F3E6152093
:105AC00007F05EFA00F59671B1F52F7F30DA40F2FB
:105AD00014534FF42F712A4A11802C4D06202B802D
:105AE00003F06EFC2988082003F06AFCB4F900304A
:105AF000E3E640F23A72A5F5B975254B02FB05F5D0
:105B000083FB0523ED17A5EB631389B2323311E74D
:105B10004FF4AF6383E74FF4AF6173E740F24C4358
:105B20004FF4FA71BDE740F214534FF4FA7149E7AC
:105B300041F25C2399420ADC114A00F5617089B296
:105B4000B0F52F7F118091DA4FF42F73C5E7194616
:105B5000C1E700BFB49EFF1FA89CFF1F67BBCF46D5
:105B6000749EFF1F9489FF1F7C9EFF1FB49CFF1F24
:105B7000189EFF1F389CFF1FB89CFF1F389EFF1FF9
:105B8000769CFF1FC69DFF1FC29DFF1F4C9EFF1FDF
:105B9000B5814E1B2DE9F041224D82B0012602B2A3
:105BA00084B20092284601967823192106F008FB5A
:105BB00004F10C0212B28DE844002846A71978239C
:105BC000192104F1020806F0FBFA3FB20FFA88F837
:105BD00019233A46284619460196CDF8008006F06A
:105BE000EFFA78233A4628461946CDF80080019608
:105BF00004F10A070B3406F0E3FA3FB224B278232B
:105C00003A46284619468DE8500006F0D9FA19237D
:105C100000943A4601962846194606F0D1FA02B099
:105C2000BDE8F081D89EFF1F30B583B000230C463D
:105C300005B2009326225B231C210C4806F010F8C5
:105C4000294601232622094805F01AFB002C24B21C
:105C500005DB214601232622044805F011FB044AF6
:105C6000044B15801C8003B030BD00BFD89EFF1FC1
:105C7000AA89FF1FAC89FF1F70B59F4C237882B0A3
:105C80001BB19E4B4FF6FF721A809D4BB3F900304B
:105C9000C3B99C4A994B1068B3F9002080F30C00FB
:105CA0005B2303FB00F000131C30824243D04FF013
:105CB000FF31FFF7B9FF944806F036F80023237050
:105CC00002B070BD012B1BD0022B53D0032B38D058
:105CD000042B00F08D80052BF0D10F2008F094F8F4
:105CE000C0F53B600830B0F5AF6F41DBB0F5FA6F3F
:105CF000A8BF4FF4FA60A0F5AF625B2383482EE0A3
:105D0000834B1A68B2F52F7F32DB41F25C2393425A
:105D1000A8BF1346A3F52F735B227E4802FB03F353
:105D200080FB0320DB17C3EBA0201C30734BB3F9BF
:105D300000308342BBD1784BB3F900300133B6D188
:105D4000BCE7764B1B68B3F5FA7F11DBB3F57A6FCE
:105D5000A8BF4FF47A637248A3F5FA725B2303FB82
:105D600002F380FB0320DB17C3EB20201C30DDE7B0
:105D70001C20DBE76B4B1B68B3F5FA7F2EDBB3F51A
:105D80007A6FA8BF4FF47A63A3F5FA7264485B2375
:105D900003FB02F380FB0320DB17C3EB20201C3046
:105DA000614B1B68B3F5FA7F1ADBB3F57A6FA8BFB6
:105DB0004FF47A63A3F5FA7259495B2303FB02F3AC
:105DC00081FB0321DB17C3EB21211C314B4BB3F9C2
:105DD0000030834206D0FFF727FF6CE71C20DFE787
:105DE0001C21F3E74C4BB3F900308B42F3D165E74C
:105DF000272200258DE8240076231C2142484B4EA3
:105E000006F0DEF916E0B0F5AF7FA8BF4FF4AF7033
:105E1000323803FB00F386FB0321DB17C3EB611170
:105E20001C3109B201231D442722374805F028FA06
:105E30000C2D09D0E9B23E4805F0E0F831284FF0CA
:105E40005B03E0DC1C21EDE7012007F0DDFF6FF4D0
:105E500095733238374A03FB00F082FB0023C017EA
:105E6000C0EB632303F5AF73312B42DDB3F5AF7F96
:105E7000A8BF4FF4AF735B22323B2C4D02FB03F300
:105E800085FB0325DB17C3EB65151C35002007F0E8
:105E9000BBFF6FF495733238264A03FB00F082FB98
:105EA0000023C017C0EB632303F5AF73312B1EDD56
:105EB000B3F5AF7FA8BF4FF4AF735B22323B1B49F2
:105EC00002FB03F381FB0321DB17C3EB61111C31E0
:105ED0000A4BB3F90030AB4201D028467BE70E4BAA
:105EE000B3F900308B423FF4E6AE284673E71C213D
:105EF000EEE71C25CAE700BFAE9EFF1FAA89FF1F61
:105F0000B49EFF1F1C9EFF1FD89EFF1F37800B6D86
:105F1000009CFF1FD3058541AC89FF1F489CFF1FD4
:105F2000011FB812589CFF1F1C9CFF1F4B48371BBA
:105F3000A89CFF1F67BBCF462DE9F041044682B005
:105F400056482768E56805F0E3FD1120FFF722FEBB
:105F5000012619234FF02808194624224F4801969C
:105F6000CDF8008006F02CF97823194624224B48FE
:105F70000196CDF8008006F023F93146474806F037
:105F8000B5FC02221921454806F0ACFC38460BF05E
:105F900017FB39460246414806F03EFE3F4806F0F0
:105FA00051FE142200213D4806F09CFC03223C498E
:105FB0003A4806F031FE394806F044FE232200211B
:105FC000364806F08FFC03223649344806F024FE9A
:105FD000324806F037FE7DB12F20FFF7DBFD32227D
:105FE00000212E4806F07EFC03222F492B4806F0A4
:105FF00013FE2A4806F026FE01232C4A1846137089
:10600000FFF72AFC2189638962685B1A5C2B12887E
:1060100032DD521A02EB4202C2EB4212013392FB12
:10602000F3F31B33224A1D48138001261A221BB2A8
:106030008DE844001946142206F0C2F8CDB1218A39
:10604000638AE2685B1A5C2B12881DDC511A5C22A1
:1060500002FB01F292FBF3F31B33164A0F48138045
:10606000012438221BB28DE814001946322206F0B2
:10607000A7F802B0BDE8F081511A5C2202FB01F2E0
:1060800092FBF3F31B33CDE7521A02EB4202C2EB51
:106090004212334492FBF3F31B33DEE7D89EFF1F1B
:1060A000D8240100DC240100E0240100559FFF1FDB
:1060B000B09EFF1FB29EFF1F2DE9F0411E4682B029
:1060C00014461AB3052A054600F09C80099B6F4AC6
:1060D00000EBC305012C6F8929896868A7EB0103D0
:1060E00082FB03E21A444FEAE373C3EBA213028874
:1060F00029D0042C69D0664A022CB2F9001060D075
:10610000082C65D0012002B0BDE8F081614D624AE3
:106110002B681268CB1A93420F466FD95F4A3388B7
:1061200011785F48012918BF01241470089A0632BB
:106130001BB212B28DE814001946BDF9202006F0FA
:106140003FF82F60DEE79BB2D31A994203DC9F42EF
:106150003946A8BF1946089A0180B6F90030BDF942
:1061600020804F48971D4FF0000E3FB2194642461F
:106170000097CDF804E006F023F829896A896B6856
:10618000521A1B885C2AA3EB010377DD03EB430360
:106190000132C3EB431393FBF2F303F11B0213B27F
:1061A0000120328019464246019000973C4806F093
:1061B00007F83A4B00221A70354A022CB2F9001047
:1061C0009ED14B1C1BB2138004E012FA83F3BCE790
:1061D00000231380994295D0089AB6F900303048D0
:1061E0000632012412B2009219460194BDF9202012
:1061F00005F0E6FF204602B0BDE8F081204602B07F
:10620000BDE8F081072400265A2323228DE85000A0
:106210001A21234805F0A2FF0121214806F066FB60
:1062200001211F4806F068FB232235211C4806F097
:1062300059FB22461B491A4806F0EEFC184806F0A6
:1062400001FD174805F070FD4FF4FA6007F0EAFB16
:10625000FFF722FB5A2323221A218DE85000104811
:1062600005F07CFF0E4805F05FFD2846FFF764FE51
:106270000D4B01221A70FFF7FFFC43E75C2101FB85
:1062800003F393FBF2F21B3289E700BFC94216B257
:10629000B89EFF1F409FFF1F8C340100559FFF1FBA
:1062A000D89EFF1FE4240100AE9EFF1F2DE9F04F92
:1062B0005A4E5B4DB6F900704C7855F8277085B092
:1062C0008146984604B10C78DFF874A11AB99AF89F
:1062D0000030002B39D0534D002338462B808AF8EC
:1062E0000030FFF729FE504A504BB5F9000001215C
:1062F00011704FF6FF721A8060B301285ED0012042
:1063000032232246019000934946494B3846FFF715
:10631000D3FE00240346B5F90020022A39DD00220D
:106320002A80B6F900203D49002A3BDB052AC4BF7C
:1063300000220A80B8F1000F39D1002C0CBF18469A
:106340004FF0FF3005B0BDE8F08F364DB5F90000D5
:106350000028D2D1DFF8ECB0364ADBF80030126802
:10636000C3EB0903934227D9334B1A78012A18BF8C
:1063700001201870FFF770FA0123CBF80090012C70
:106380002AD0042C35D0022C3AD0082C3ED0002440
:10639000C1E7C6D1FA68002AC1D0B6F900201F496A
:1063A000002AC3DA05220A80B8F1000FC5D0039392
:1063B000FFF762FC039BC0E70346E0E74FF0000EE7
:1063C000142322468DE8084049461C4B3846744643
:1063D000FFF772FE03469EE732888AF800400132DA
:1063E00032807A6982B10024384603939047039B38
:1063F00091E732880121013A32808AF80010F0E7F3
:1064000001222A8000248CE7144684E77A6900215F
:1064100029804FF0FF34002AE6D182E7B49EFF1FA7
:10642000B089FF1FB89EFF1FAE9EFF1FAA89FF1FE6
:10643000B29EFF1F8C340100559FFF1FB09EFF1FAF
:10644000B69EFF1F409FFF1F01210D2007F0AEBA2F
:1064500000210D2007F0AABA01460D2007F0A6BAC8
:1064600008B50D2007F0A8FAB0FA80F149090D200F
:10647000BDE8084007F09ABA10B5002144080D2085
:1064800007F094FA204607F0CDFA0D20012107F01D
:106490008DFA2046BDE8104007F0C4BA214A224BCD
:1064A00010881B68984210B535DA204A1288141AF1
:1064B0009A42A8BF1A46B4F5157F22DA121A40F2A2
:1064C000532303FB02F393FBF4F105310A2007F099
:1064D000DDF8174B197801B3164B17491B6840F2CA
:1064E000271283F3070302FB03F381FB0321194403
:1064F000DB17C3EBA11105310920BDE8104007F0FF
:10650000C5B8131A4FF41572611C02FB03F393FB19
:10651000F1F10531DAE70021D8E70920BDE81040A4
:1065200007F0B4B8B49CFF1FF89BFF1F7C9EFF1FB1
:10653000789CFF1F649EFF1F090402817F2838B5E5
:10654000A8BF7F200F4C4FF4167202FB00F284FBB1
:1065500002311144D2170546C2EBA1110A2007F0FF
:1065600095F87F3D4FF4967303FB05F384FB0321FD
:106570001944DB17A3EBA1110920BDE8384007F04F
:1065800085B800BF09040281C368B3F9003030B593
:1065900083EAE374A4EBE374002BA0B218DB0123BD
:1065A00000E0134603EB830252009442F9DA0A4DED
:1065B00090FBF3F285FB03E403FB1200DB173032A0
:1065C000D3EBA40380B201F8012BF1D10B7030BDE5
:1065D0002D230B700131E2E76766666638B5094D19
:1065E0008224204602F006FF35F8021B00B28842E2
:1065F000204601D002F0E4FE0234A4B28A2CF0D18D
:1066000038BD00BFA49DFF1F024B8020198802F0F7
:10661000D7BE00BF3C9CFF1F38B5094D78242046EB
:1066200002F0E8FE35F8021B00B28842204601D095
:1066300002F0C6FE0234A4B2802CF0D138BD00BFF7
:106640009C9DFF1F024B7620198802F0B9BE00BF47
:106650003A9CFF1F38B5094D4624204602F0CAFE79
:1066600035F8021B00B28842204601D002F0A8FE95
:106670000234A4B24E2CF0D138BD00BF289EFF1FBB
:10668000024B4420198802F09BBE00BF329CFF1FC2
:10669000024B4E20198802F093BE00BF549CFF1F8E
:1066A000024B9A20198802F08BBE00BF9A9CFF1FF4
:1066B000024B9820198802F083BE00BF429CFF1F46
:1066C000024B8C20198802F07BBE00BFBC9DFF1FCF
:1066D000024B9C20198802F073BE00BF289CFF1F4C
:1066E000024BA020198802F06BBE00BF309EFF1F36
:1066F000024B9620198802F063BE00BF0C9EFF1F5C
:10670000024B8A20198802F05BBE00BFCE9DFF1F9E
:1067100008B5034B1020198802F052FE012008BD75
:10672000CC9DFF1F024B1020198802F049BE00BF0C
:10673000CC9DFF1F024B2C20198802F041BE00BFE8
:10674000269CFF1F024B1E20198802F039BE00BF95
:10675000409CFF1FC3680E20198802F031BE00BFA5
:10676000024B2820198802F02BBE00BF269EFF1F77
:10677000024B6220198802F023BE00BF649CFF1FF9
:10678000024B6420198802F01BBE00BF209EFF1F31
:10679000024B5A20198802F013BE00BF089CFF1F4D
:1067A000024B1620198802F00BBE00BF129CFF1F7F
:1067B000024B2E20198802F003BE00BFA09CFF1FD1
:1067C000024B3020198802F0FBBD00BF8C9EFF1FDA
:1067D000024B9E20198802F0F3BD00BF9089FF1F75
:1067E000024BAC20198802F0EBBD00BF229EFF1FB8
:1067F000024BAE20198802F0E3BD00BF4C9CFF1F86
:10680000024BB020198802F0DBBD00BFB09DFF1F16
:10681000024BB220198802F0D3BD00BF6E9CFF1F4F
:10682000024B1820198802F0CBBD00BFBA9CFF1F95
:10683000024BA220198802F0C3BD00BF529EFF1F69
:10684000024B1A20198802F0BBBD00BF5C9CFF1FE1
:10685000024B1C20198802F0B3BD00BF569CFF1FDD
:10686000024B6620198802F0ABBD00BF609EFF1F7F
:10687000024B7220198802F0A3BD00BF889EFF1F43
:10688000024B2020198802F09BBD00BF5E9EFF1FB7
:10689000024B3220198802F093BD00BF4E9EFF1FAD
:1068A000024B6820198802F08BBD00BF949CFF1F2B
:1068B000024B6C20198802F083BD00BFFC9BFF1FB8
:1068C000024B5220198802F07BBD00BF2E89FF1FAA
:1068D000024B5020198802F073BD00BF2089FF1FB2
:1068E000024B5420198802F06BBD00BFA489FF1F22
:1068F000024B5C20198802F063BD00BFA889FF1F0E
:10690000024B5E20198802F05BBD00BF2C89FF1F7F
:10691000024B5620198802F053BD00BF969CFF1F02
:10692000244B1B880B2B43D8DFE803F00B10151A00
:106930001F24292E33383D06084604221E490AF03A
:10694000FDBE084604221D490AF0F8BE084604228E
:106950001B490AF0F3BE084604221A490AF0EEBEAB
:106960000846042218490AF0E9BE084604221749DD
:106970000AF0E4BE0846042215490AF0DFBE0846C4
:10698000042214490AF0DABE0846042212490AF029
:10699000D5BE0846042211490AF0D0BE084604229A
:1069A0000F490AF0CBBE084604220E490AF0C6BEC3
:1069B000704700BF0C9EFF1F282D0100982A010080
:1069C00004290100DC2D010008290100C42D01006B
:1069D0000C29010010290100BC2B01001429010021
:1069E000342D010018290100064B074A10B41C88F9
:1069F000064B0846002C14BF11461946042210BC51
:106A00000AF09CBE749CFF1F1C2901002029010074
:106A1000064B074A10B41C88064B0846002C14BFCE
:106A200011461946042210BC0AF088BEA29CFF1F22
:106A30001C29010020290100064B074A10B41C88BC
:106A4000064B0846002C14BF11461946042210BC00
:106A50000AF074BEC09DFF1F1C29010020290100FF
:106A6000064B074A10B41C88064B0846002C14BF7E
:106A700011461946042210BC0AF060BED49DFF1FC7
:106A80001C29010020290100064B074A10B41C886C
:106A9000064B0846002C14BF11461946042210BCB0
:106AA0000AF04CBE0E9EFF1F1C2901002029010088
:106AB000064B074A10B41C88064B0846002C14BF2E
:106AC00011461946042210BC0AF038BEAA9CFF1FCA
:106AD0001C290100202901001B4B1B880A2B0AD806
:106AE000DFE803F00A0E12161A1E22262A2E0600CE
:106AF000164B186808607047154B18680860704797
:106B0000144B186808607047134B1868086070478A
:106B1000124B186808607047114B1868086070477E
:106B2000104B1868086070470F4B18680860704772
:106B30000E4B1868086070470D4B18680860704766
:106B40000C4B186808607047CE9DFF1F4829010054
:106B50002029010024290100282901002C290100F5
:106B60003029010034290100382901003C290100A5
:106B70004029010044290100F0B52B4E2B4FDFF8CE
:106B8000C4E005460FCE87B06C460FC496E80300FC
:106B90003B68274A274F44F8040B40F6CC30834229
:106BA000C8BF3A46BEF800602180012E1188927855
:106BB000ADF80D108DF80F202AD032D340F6CA025E
:106BC000022E18BF00229A4226DAA3F698031A4929
:106BD0001A4AC3EB031381FB03011944DB17C3EB10
:106BE0006123243382FB0321DA17C2EBA10202EBFB
:106BF0008201A3EB4103303330328DF813308DF82E
:106C000011206946284616220AF098FD07B0F0BD0B
:106C100040F698029A42D8DB094B1868CDF811006B
:106C2000EFE740F6FC02CEE75C290100149EFF1F4F
:106C3000502901004C2901003B773B986766666646
:106C400054290100AC9DFF1FF8B5174C174E227850
:106C5000174D33782F888E46003218BF0122014627
:106C60007046FFF723FB002398423370237015DB37
:106C700014BF012000202B889F420ED040F23A72B0
:106C8000A3F5AF730B490C4C02FB03F381FB03121A
:106C9000DB17A3EB621332332360F8BD07490122EF
:106CA00018460A702270E6E7A08AFF1FC99EFF1FE0
:106CB000749EFF1FB5814E1B9489FF1F549FFF1FB9
:106CC000014B187802F014BB3C9FFF1F014B187852
:106CD00002F028BB9490FF1F134BB3F9003030B57E
:106CE00083EAE374A4EBE374002BA0B218DB012366
:106CF00000E0134603EB830252009442F9DA0B4D95
:106D000090FBF3F285FB03E403FB1200DB17303248
:106D1000D3EBA40380B201F8012BF1D10B7030BD8D
:106D20002D230B700131E2E79490FF1F67666666C2
:106D3000144BB3F9003070B583EAE375A5EBE37546
:106D4000002BACB21ADB012300E0034603EB830007
:106D500040008542F9DA0C4E94FBF3F086FB03E524
:106D600003FB1044DB173030D3EBA503A4B201F8CA
:106D7000010BF1D105480B70106070BD2D230B7015
:106D80000131E0E7089CFF1F676666667429010011
:106D9000134BB3F9003030B583EAE374A4EBE3742A
:106DA000002BA0B218DB012300E0134603EB8302A3
:106DB00052009442F9DA0B4D90FBF3F285FB03E4A9
:106DC00003FB1200DB173032D3EBA40380B201F8CF
:106DD000012BF1D10B7030BD2D230B700131E2E797
:106DE0009089FF1F67666666134BB3F9003030B5B4
:106DF00083EAE374A4EBE374002BA0B218DB012355
:106E000000E0134603EB830252009442F9DA0B4D83
:106E100090FBF3F285FB03E403FB1200DB17303237
:106E2000D3EBA40380B201F8012BF1D10B7030BD7C
:106E30002D230B700131E2E74C9CFF1F67666666ED
:106E4000134BB3F9003030B583EAE374A4EBE37479
:106E5000002BA0B218DB012300E0134603EB8302F2
:106E600052009442F9DA0B4D90FBF3F285FB03E4F8
:106E700003FB1200DB173032D3EBA40380B201F81E
:106E8000012BF1D10B7030BD2D230B700131E2E7E6
:106E90006E9CFF1F67666666134BB3F9003030B512
:106EA00083EAE374A4EBE374002BA0B218DB0123A4
:106EB00000E0134603EB830252009442F9DA0B4DD3
:106EC00090FBF3F285FB03E403FB1200DB17303287
:106ED000D3EBA40380B201F8012BF1D10B7030BDCC
:106EE0002D230B700131E2E7529EFF1F6766666635
:106EF000134BB3F9003030B583EAE374A4EBE374C9
:106F0000002BA0B218DB012300E0134603EB830241
:106F100052009442F9DA0B4D90FBF3F285FB03E447
:106F200003FB1200DB173032D3EBA40380B201F86D
:106F3000012BF1D10B7030BD2D230B700131E2E735
:106F40002E89FF1F67666666134BB3F9003030B5B4
:106F500083EAE374A4EBE374002BA0B218DB0123F3
:106F600000E0134603EB830252009442F9DA0B4D22
:106F700090FBF3F285FB03E403FB1200DB173032D6
:106F8000D3EBA40380B201F8012BF1D10B7030BD1B
:106F90002D230B700131E2E72089FF1F67666666CB
:106FA000134BB3F9003030B583EAE374A4EBE37418
:106FB000002BA0B218DB012300E0134603EB830291
:106FC00052009442F9DA0B4D90FBF3F285FB03E497
:106FD00003FB1200DB173032D3EBA40380B201F8BD
:106FE000012BF1D10B7030BD2D230B700131E2E785
:106FF000A489FF1F67666666134BB3F9003030B58E
:1070000083EAE374A4EBE374002BA0B218DB012342
:1070100000E0134603EB830252009442F9DA0B4D71
:1070200090FBF3F285FB03E403FB1200DB17303225
:10703000D3EBA40380B201F8012BF1D10B7030BD6A
:107040002D230B700131E2E7A889FF1F6766666692
:10705000134BB3F9003030B583EAE374A4EBE37467
:10706000002BA0B218DB012300E0134603EB8302E0
:1070700052009442F9DA0B4D90FBF3F285FB03E4E6
:1070800003FB1200DB173032D3EBA40380B201F80C
:10709000012BF1D10B7030BD2D230B700131E2E7D4
:1070A0002C89FF1F6766666608B5702002F0A2F99A
:1070B000044B1988884204D07020BDE8084002F0D3
:1070C0007FB908BDAC9DFF1F08B5742002F092F98E
:1070D000044B1988884204D07420BDE8084002F0AF
:1070E0006FB908BD449EFF1F054B1B88084604224C
:1070F00013B904490AF022BB03490AF01FBB00BFC1
:10710000549CFF1F7C290100782901000E4B1B882D
:10711000032B17D8DFE803F0110C070208460422FE
:107120000A490AF00BBB0846042209490AF006BBCB
:107130000846042207490AF001BB08460422064912
:107140000AF0FCBA704700BFBC9DFF1F8C290100EC
:1071500088290100842901008029010010B40A4B0C
:107160000A4C0A4693E8030083B0238802AC04E982
:10717000030004EB8303104653F8081C052203B0F8
:1071800010BC0AF0DBBA00BF7C250100209EFF1F67
:1071900030B40A4B0A4D0C4693E8070084B02B88A4
:1071A00004AD05E9070005EB8303204653F80C1CEA
:1071B000042204B030BC0AF0C1BA00BF842501002B
:1071C000AC9DFF1FF0B40C4D0C4F0E460FCD8CB094
:1071D00001AC0FC40FCD0FC495E807003B8884E8CD
:1071E00007000CAA02EB8303304653F82C1C042240
:1071F0000CB0F0BC0AF0A2BA90250100029EFF1F5D
:1072000030B50A4B0A4D0C460FCB85B00DF1100E70
:107210000EE90F002B880EEB8303204653F8101C59
:10722000042205B0BDE830400AF088BACC25010040
:10723000229EFF1F30B50A4B0A4D0C460FCB85B07E
:107240000DF1100E0EE90F002B880EEB8303204684
:1072500053F8101C042205B0BDE830400AF06EBAA5
:10726000CC250100B09DFF1FF0B40B4D0B4F0E4617
:107270000FCD86B06C460FC495E803003B8884E8C8
:10728000030006AA02EB8303304653F8181C0422BD
:1072900006B0F0BC0AF052BADC250100BA9CFF1F10
:1072A000F0B40A4D0A4F0E460FCD86B001AC0FC4A4
:1072B0002A683B88226006AA02EB8303304653F813
:1072C000141C0C2206B0F0BC0AF038BAF4250100F8
:1072D000569CFF1FF0B40B4D0B4F0E460FCD86B0E2
:1072E0006C460FC495E803003B8884E8030006AAB7
:1072F00002EB8303304653F8181C042206B0F0BC9E
:107300000AF01CBA08260100449EFF1F164B1B887A
:107310000BB31BB283EAE370A0EBE370002B30B534
:1073200084B21DDB012300E0134603EB830252000D
:107330009042F9DA0D4894FBF3F280FB03E503FB7E
:107340001244DB173032D3EBA503A4B201F8012BB2
:10735000F1D10B7030BD0846042205490AF0EEB9A0
:107360002D230B700131DDE7949CFF1F6766666675
:107370009029010030B40A4B0A4D0C4693E80700EF
:1073800084B02B8804AD05E9070005EB8303204694
:1073900053F80C1C042204B030BC0AF0CFB900BF73
:1073A00020260100FC9BFF1F054B1B881BB9054BCA
:1073B0001868086070470846042203490AF0BEB9FD
:1073C0009A9CFF1F202901001C290100164B1B88D5
:1073D0000BB31BB230B583EAE374A4EBE374002B68
:1073E000A0B21CDB012300E0134603EB8302520032
:1073F0009442F9DA0D4D90FBF3F285FB03E403FBB5
:107400001200DB173032D3EBA40380B201F8012B5A
:10741000F1D10B7030BD064B1868086070472D2302
:107420000B700131DEE700BF409CFF1F6766666698
:1074300020290100164B1B880BB31BB230B583EA21
:10744000E374A4EBE374002BA0B21CDB012300E087
:10745000134603EB830252009442F9DA0D4D90FB80
:10746000F3F285FB03E403FB1200DB173032D3EBAE
:10747000A40380B201F8012BF1D10B7030BD064B93
:107480001868086070472D230B700131DEE700BFDC
:10749000129EFF1F6766666620290100164B1B8837
:1074A0000BB31BB230B583EAE374A4EBE374002B97
:1074B000A0B21CDB012300E0134603EB8302520061
:1074C0009442F9DA0D4D90FBF3F285FB03E403FBE4
:1074D0001200DB173032D3EBA40380B201F8012B8A
:1074E000F1D10B7030BD064B1868086070472D2332
:1074F0000B700131DEE700BF129CFF1F67666666F6
:1075000094290100174B1B881BB31BB270B583EA8B
:10751000E375A5EBE375002BACB21EDB012300E0A5
:10752000034603EB830040008542F9DA0E4E94FBDC
:10753000F3F086FB03E503FB1044DB173030D3EB9D
:10754000A503A4B201F8010BF1D108480B7010603B
:1075500070BD074B1868086070472D230B70013110
:10756000DCE700BFA09CFF1F6766666698290100E4
:1075700020290100164B1B880BB31BB230B583EAE0
:10758000E374A4EBE374002BA0B21CDB012300E046
:10759000134603EB830252009442F9DA0D4D90FB3F
:1075A000F3F285FB03E403FB1200DB173032D3EB6D
:1075B000A40380B201F8012BF1D10B7030BD064B52
:1075C0001868086070472D230B700131DEE700BF9B
:1075D0008C9EFF1F6766666620290100164B1B887C
:1075E0000BB31BB230B583EAE374A4EBE374002B56
:1075F000A0B21CDB012300E0134603EB8302520020
:107600009442F9DA0D4D90FBF3F285FB03E403FBA2
:107610001200DB173032D3EBA40380B201F8012B48
:10762000F1D10B7030BD064B1868086070472D23F0
:107630000B700131DEE700BF609EFF1F6766666664
:1076400020290100164B1B880BB31BB230B583EA0F
:10765000E374A4EBE374002BA0B21CDB012300E075
:10766000134603EB830252009442F9DA0D4D90FB6E
:10767000F3F285FB03E403FB1200DB173032D3EB9C
:10768000A40380B201F8012BF1D10B7030BD064B81
:107690001868086070472D230B700131DEE700BFCA
:1076A000889EFF1F6766666620290100174B1B88AE
:1076B0001BB31BB270B583EAE375A5EBE375002B32
:1076C000ACB21EDB012300E0034603EB8300400065
:1076D0008542F9DA0E4E94FBF3F086FB03E503FBDB
:1076E0001044DB173030D3EBA503A4B201F8010B33
:1076F000F1D108480B70106070BD074B1868086026
:1077000070472D230B700131DCE700BF5E9EFF1F29
:10771000676666669829010020290100054B1B88D1
:107720001BB1054B186808607047044B1868086067
:10773000704700BF969CFF1FAC290100A8290100DB
:10774000184B1A8852B3184A128830B50A80B3F918
:107750000030002B83EAE374A4EBE374BCBF2D2359
:107760008B70A0B2ACBF02310331012300E013469D
:1077700003EB830252009442F9DA0C4D90FBF3F2D2
:1077800085FB03E403FB1200DB173032D3EBA403C9
:1077900080B201F8012BF1D10B7030BD044B186899
:1077A000086070475C9CFF1FB02901006766666631
:1077B0002029010070B53C4D2B780646002B35D1B1
:1077C0001C4673780BB9204670BDFAF7D7FB374AD1
:1077D000374B3848127831781B78007802EB430336
:1077E0004A1E03EB80030E2AEDD801A050F822F0C8
:1077F000597800007B780000C777000059780000B6
:10780000C7770000C7770000C777000047780000FF
:10781000C7770000C7770000C7770000C777000070
:10782000C7770000C777000043780000AE212248E8
:1078300003F01EFF204804F06BF900232B70012495
:10784000BFE706F001FCAF211B4803F011FF1B4A04
:10785000012313702B70B6E783B9194803880429F4
:107860004FF6FF7103F1FF320CBF01230B461344A7
:1078700003F07F03013303800FE073B1013B114A32
:1078800032F813304BB10E4E0F481049104A338076
:107890000123002606700B701370084A0221012391
:1078A00011702B70204670BDA08AFF1FA99EFF1F7C
:1078B000AA9EFF1F549EFF1FD89EFF1F549FFF1FAD
:1078C000509EFF1F8C9DFF1F8C9CFF1F149CFF1F51
:1078D000579FFF1F10B5064B064C1A882046012102
:1078E00001F05CFD21884220BDE8104001F068BD38
:1078F000749CFF1F309CFF1F10B5064B064C1A8866
:107900002046022101F04AFD21884220BDE81040B6
:1079100001F056BDA29CFF1F309CFF1F10B5064B07
:10792000064C1A882046042101F038FD21884220A7
:10793000BDE8104001F044BDC09DFF1F309CFF1FFB
:1079400010B5064B064C1A882046062101F026FD8C
:1079500021884220BDE8104001F032BDD49DFF1FB8
:10796000309CFF1F10B5064B064C1A88204600219C
:1079700001F014FD21884220BDE8104001F020BD37
:107980000E9EFF1F309CFF1F08B5122001F032FD34
:10799000054B1988884206D0122001F011FDBDE880
:1079A000084001F025BC08BD029EFF1F08B5582005
:1079B00001F020FD054B1988884206D0582001F0BF
:1079C000FFFCBDE8084001F013BC08BD129EFF1F7C
:1079D00008B5142001F00EFD054B1988884206D029
:1079E000142001F0EDFCBDE8084001F001BC08BD29
:1079F000AA9CFF1FF0B480EAE075A5EBE0750028B3
:107A0000ACB21FDB1DBF2B230B704E1C0E46012397
:107A100000E0134603EB830252009542F9DA0B4F64
:107A200094FBF3F287FB030503FB1244DB173032B0
:107A3000D3EBA503A4B206F8012BF1D133700846AD
:107A4000F0BC70472D230B704E1CE0E7676666663E
:107A5000174B18880C2813D0192815D01A2817D0BE
:107A60001B2819D01C281BD01D281DD01E2803D070
:107A70000C3800B2FFF7BEBF0E4A106808607047AE
:107A80000D4A1068086070470C4A1068086070471B
:107A90000B4A1068086070470A4A1068086070470F
:107AA000094A106808607047084A10680860704703
:107AB0004E9EFF1FD0290100B8290100BC290100FA
:107AC000C0290100C4290100C8290100CC290100F6
:107AD000034B1888A0EB8000400000B2FFF78ABF7C
:107AE0003C9FFF1F024BB3F90000FFF783BF00BFAD
:107AF000649CFF1F024B1888033800B2FFF77ABF5F
:107B0000269EFF1F024B18880C3800B2FFF772BF89
:107B10000E9CFF1F024B1888183800B2FFF76ABF8F
:107B20003C9CFF1F024B1888183800B2FFF762BF59
:107B30003A9CFF1F024B1888183800B2FFF75ABF53
:107B4000329CFF1FC3681888183800B2FFF752BF75
:107B5000054B1B881BB9054B186808607047084621
:107B60000422034909F0EABD309EFF1F20290100CD
:107B70001C290100054B1B881BB9054B18680860C0
:107B8000704708460422034909F0D8BD429CFF1FF4
:107B9000202901001C29010030B5134C85B00125B6
:107BA0002B463C2202212046009503F0D7FD2046BB
:107BB00003F0AEFF00224021802320460191009374
:107BC00011460A4B029504F051FC204604F0ACF833
:107BD00007480849084A0023036083800B608B80B4
:107BE0001360938005B030BDD89EFF1F4430010064
:107BF000BC9EFF1FD09EFF1F449FFF1F10B500EBD0
:107C0000C00000F10F02D2B293B284B09C1E981C47
:107C10003D2303918DE819003921024804F08AFBC5
:107C200004B010BDD89EFF1F014B01221A7070478F
:107C3000C99EFF1FF0B5734B734C744D744F754E56
:107C400085B004228DE80C0002932046724B40223E
:107C5000802103F08BFB2046704A7149714C08F07B
:107C6000EDFEAF61704FEF61704FA7617048714FCB
:107C7000E761714F87617149714FC761714F8F61C2
:107C8000714A724FCF61724F9761724B724FD761D9
:107C9000724F9F61724FDF61724FB761724D734FC8
:107CA000F761734FAF61734C734FEF61734FA7610F
:107CB0007348744FE761744F74498761744FC761AB
:107CC000744F754A8F61754FCF61754F754B9761D2
:107CD000754FD761754F764E9F61764FDF61764F56
:107CE000764DB761764FF761764F774CAF61774F3E
:107CF000EF61774F7748A761774FE761774F8761EB
:107D00007749784FC761784F8F61784A784FCF6154
:107D1000784F9761784B794FD761794F9F61794E52
:107D2000794FDF61794FB761794D7A4FF7617A4FBB
:107D3000AF617A4C7A4FEF617A4FA7617A487B4FF7
:107D4000E7617B4F87617B497B4FC7617B4F8F61C9
:107D50007B4A7C4FCF617C4F97617C4B7C4FD761D6
:107D60007C4F7D4E9F617D4FDF617D4F7D4DB761C3
:107D70007D4FF7617D4F7E4CAF617E4FEF617E4F4F
:107D80007E48A7617E4FE7617E4F7F4987617F4FC5
:107D9000C7617F4F7F4A8F617F4FCF617F4F804B9D
:107DA0009761804FD761804F9F61804E804FDF6128
:107DB000804F814DB761814FF761814F814CAF6139
:107DC000814F82488249EF61824F834DA761E5610F
:107DD000824F834D834CDFF830E2834A834B8761C7
:107DE000C5618C61824E834F834D844CC1F81CE089
:107DF000834884499761D5619C61D861B16005B0C1
:107E0000F0BD00BF40420F00D89EFF1F108AFF1F29
:107E1000057B0000B88CFF1FE090FF1F1C89FF1F2F
:107E2000C5B30000EC8EFF1F55670000F57A000017
:107E3000388EFF1F61670000E9690000288CFF1F72
:107E4000D5780000116A0000108FFF1FF97800003C
:107E5000396A0000348AFF1F1D790000E57A0000AE
:107E600071670000616A0000488DFF1F41790000C2
:107E70005D710000948CFF1F81670000896A00001B
:107E8000248DFF1F65790000D17A0000008DFF1F4F
:107E9000C16C0000D96C0000C88EFF1FCD6C0000C3
:107EA00091710000BC8BFF1FA9700000C57100001C
:107EB0007C8FFF1F8979000035740000708CFF1FD4
:107EC000AD790000316D00007C8BFF1F91670000D1
:107ED000B16A00000C90FF1FD17900009D74000072
:107EE0004C8CFF1FA1670000057500006C8DFF1F03
:107EF000B167000075750000048CFF1FC1670000AA
:107F0000916D0000348BFF1FD167000001720000EB
:107F1000C48FFF1FE1670000E96D0000808EFF1F26
:107F2000F167000035720000108BFF1F0168000030
:107F3000416E0000C889FF1F1168000069720000CF
:107F4000588AFF1F21680000996E0000DC8CFF1F1B
:107F50003168000041770000A48EFF1F41680000D7
:107F6000A1720000A490FF1F51680000DD750000A1
:107F7000148EFF1F6168000045760000EC8AFF1F29
:107F800071680000D5720000A08FFF1FC97000004B
:107F9000AD7600005C8EFF1F81680000517A000002
:107FA000C88AFF1F916800000D730000A48AFF1F9C
:107FB000A1680000757300007090FF1FB168000099
:107FC000F16E0000E08BFF1FC16800007C8AFF1F7C
:107FD000588BFF1F496F0000D1680000A16F00009F
:107FE000E1680000F96F0000348FFF1FEC89FF1F6C
:107FF0009890FF1F51700000016900001D7700007C
:108000001169000091850000F1680000F0B5461C80
:1080100083B00D460127032336B22AB20446314607
:108020008DE888002448ADB204F01AF90C23AA1C8C
:1080300012B200930197052321B21F4804F010F9F2
:108040001E4A1F4B12881B68BA422AD023D3022A29
:1080500010D11C4CA3F6CA0384FB03241C44DB1779
:10806000C3EB24140A2CA8BF0A2424EAE474A2B2A5
:1080700023B202E000231A461C460D35AA1A01203D
:108080000093019012B2314603230B4804F066F8C6
:10809000204603B0F0BD0C4CA3F6FC0384FB032484
:1080A000DDE7084CA3F6980384FB03241C44DB178C
:1080B000C3EBE404D6E700BFD89EFF1FAC9DFF1FB3
:1080C000149EFF1F898888881F85EB512DE9F04396
:1080D0008FB283B0DFF84C80BD1D461D2DB204B2B7
:1080E00036B24FF001090AB22346314640460095A8
:1080F000CDF8049004F064F82A4633462146404601
:108100008DE8200204F05CF807F10C02009533467C
:1081100012B22146CDF80490404604F051F803B065
:10812000BDE8F083D89EFF1F2DE9F043804685B05F
:10813000002956D10121304804F0D8FB2F4998F886
:10814000062098F8083011F80290994522DA4FEA93
:1081500089064D460C24D8F80C3027489B595F6897
:1081600022B2002104F0BEFB384609F029FA394654
:108170000246214804F050FD1F4804F063FD98F8C2
:10818000083001350934AB42A4B206F1040601DD22
:10819000422CE0D1B9F1000F13D109F1060999453C
:1081A0000CDA3C2301213B220391029300930192BC
:1081B00039233F223A21104804F0BCF805B0BDE84D
:1081C000F0830F2301213B2203910293009301923C
:1081D00039230C223A21084804F0ACF898F808300A
:1081E000DBE700213423009301913F230C22024856
:1081F00003F0B4FF9EE700BFD89EFF1FD09EFF1F75
:1082000010B5104C0121204604F076FB20460121D8
:1082100004F06CFB20463422552104F063FB204619
:108220000222094904F0F8FC20460522074904F01F
:10823000F3FC204604F006FD2046BDE8104003F0A4
:1082400073BD00BFD89EFF1F1C2A0100202A010019
:1082500070B50D46064609F0B3F900EB4000840006
:10826000002D36D0284609F0ABF900EB4000400065
:1082700023185B1003F16001091A282209B217487C
:10828000C3F1600404F02EFB0121144804F02EFB1E
:10829000284609F095F929460246104804F0BCFC2E
:1082A0000E4804F0CFFC02210C4804F01FFB21B261
:1082B00021220A4804F016FB304609F081F93146C4
:1082C0000246064804F0A8FC0448BDE8704004F0EB
:1082D000B9BC6410C4F16004E5E700BFD89EFF1F7D
:1082E000184B70B5B3F9003083EAE374A4EBE37480
:1082F000002B82B0A1B21EDB68466D46012300E070
:10830000134603EB830252009442F9DA0E4E91FBBE
:10831000F3F286FB03E403FB1211DB173032D3EBDD
:10832000A40389B205F8012BF1D119462B70FFF790
:108330008FFF02B070BD2D238DF800300DF10105C7
:108340006846DBE7CC9DFF1F6766666610B50D4B80
:108350001B5C51F82340237884B013B1012004B092
:1083600010BD04AA01A942F8103D2046A369984710
:10837000A38A9B07F2D401A80099FFF769FF0120A7
:1083800004B010BDBC9EFF1F2DE9F04F2F4DDFF84C
:10839000CCB0DFF8C4A0DFF8C8900FCD91B003AC2B
:1083A0000FC40FCD0FC40FCD0FC42B682360002561
:1083B000A8462F462E4600E09846BAF800302449D9
:1083C0005BF8232028461123F8F7F6F900EBC004E8
:1083D00000EB840089FB00340444C017C0EB643414
:1083E000C4F13C00C6F13C0207F14101012600B294
:1083F00008F1410300901BB2019612B209B2154870
:1084000003F0DEFE08EB060305F211153C2B2646B1
:10841000ADB24746D0D134226B210E4804F062FA47
:1084200000210C4804F062FA0B4B1B8810AA02EBE7
:10843000830353F8344C204609F0C2F8024605483D
:10844000214611B0BDE8F04F04F0E6BB2C26010038
:10845000FC1F0100D89EFF1F269CFF1F601E01000D
:108460000900028010B5424C424882B003F050FB34
:108470002378C3B906213F4804F038FA2378012B4A
:1084800037D90A22022B11463A486BD004F02AFA57
:1084900039490322374804F0BFFB364802B0BDE833
:1084A000104004F0CFBB354B1A7801210523002A78
:1084B00035D10191009311462E4803F0D1FE304B87
:1084C0001A78002A36D00523012201920093002257
:1084D0000A21284803F042FE2A4B1A78002A35D197
:1084E00001210523019100931421224803F0B8FED5
:1084F000C0E7254C2388092B32D9632B8CBF0A2176
:108500001F210A221B4804F0EDF92188194804F0C4
:10851000E9FB184802B0BDE8104004F093BB00220C
:10852000019100931146134803F018FE144B1A787A
:10853000002AC8D105230121019100930A210D4889
:1085400003F08EFE0F4B1A78002AC9D001220523B2
:108550000192009300221421064803F0FFFD89E7F1
:108560003021CEE704F0BEF90322084992E700BFAC
:10857000579FFF1FD89EFF1F2C2A0100A99EFF1F97
:10858000AA9EFF1F549EFF1F509EFF1F282A010016
:10859000F8B56D4D287840B96C4B1B6899425CD397
:1085A0006B4A012313702B70F8BD0C4600266948F6
:1085B000664F03F0ADFA04F6AC53324665483B60B3
:1085C00031212E7004F08EF901216248624D04F0D1
:1085D00093F931465F4804F089F905225F495D4807
:1085E00004F01AFB5B4804F02DFB0C2210215948C3
:1085F00004F078F90B225A49564804F00DFB052285
:108600005849544804F008FB524804F01BFB564BF1
:1086100050481C68A4F69803C3EB031385FB03259D
:108620001D441021DB172022C3EB652504F05AF905
:1086300040F6CC339C4205F124054FF022014FF067
:1086400004000BDCFFF7E2FC484B1C88064674B3C1
:10865000012C46D0022C41D00120F8BDFFF736FD99
:10866000092243493B4804F0D7FA2A22102139480D
:1086700004F038F93F4C374884FB0534EB17C3EB63
:10868000A404214604F02EFB01223B49314804F0AA
:10869000C3FA04EB8401A5EB41012E4804F022FB50
:1086A000012236492B4804F0B7FA0120F8BD3449BD
:1086B0001022284804F0B0FA264804F0C3FA2A220F
:1086C0001021244804F00EF93146224804F00AFB38
:1086D00007222C491F4804F09FFACBE70C222A49B5
:1086E000E7E70C2229491B4804F096FA194804F0E0
:1086F000A9FA2A221021174804F0F4F83146154847
:108700001C4E04F0EFFA07221E49124804F084FAC6
:1087100086FB0536EB17C3EBA60631460D4804F081
:10872000E1FA224614490B4804F076FA06EB86017A
:10873000A5EB4101074804F0D5FA22460F49054848
:1087400004F06AFA2046F8BDA08AFF1F389FFF1F79
:10875000549FFF1FD89EFF1F3B773B98302A010094
:10876000382A0100202A0100149EFF1FAC9DFF1F24
:10877000442A0100676666662C360100A4350100B4
:10878000502A0100642A01007C2A01006C2A0100A1
:108790002DE9F041754C2278002A05460F4614BF9A
:1087A0004FF001084FF000084ED1714E3368CB1ADC
:1087B000B3F5FA6F04D86B78A3B94046BDE8F081F1
:1087C0006C4B6D486D49DFF8D0E11A7001230370DE
:1087D0000988237026208EF8002000F0F1FD6B78C8
:1087E000002BEAD03760F9F7C9FB654A654B66494B
:1087F000127828781B78097802EB4303421E03EBBA
:1088000081030E2AD9D801A151F822F0FD88000079
:10881000C9880000BB870000FD880000BB870000FE
:10882000BB870000BB870000B1880000BB87000049
:1088300063880000BB870000BB870000BB87000087
:10884000BB8700005F880000AF215048484E02F00F
:108850000FFFFFF707FE002337602370ABE705F03B
:10886000F3FB4A4803F054F90221484804F03EF86B
:108870000F222321454804F035F805224449434896
:1088800004F0CAF9414804F0DDF91E2223213F48D3
:1088900004F028F805223F493C4804F0BDF93B4864
:1088A00004F0D0F9394803F03FFA00F0ADFC84E75A
:1088B000394D2B78012B50D9304B2620198800F0E8
:1088C0007FFD00232B7078E7002B3FF476AF013B50
:1088D000324A32F81330002B3FF46FAF274C304848
:1088E00025492D4A23804FF001080023037081F8A9
:1088F000008082F80080FFF7B5FD5EE793B1013B91
:10890000264A32F8131019B31C4B254D1A4C224A33
:1089100019800026012326202E702370137000F08A
:108920004FFD15E0154C1E4922880B7004284FF6A8
:10893000FF7002F1FF310CBF012202460A440E4EC5
:10894000154D02F07F0201320121228031702B701F
:10895000FFF788FD4FF001082FE70649064A01237B
:108960000020087013702370A6E700BFA08AFF1FC5
:10897000509FFF1F549FFF1F149CFF1F509EFF1FFF
:10898000A99EFF1FAA9EFF1F549EFF1FD89EFF1F78
:108990008C2A0100942A0100579FFF1F8C9DFF1F06
:1089A0008C9CFF1F2DE9F04F05468BB00F46AD485C
:1089B0000121164603F0A0FFAA8812F0010440F03E
:1089C000B080DFF8CC8298F80030002B7DD1AB79F5
:1089D000A54AD15CA1B9DFF8BCA279781AF8039056
:1089E00041B339780139072900F2B780DFE811F087
:1089F000F1005401B5006C01B500B500B500E90007
:108A00007C78002C00F0CA800139EC68387854F882
:108A10002170FC68411EB4F80080072900F2A7808D
:108A2000DFE811F074015901A5006C01A500A50053
:108A3000A5009F00DFF854A2DAF80020B21AB2F5C0
:108A4000967F75D9894A107801281ABF01201070C5
:108A50001170874A18BF0146D05CC0EB0900C0B254
:108A6000FFF7CCF80124CAF80060AB889B0770D5EB
:108A70007B78002B6DD0F9F781FA7E4B7E4A7F48D8
:108A80001B78127839780078022515FB02330A2901
:108A900003EB800300F04E810C295AD1002B58D0F3
:108AA00003F11900764E774A013B0021400080B265
:108AB00026F813100123157088F8003000F080FCB0
:108AC000714B032220461A702FE0664803F020F80D
:108AD0000121644803F00AFF62482246214603F060
:108AE00001FFAB88580725D42C68204608F068FDA4
:108AF000214602465B4804F08FF85A4804F0A2F879
:108B0000092201238DE80C0000217F23554803F042
:108B100057FB00212846FFF707FB002388F80030A9
:108B200055E7AB683146384698470BB0BDE8F08F43
:108B30000846FAE72B6804A8984704A808F040FD07
:108B400004A90246474804F067F8464804F07AF85A
:108B5000D6E720460BB0BDE8F08F00240AF803905A
:108B600083E70021D1543846FB699847FC68A4F894
:108B70000080002725223C238DE884004121182213
:108B8000384803F0EBFAE968A879FFF7DFFB374ACA
:108B90003E4B17701E600BB0BDE8F08F3B490A6872
:108BA000B21AB2F5967FD4D9304F0E603E78012EBE
:108BB00000F0B480E968184601233B70FFF7C6FB5C
:108BC000B3E7304AE9791170012288F800200024C7
:108BD000C4E72A7A013A4A45BFDD09F10104E4B24B
:108BE000A145BAD0224E16F803B0CBEB0900C0B2B3
:108BF0000021FFF703F82B7A052BD9461BD9CBEBC5
:108C00000402042A40F3AE80A4F1040BBBF1000F70
:108C1000C0F2B080063B5B45A8BF5B465FFA83F9B4
:108C2000AA791348B15C994205D000F8029001215D
:108C30002846FFF779FAC9EB0400C0B201210B4EB8
:108C4000FEF7DCFF002134230191009305483170C9
:108C500040230B223F21A14603F080FA0124AB7987
:108C60007CE700BFD89EFF1F449FFF1F559FFF1F3B
:108C7000D09EFF1FA99EFF1FAA9EFF1F549EFF1F8D
:108C80008C9DFF1F549FFF1F579FFF1F409FFF1F7B
:108C9000A08AFF1FBC9EFF1F0FFA89F1E868604C95
:108CA00050F821602168049134785E490498086086
:108CB000002C71D0012C7FF450AF5B4A317A88F8D8
:108CC00000401170002449E7B9F1000F50D009F1BC
:108CD000FF34E4B284E7B98A01F0040189B20029C3
:108CE0003FF440AF3B6A03929847039A00283FF451
:108CF0003DAFAB79FC680021D15438E77B8A43450E
:108D00003CD908F101081FFA88F830E73B8A43454F
:108D10003BD208F1FF381FFA88F828E725238DE8B1
:108D2000180042483C703C231822412103F016FAF7
:108D30003046FAE6002B3FF40CAF3D4A3D4E118819
:108D4000394A03F11900013B400080B226F81310A4
:108D5000012388F80030157000F032FB364B2046B6
:108D60001D70E2E6002A3FF755AF04F1FF3B4DE7E7
:108D70004C46F3E64FF000094B4651E7BB8ADA0751
:108D80007FF5F5AEB7F81080F1E6BB8AD9077FF51D
:108D9000EEAEB7F81280EAE62849C85CC0EB0900DD
:108DA00009F1010EC0B201214FF0340B02F803E0CB
:108DB000FEF724FFB6681D48019440230B223F2193
:108DC0000124CDF800B003F0C9F940230B223F2164
:108DD0001648CDF800B0019403F042FA214613483A
:108DE00003F084FD304608F0EBFBA0EB800000F1BF
:108DF0005F0109B20F220D4803F074FD304608F000
:108E0000DFFB31460246094803F006FF074803F03E
:108E100019FFE968A879FFF799FAAB799EE600BFD8
:108E2000949FFF1F409FFF1F549FFF1FD89EFF1F4F
:108E3000509EFF1F8C9DFF1F579FFF1FD09EFF1F3F
:108E40002DE9F047DFF808926D4B99F800601B6838
:108E5000DFF800A282B0003601934FF0030018BF84
:108E60000126019F9AF8008004F0A6FD0546042023
:108E700004F0A2FD0446052004F09EFD800040EAB7
:108E80004404062004F098FD2C4364B25D4944EA92
:108E9000C0000A7880F00F03DBB29A425A4A3CD0F5
:108EA0001760002259480B7003788DF800808DF808
:108EB000012053B3564A12684EF66021BA1A8A420C
:108EC00019D8022B59D0012B5FD0062B48D0032B89
:108ED00063D0042B69D0052B77D0072B7DD0082BCE
:108EE00000F08380092B68D016B14A4802F01CFFBD
:108EF00002B0BDE8F087484A484C002301212370A6
:108F000003701360938089F800103A46694644481C
:108F1000FFF748FD3043C6B2E6E71268BA1A1E2AC8
:108F20006BD99AF80020934222D0394C3D488AF8F8
:108F30000030012B276082EA030207609846B1D017
:108F4000042BAFD137480068381AB0F5C87FA9D9CB
:108F5000354C2068381A3228A4D927601A46A1E770
:108F60003A4669463148FFF71DFD3043C6B2BBE7BC
:108F7000012B4FF00002E3D1E4E73A4669462C4862
:108F8000FFF710FD3043C6B2AEE73A4669462948BE
:108F9000FFF708FD3043C6B2A6E73A4669462648C1
:108FA000FFF700FD3043C6B29EE73A4669462348C4
:108FB000FFF7F8FC3043C6B296E73A4669462048C8
:108FC000FFF7F0FC3043C6B28EE73A4669461D48CB
:108FD000FFF7E8FC3043C6B286E73A4669461A48CE
:108FE000FFF7E0FC3043C6B27EE73A4669461748D1
:108FF000FFF7D8FC3043C6B276E7002252E700BF45
:10900000949FFF1F589FFF1FC49EFF1F549FFF1F69
:109010004C9FFF1FD89EFF1F449FFF1F569FFF1F9F
:10902000582801005C9FFF1FCC9EFF1F882801006D
:10903000D4270100E8260100E8340100D8340100FB
:10904000D826010040270100243501009890FF1F19
:10905000A08AFF1FC89EFF1F28B11028044BA8BF7D
:10906000102018607047024B01201860704700BF45
:10907000609FFF1F38B50F4D2B78013B01381B0255
:10908000C4B203F47063200443F4404343F00C0380
:1090900000F4FE00184305F0F7FD2868013860F081
:1090A0003F00C0B204F01EFE2046BDE8384004F088
:1090B00019BE00BF609FFF1F70B5124D2B78013B9A
:1090C0001B0203F47063064643F43043080632047F
:1090D00000F0FE4043F00B03034302F4FE0018438C
:1090E0000C4605F0D1FD2868013860F04F00C0B291
:1090F00004F0F8FD304604F0F5FD2046BDE8704070
:1091000004F0F0BD609FFF1F70B5124D2B78013B3E
:109110001B0203F47063064643F41043080632044E
:1091200000F0FE4043F00903034302F4FE0018433D
:109130000C4605F0A9FD2868013860F06F00C0B248
:1091400004F0D0FD304604F0CDFD2046BDE870406F
:1091500004F0C8BD609FFF1F38B5104D2B78013B50
:109160001B0203F47063044643F41043000443F00D
:10917000090300F4FE00184305F086FD2868013855
:1091800060F06F00C0B204F0ADFD204604F0AAFD0F
:109190000020BDE8384004F0A5BD00BF609FFF1F60
:1091A00038B50E4D2B78013B1B0203F47063044667
:1091B00043F45043000443F00D0300F4FE00184351
:1091C00005F062FD2868013860F02F00C0B204F09D
:1091D00089FD2046BDE8384004F084BD609FFF1F34
:1091E00008B5002005F01AFE0028FAD108BD00BF1E
:1091F00008B564210720FFF75FFF7F210B20BDE842
:109200000840FFF759BF00BF10B500217B20FFF7D2
:1092100053FF0024E0B2FFF79FFF0134022004F067
:1092200001FC802CF6D110BD10B504464FF440600F
:1092300004F008FD04F060FD2CB1102C044BA8BF15
:1092400010241C6010BD024B01241C6010BD00BF27
:10925000609FFF1F10B5044641F0E00004F042FD9E
:1092600004F07F0004F03EFDC4F3C610BDE81040DA
:1092700004F038BD38B5134D2B78044641F6FF7223
:10928000A0F50050824203F1FF33A8BF02461B0243
:1092900002F5005203F47063100443F4604343F09A
:1092A0000E0300F4FE005204184302F0FE42104385
:1092B00005F0EAFC296801392046C9B2BDE838400A
:1092C000FFF7C8BF609FFF1F38B504460D46F0206A
:1092D00004F008FD35B1254414F8010B04F002FD3B
:1092E000AC42F9D1F720BDE8384004F0FBBC00BF28
:1092F00000B50B4B83B00246998818680090032A8A
:10930000ADF8041002D903B05DF804FB68460621ED
:109310008DF80520FFF7D8FF03B05DF804FB00BF10
:109320006435010000B50B4B024683B0186899887C
:109330000090131F4C2BADF8041002D903B05DF858
:1093400004FB684606218DF80520FFF7BDFF03B03A
:109350005DF804FB6C350100030203F4FE43C0F327
:10936000C6101843704700BF03784078DB0103F450
:109370007E5300F07F001843704700BF82B002AAFE
:10938000114642F8040D002012F8013B03F07F0360
:10939000914243EA0020F7D102B07047003210B486
:1093A00003884FF0010404FA01F418BF012202FA05
:1093B00001F123EA04020A43028010BC704700BF97
:1093C00070B5CEB20C46054603F0BEFE864203D011
:1093D0003146284603F0D2FE0135284603F0B4FE9C
:1093E000240A844205D021462846BDE8704003F097
:1093F000C5BE70BD38B5054603F0A6FE4FF00004AB
:1094000060F30704681C03F09FFE60F30F24A0B212
:1094100038BD00BFF8B504460020FFF7EBFF002C75
:1094200000F077814FF4AF610220FFF7C9FF0420FD
:109430004FF47A61FFF7C4FF0B2004F0BDFA002857
:1094400040F02E874FF496610620FFF7B9FF4FF4E6
:10945000FA610820FFF7B4FF4FF4FA610A20FFF722
:10946000AFFF40F6B8310C20FFF7AAFF4FF42F6191
:109470002220FFF7A5FF40F6AC512420FFF7A0FF04
:109480007D212A20FFF79CFF0C210E20FFF798FF7B
:1094900001211020FFF794FF02211220FFF790FF17
:1094A00000211420FFF78CFF00211620FFF788FF12
:1094B00002211820FFF784FF01211A20FFF780FF07
:1094C00001211C20FFF77CFF04211E20FFF778FFFD
:1094D00014212020FFF774FF01212620FFF770FFE1
:1094E00003212820FFF76CFF04212C20FFF768FFE1
:1094F00014212E20FFF764FF00213020FFF760FFCA
:109500000C213220FFF75CFF00213420FFF758FFC9
:1095100000213620FFF754FF00213820FFF750FFCD
:1095200000213A20FFF74CFF00213C20FFF748FFC5
:1095300000213E20FFF744FF00214020FFF740FFBD
:1095400000214220FFF73CFF1F214420FFF738FF96
:1095500013214620FFF734FF0E214820FFF730FF8C
:1095600011214A20FFF72CFF0A214C20FFF728FF8A
:1095700000214E20FFF724FF06215020FFF720FF97
:1095800002215220FFF71CFF0C215420FFF718FF87
:1095900000215620FFF714FF00215820FFF710FF8D
:1095A00001215A20FFF70CFF08215C20FFF708FF7C
:1095B0000A215E20FFF704FF00216020FFF700FF73
:1095C00004216220FFF7FCFE01216420FFF7F8FE72
:1095D00000216620FFF7F4FE0B216820FFF7F0FE64
:1095E0007F216A20FFF7ECFE00216C20FFF7E8FEE8
:1095F00000216E20FFF7E4FE00217020FFF7E0FE5F
:1096000000217220FFF7DCFE00217420FFF7D8FE56
:109610001F217620FFF7D4FE13217820FFF7D0FE1C
:109620000E217A20FFF7CCFE11217C20FFF7C8FE27
:109630000A217E20FFF7C4FE1F218020FFF7C0FE15
:1096400013218220FFF7BCFE0E218420FFF7B8FE15
:1096500011218620FFF7B4FE0A218820FFF7B0FE13
:1096600000218A20FFF7ACFE00218C20FFF7A8FE26
:1096700000219620FFF7A4FE00219820FFF7A0FE0E
:1096800000219A20FFF79CFE05219C20FFF798FE01
:1096900006219E20FFF794FE0021A020FFF790FEF8
:1096A0007F21A220FFF78CFE40F2A461A420FFF7E7
:1096B00087FE4FF4E161A620FFF782FE0021A8207B
:1096C000FFF77EFE0021AA20FFF77AFE0221AC20E0
:1096D000FFF776FE0121AE20FFF772FE0121B020D8
:1096E000FFF76EFE0B21B220FFF76AFE2A21002051
:1096F000FFF766FE0220FFF77DFEB0F5805F0346B0
:1097000016D34FF4AF610220FFF75AFE4FF4AF6358
:109710000EE04FF6FF7398423FF484AE2A2840F0E3
:10972000CB850220FFF766FEB0F5805F0346E8D2E6
:10973000D24A04201380FFF75DFEB0F5805F034638
:1097400080F06285CE4A06201380FFF753FEA0F515
:109750002F739BB2B3F57A6F024606D940F62821E3
:109760000620FFF72DFE40F62822C64B08201A805F
:10977000FFF740FEA0F52F739BB2B3F57A6F024658
:1097800006D940F6E4410820FFF71AFE40F6E4420D
:10979000BD4B0A201A80FFF72DFEA0F5FA739BB28D
:1097A00040F6AC518B42024606D94FF4FA610A20CA
:1097B000FFF706FE4FF4FA62B44B0C201A80FFF755
:1097C00019FEA0F5FA739BB240F6AC518B420246EB
:1097D00006D940F6B8310C20FFF7F2FD40F6B8325A
:1097E000AB4B0E201A80FFF705FE1828034600F247
:1097F0000A84A84A10201380FFF7FCFD431E9BB289
:109800000F2B024604D901211020FFF7D9FD0122B8
:10981000A14B12201A80FFF7EDFD0A28034600F243
:10982000EC839E4A14201380FFF7E4FD01280346D1
:1098300004D900211420FFF7C3FD0023984A162005
:109840001380FFF7D7FD7F28034600F2D083954AA7
:1098500018201380FFF7CEFD0528034600F2C183D0
:10986000914A1A201380FFF7C5FD0C28034600F229
:10987000C4848E4A1C201380FFF7BCFD04280346D5
:1098800000F2B4848A4A1E201380FFF7B3FD092832
:10989000034600F2A484874A20201380FFF7AAFD24
:1098A0004628034600F29484834A22201380FFF75F
:1098B000A1FDA0F5FA739BB240F6AC518B42024673
:1098C00006D94FF42F612220FFF77AFD4FF42F6263
:1098D0007A4B24201A80FFF78DFDA0F5FA739BB216
:1098E00040F6AC54A342024604D921462420FFF797
:1098F00067FD2246724B26201A80FFF77BFD7F28EA
:10990000034600F25E846F4A28201380FFF772FD41
:109910000628034600F24E846B4A2A201380FFF784
:1099200069FDA0F132039BB2B3F5967F024604D9DC
:109930007D212A20FFF744FD7D22644B2C201A80D4
:10994000FFF758FD0C28034600F22D84604A2E20B4
:109950001380FFF74FFD1E28034600F21D845D4A69
:1099600030201380FFF746FD0928034600F20D84DE
:10997000594A32201380FFF73DFD1E28034600F2AE
:10998000FD83564A34201380FFF734FD7F280346B9
:1099900000F2EE83524C36202380FFF72BFD7F2808
:1099A000034600F2DF8338206380FFF723FD7F2822
:1099B000034600F2D1833A20A380FFF71BFD7F28E6
:1099C000034600F2C3833C20E380FFF713FD7F28AA
:1099D000034600F2B5833E202381FFF70BFD7F286D
:1099E000034600F2A78340206381FFF703FD7F2831
:1099F000034600F299834220A381FFF7FBFC394D17
:109A000028804420FFF7F6FC3028034600F28683C6
:109A1000354A46201380FFF7EDFC3028034600F25C
:109A20007783324C48202380FFF7E4FC302803463C
:109A300000F268834A206380FFF7DCFC302803468D
:109A400000F25A834C20A380FFF7D4FC3028034651
:109A500000F24C834E20E380FFF7CCFC0128034644
:109A600004D900214E20FFF7ABFC0023204A5020F0
:109A70001380FFF7BFFC431E3CE000BFB49CFF1FF8
:109A80007C9EFF1F769CFF1F4C9EFF1F189EFF1F92
:109A9000389CFF1F0E9CFF1FCC9DFF1F029EFF1FC7
:109AA000AA9CFF1F129CFF1FBA9CFF1F5C9CFF1FFC
:109AB000569CFF1F409CFF1F5E9EFF1FC69DFF1F01
:109AC000C29DFF1F509EFF1F269EFF1F749EFF1FFB
:109AD000269CFF1FA09CFF1F8C9EFF1F4E9EFF1FFA
:109AE0008C9DFF1F309CFF1F329CFF1F289EFF1F75
:109AF000549CFF1F9BB20B2B024604D90621502019
:109B0000FFF75EFC0622CF4B52201A80FFF772FC53
:109B10000428034600F2E482CB4A54201380FFF766
:109B200069FC431E9BB21D2B024604D90C21542014
:109B3000FFF746FC0C22C54B56201A80FFF75AFC53
:109B40000128034604D900215620FFF739FC0023E1
:109B5000BF4A58201380FFF74DFC7F28034600F2D0
:109B6000B982BC4A5A201380FFF744FC431E9BB2C3
:109B7000092B024604D901215A20FFF721FC0122BA
:109B8000B54B5C201A80FFF735FC431E9BB2102BAF
:109B9000024604D908215C20FFF712FC0822AF4BD3
:109BA0005E201A80FFF726FC431E9BB21D2B024647
:109BB00004D90A215E20FFF703FC0A22A84B60208B
:109BC0001A80FFF717FC0228034600F27D82A54A9F
:109BD00064201380FFF70EFC0128034604D90121FD
:109BE0006420FFF7EDFB01239F4A62201380FFF7FB
:109BF00001FCC31E9BB2012B024604D90421622042
:109C0000FFF7DEFB0422994B66201A80FFF7F2FB78
:109C10007F28034600F25282954A68201380FFF79E
:109C2000E9FB7F28034600F24382924A6A201380B0
:109C3000FFF7E0FB7F28034600F234828E4A6C2057
:109C40001380FFF7D7FB0228034600F225828B4AD8
:109C50006E201380FFF7CEFB1928034600F2168210
:109C6000874A70201380FFF7C5FB0228034600F2E5
:109C70000782844A72201380FFF7BCFB0628034644
:109C800000F2F881804A74201380FFF7B3FB0528A7
:109C9000034600F2E9817D4A8A201380FFF7AAFB80
:109CA0000A28034600F2DA81794A8C201380FFF7F4
:109CB000A1FB0428034600F2CB81764A982013804A
:109CC000FFF798FB0128034604D900219820FFF7ED
:109CD00077FB0023704A9A201380FFF78BFB012843
:109CE000034604D900219A20FFF76AFB00236B4A40
:109CF00096201380FFF77EFB0B28034600F2A2811B
:109D0000674A9C201380FFF775FB831E9BB2032BD1
:109D1000024604D905219C20FFF752FB0522614B26
:109D200076201A80FFF766FB3028034600F2848114
:109D30005D4A78201380FFF75DFB3028034600F270
:109D400075815A4C7A202380FFF754FB3028034654
:109D500000F266817C206380FFF74CFB30280346CD
:109D600000F258817E20A380FFF744FB3028034691
:109D700000F231818020E380FFF73CFB302803466E
:109D800000F223814A4A82201380FFF733FB3028F8
:109D9000034600F21481474C84202380FFF72AFBFE
:109DA0003028034600F2058186206380FFF722FBFE
:109DB0003028034600F2F7808820A380FFF71AFBC3
:109DC0003028034600F2E980A020E380FFF712FB71
:109DD0000128034604D90021A020FFF7F1FA00234F
:109DE000354A9E201380FFF705FBC31E9BB20C2B48
:109DF000024604D906219E20FFF7E2FA06222F4BE5
:109E0000A2201A80FFF7F6FA431E9BB27E2B024671
:109E100004D97F21A220FFF7D3FA7F22284BA42068
:109E20001A80FFF7E7FAA0F5AF639BB2B3F5167F90
:109E3000024647D940F2A461A420FFF7C1FA40F2DC
:109E4000A4623FE02089FF1F2E89FF1FA489FF1F06
:109E5000969CFF1F129EFF1F089CFF1FA889FF1FD3
:109E60002C89FF1FBE9DFF1F209EFF1F649CFF1FAC
:109E7000609EFF1F949CFF1F449CFF1FFC9BFF1FC5
:109E8000AC9EFF1FAC9DFF1F889EFF1F449EFF1FBF
:109E9000CE9DFF1FBC9DFF1F429CFF1F9A9CFF1F72
:109EA0000C9EFF1F289CFF1F3A9CFF1F9C9DFF1FBD
:109EB0003C9CFF1FA49DFF1F309EFF1F9089FF1F2A
:109EC000529EFF1FD84BA6201A80FFF793FAA0F5E9
:109ED000AF639BB2B3F5167F024606D94FF4E1613A
:109EE000A620FFF76DFA4FF4E162D04BA8201A804C
:109EF000FFF780FA0628034600F2CC81CC4AAA205C
:109F00001380FFF777FA0328034600F2BD81C94AA0
:109F1000AC201380FFF76EFA0328034600F2AE81EF
:109F2000C54AB0201380FFF765FA0328034600F204
:109F30009F81C24AAE201380FFF75CFA7F28034658
:109F400000F29081BE4AB2201380FFF753FA7F28B7
:109F500000F263812B88DFF808E3BA4FBA4ABB4DA1
:109F6000BB4EBC4CBC4903F0010CAEF800C0C3F3BF
:109F7000400EA7F800E0C3F380071780C3F3C007C3
:109F8000B64A2F70C3F30017C3F34015C3F3801311
:109F9000378025800B801080F8BD0A218820FFF7CC
:109FA0000FFA0A2310E711218620FFF709FA11237F
:109FB00002E70E218420FFF703FA0E23F4E61321B3
:109FC0008220FFF7FDF91323E5E61F218020FFF72C
:109FD000F7F91F23D6E60A217E20FFF7F1F90A23BD
:109FE000C8E602211820FFF7EBF9022338E400212C
:109FF0001620FFF7E5F9002329E402211220FFF7DC
:10A00000DFF902230DE40C210E20FFF7D9F90C2310
:10A01000FFF7EFBB11217C20FFF7D2F91123A1E656
:10A020000E217A20FFF7CCF90E2393E61321782036
:10A03000FFF7C6F9132384E61F217620FFF7C0F946
:10A040001F2375E600219620FFF7BAF9002357E693
:10A0500000218C20FFF7B4F900232EE600218A208E
:10A06000FFF7AEF900231FE600217420FFF7A8F9DF
:10A07000002310E600217220FFF7A2F9002301E679
:10A0800000217020FFF79CF90023F2E500216E20EB
:10A09000FFF796F90023E3E500216C20FFF790F924
:10A0A0000023D4E57F216A20FFF78AF97F23C5E5E5
:10A0B0000B216820FFF784F90B23B6E50021662009
:10A0C000FFF77EF90023A7E500216020FFF778F96C
:10A0D00000237CE500215820FFF772F9002340E5BA
:10A0E00002215220FFF76CF9022315E50A214C20CA
:10A0F000FFF766F90A23ADE411214A20FFF760F962
:10A1000011239FE40E214820FFF75AF90E2391E412
:10A1100013214620FFF754F9132382E41F21442022
:10A12000FFF74EF91F2373E400214020FFF748F9A1
:10A13000002360E400213E20FFF742F9002352E4AF
:10A1400000213C20FFF73CF9002344E400213A20A1
:10A15000FFF736F9002336E400213820FFF730F905
:10A16000002328E400213620FFF72AF900231AE40F
:10A1700000213420FFF724F900230BE40C213220C6
:10A18000FFF71EF90C23FFF7FCBB00213020FFF77F
:10A1900017F90023FFF7ECBB14212E20FFF710F96D
:10A1A0001423FFF7DCBB04212C20FFF709F904235B
:10A1B000FFF7CCBB03212820FFF702F90323FFF7A9
:10A1C000ABBB01212620FFF7FBF80123FFF79BBB68
:10A1D00014212020FFF7F4F81423FFF765BB0421B6
:10A1E0001E20FFF7EDF80423FFF755BB01211C20CB
:10A1F000FFF7E6F80123FFF745BB01211A20FFF71F
:10A20000DFF80123FFF735BB4FF47A610420FFF735
:10A21000D7F84FF47A63FFF795BAB2200B21FFF716
:10A22000CFF80B2096E600BFB89CFF1F389EFF1F9B
:10A230000A9CFF1F7A9CFF1F229EFF1FB09DFF1FDD
:10A240004C9CFF1F749CFF1FA29CFF1FB29DFF1F11
:10A25000C09DFF1F249EFF1FD49DFF1F6E9CFF1FEC
:10A260000E9EFF1F0121AE20FFF7AAF8012369E629
:10A270000121B020FFF7A4F801235AE60221AC2007
:10A28000FFF79EF802234BE60021AA20FFF798F87B
:10A2900000233CE60021A820FFF792F800232DE6DA
:10A2A00040F628210620FFF78BF840F6E44108200D
:10A2B000FFF786F8FFF7D0B817287FF6B3A819285C
:10A2C0007FF622A91B287FF63FA91C283FF454A93A
:10A2D0001E287FF659A91F283FF45EA920283FF4C5
:10A2E00077A921283FF480A922283FF485A92328B3
:10A2F0003FF48EA924283FF4BFA925283FF4C4A920
:10A3000026283FF4C5A927283FF4CAA928283FF4E6
:10A31000D5A929287FF4EAA9FFF7D8B9F8B5C5204F
:10A3200006F0C6FB204B214A054603CB1368C5F84F
:10A3300003001A0CB420C5F807102B80AA70FFF791
:10A340000BF82E46002426F80B0FA0B2FFF752F8A8
:10A35000FFF702F80234B42C26F8020FF5D16C1E78
:10A3600005F1C0064FF0FF3014F8013F08275840B0
:10A370000F4B40F300017A1E0B4012F0FF0783EAF7
:10A380005000F5D1B442EFD1C043FEF7F7FF3A4693
:10A39000C5F8C100C521284604F0C4FC2846BDE824
:10A3A000F84006F08DBB00BF783501007435010020
:10A3B0002083B8EDF0B50E4B0E4C054693E8070030
:10A3C00085B024682E88AD7801AB83E80700270CA0
:10A3D000184600220B21ADF804408DF80670ADF848
:10A3E0000C608DF80E5004F09DFC05B0F0BD00BF70
:10A3F0008435010074350100F0B5124B124D1E6812
:10A40000124F0FCD87B06C460FC495E8030044F897
:10A41000040B38683B79CDF80D00320C2A202180DE
:10A420008DF802208DF81130ADF80060FEF794FF32
:10A430000022ADF80B001221684604F073FC07B04F
:10A44000F0BD00BF7435010090350100202A0100E5
:10A45000002004F0E3BC00BF02F02EBE70B5124C29
:10A4600082B00025402306462946204600930195E8
:10A470008023202201F072FE20222946204602F08D
:10A4800031FA2046012102F037FA304607F098F8F9
:10A4900031460246204602F0BFFB204602B0BDE82E
:10A4A000704001F041BC00BFD89EFF1FF0B5C42929
:10A4B00083B075D90546441E00F1C0064FF0FF3049
:10A4C00014F8012F08275040404A40F300017B1E3A
:10A4D0000A4013F0FF0782EA5000F5D1B442EFD1F1
:10A4E000C043FEF74BFF0146D5F8C1000190019A29
:10A4F000914202D0B2F17F2F0BD105F10B00FEF794
:10A5000033FFB4280BD03248FFF7A8FF002003B078
:10A51000F0BD3048FFF7A2FF384603B0F0BD05F1AB
:10A520000D00FEF721FF2A2840D1002440F6AC564A
:10A5300013E004281AD0062821D008281FD00A28A2
:10A5400028D00C2822D1A1F5FA7292B2B24201D8D9
:10A55000FEF736FF0234B42C0ED004F10D0028446F
:10A56000FEF702FF022C0146A0B2E2D1B1F5805FF6
:10A57000EED30234B42CF0D1012003B0F0BDA1F52C
:10A580002F7292B2B2F57A6FE4D8E1E7222801D0B7
:10A59000242811D1A1F5FA7292B2B242DAD8D7E7E3
:10A5A0000D48FFF75BFF002003B0F0BD0B48FFF73D
:10A5B00055FF002003B0F0BD2A28C9D1A1F1320215
:10A5C00092B2B2F5967FC5D8C2E700BF2083B8ED3E
:10A5D000D4350100C0350100A8350100E83501007F
:10A5E00003290CD970B5461C82B005460C4630468E
:10A5F00003222A4907F052F810B102B070BD70472B
:10A600000B2C05D905222649281D07F047F840B133
:10A610002448FFF723FF244802B0BDE87040FFF74D
:10A62000C9BE05F10901032201A807F087F801A8B6
:10A6300003221E4907F032F8D8B103221C4901A8B1
:10A6400007F02CF808B301A803221A4907F026F8EE
:10A65000B0B91948FFF702FFA11E89B23046FFF7D3
:10A6600025FF0028C9D0154802B0BDE87040FFF7AB
:10A67000F5BE1348FFF7F2FEFFF750FE1148F3E76F
:10A680001148FFF7EBFE1148C6E71148FFF7E6FE59
:10A6900002B0BDE87040FFF7AFBE00BF74350100E7
:10A6A000302A01000036010014360100183601007E
:10A6B00040360100583601005C360100703601005A
:10A6C0001C36010030360100843601009836010046
:10A6D000443601002DE9F043174D2B6883B08146C5
:10A6E0000F469046F3B1154E34880A1992B21846B7
:10A6F0001146328006F05AFD28603A464946204409
:10A7000002F06CFDB8F1000F09D031882868FFF71E
:10A7100067FF286806F0D4F900232B60338003B06C
:10A72000BDE8F083054E01930846318006F0C0F97C
:10A73000019B28601C46E0E7689FFF1F649FFF1F86
:10A7400010B51F4C4FF4FA70FBF796FE204601F04F
:10A75000DFF900221146204602F0C4F8204601210C
:10A7600002F0CAF82046002102F0C0F80B22154979
:10A77000204602F051FA204602F064FA0F221249F4
:10A78000204602F049FA204602F05CFA0F490722FF
:10A79000204602F041FA204602F054FA204601F029
:10A7A000C3FA0B4B0B4A1A604FF4FA70FBF764FEC6
:10A7B000FFF722FE0848BDE81040FFF74FBE00BF7C
:10A7C000D89EFF1F9C360100A8360100B836010054
:10A7D00020A1FF1FD5A60000C03601000020704751
:10A7E00090F8392090F83800101A704790F83830F7
:10A7F00090F839209A4205D95A1C034480F8382031
:10A80000187E70474FF0FF30704700BF90F8383027
:10A8100090F839209A4286BF1B18187E4FF0FF30FF
:10A82000704700BF704700BF38B50546B0F85E00FE
:10A8300090B195F85D301446C3F1210294420CD8D2
:10A8400005F13B001844224602F0C8FC95F85D3043
:10A85000234485F85D30204638BD01201446287118
:10A86000EEE700BFB0F85E306BB190F85D30202BA2
:10A8700007D8C218013380F85D30012082F83B1000
:10A880007047012303710020704700BF0023426915
:10A8900080F8383080F8393080F85C3080F85D30EE
:10A8A00080F85E3080F85F3006CA30B40D68046905
:10A8B00043662A4383660A60A370426990F8613058
:10A8C0001649146813441D7A5B7B01EBC5051B0216
:10A8D0006D6803F4E06343F064032B6090F862302A
:10A8E00013449D7CDB7D01EBC5011B02496803F429
:10A8F000E06343F064030B6021685368194205D09C
:10A90000036927225A70036904229A71036920227D
:10A910005A71036980229A7030BC7047F44101007B
:10A9200043690CCB12681A420CD0094B99420AD9E0
:10A93000084B9942036994BF1A220D225A70036989
:10A9400004229A717047036927225A70F7E700BF03
:10A950007F1A06003F420F0010B50269D378DBB2C0
:10A96000D90604463DD510215806D17038D503F0DC
:10A97000040303F0FF02002B51D03D49626E002317
:10A980000B7084F85D30002A5BD0904794F85D30FE
:10A99000002B56D02369D0229A70236994F83B206B
:10A9A0001A712369012284F85C200222DA7010BD3A
:10A9B000304B84F860009C424AD02F4B9C4252D0CE
:10A9C00094F8391013791F29DBB207D8284800788A
:10A9D00020B16018013184F8391003760223D37056
:10A9E00010BD5906C3D4917801F0100101F0FF00A9
:10A9F0000029DDD013F001031ED194F85C1094F807
:10AA00005D00884281BF4B1C091984F85C3091F8C5
:10AA10003B3013712369D0229A702269DEE72369E3
:10AA200084F83920C0229A702369114A19790121CA
:10AA300011700222DA7010BDC0239370226913795D
:10AA4000CCE70122002384F85D2084F83B30A1E7A5
:10AA5000626994F86130094913440322187A02F0BC
:10AA600043FD2269ACE7626994F861300449F3E779
:10AA70006C9FFF1FE090FF1F4C91FF1FE1AA000099
:10AA8000EDAA00000369DB7803F0200373B190F8AE
:10AA900060300133DBB2012B80F860301AD9426993
:10AAA00090F861301344187A02F09ABD70B542698B
:10AAB00003F0FF0590F8613013440446187A02F061
:10AAC0008FFDA36E5BB184F8385094F83900BDE86F
:10AAD0007040184790F85F30002BE0D0704770BD91
:10AAE0000148FFF7CFBF00BFE090FF1F0148FFF70D
:10AAF000C9BF00BF4C91FF1F2DE9F047374FDFF86A
:10AB0000E0903B68026982B006460093DDF8008061
:10AB10000021A025D3789B065BD53B680193019B60
:10AB2000C8EB03030F2BF5D949B1102BF2D000204D
:10AB30009070336980229A7002B0BDE8F087726924
:10AB400096F8613013440521187A02F043FF7269C8
:10AB500096F861301344012193F812A0504602F098
:10AB600039FF09240021504602F020FF2B46013B0B
:10AB7000FDD10121504602F019FF2B46013BFDD1CA
:10AB8000013CEFD1706996F8611001444FF4A07256
:10AB90000C7A4B7B09EBC4011B02496803F4E063A8
:10ABA00043F064030B6096F862300344997CDB7DCC
:10ABB00009EBC1011B02496803F4E06343F064033D
:10ABC0000B60013AFDD13269D3789B064FF0010149
:10ABD000A3D4012002B0BDE8F08700BF949FFF1FFF
:10ABE000F4410100F0B503691222DA70026993782A
:10ABF00003F0200385B004460D46002B5ED0B4233D
:10AC000093703C4922690B680093009E05E00B6835
:10AC10000193019B9B1B042B42D8D37803F02003A4
:10AC200003F0FF00002BF2D094F85D30002B31D000
:10AC30004FF0000E4FF0020C04EB0E0393F83B3084
:10AC400013710B680393039F206907E09B060DD5E2
:10AC50000B680293029BDB1B052B28D8C378DBB261
:10AC600003F0020202F0FF06002AEFD080F803C0D2
:10AC70002669F378DBB2DF0632462DD49F062BD54A
:10AC8000DB0731D40EF1010E94F85D305FFA8EFED1
:10AC90007345D1D800201DBB002384F85E3004E04A
:10ACA0009070236980229A70042005B0F0BD8670F0
:10ACB0002369802204209A7005B0F0BD03F0FF06DE
:10ACC000FFF71AFF10B9042005B0F0BD236984F81E
:10ACD0005F60B0229A7094E78023B3700420DAE7B3
:10ACE00026698023B370D7E7BEF1000F0CBF0220A6
:10ACF0000320F6E7949FFF1F2DE9F0410669002528
:10AD0000122780F8385080F83950F770D0F810C00A
:10AD10009CF802E00EF0200E88B0044688461546E6
:10AD20001E46BEF1000F49D0B4238CF80230784B98
:10AD300021691A680092DDF800E006E01A680192C5
:10AD40000198CEEB0000042830D8C87800F020002D
:10AD500000F0FF070028F1D04FEA480242F001025C
:10AD6000D2B20A711A680292DDF808E0206906E0A2
:10AD70001A6803920399CEEB010105292AD8C178FC
:10AD800001F0020101F0FF070029F1D04FF0020CA1
:10AD900080F803C02269D17811F0110722D12DBBB0
:10ADA000002E0CBFA0238023937003E08F702369D3
:10ADB00080229A70384608B0BDE8F0810EF0FF0797
:10ADC000FFF79AFE0028F5D0236984F85F70B0225F
:10ADD0009A70ACE787702369802238469A7008B071
:10ADE000BDE8F081802393700027E3E7012D75D043
:10ADF000A021917021690A79BE4667464FF0A80CE0
:10AE00001A680492049805E01A680592059A121AC5
:10AE1000052A4AD8CA7802F0020202F0FF08002A86
:10AE2000F2D0CF702169CA78D2B212F0100F084662
:10AE30005AD1920658D5013DEDB2012D49D0BEF14F
:10AE40001F0F3BD90A79012DDAD11A680692069DA7
:10AE500005E01A680792079A521B052A46D8C2785D
:10AE600002F0020202F0FF01002AF2D00223C370B6
:10AE70002269D378DBB2D9063AD49B0634D5B02305
:10AE8000BEF11F0F93703FD8226904EB0E031279B5
:10AE90001A760EF1010E5FFA8EFE16B1236980223A
:10AEA0009A7084F839E0774684E781F80280236954
:10AEB00080229A70774684F839E07BE704EB0E0233
:10AEC00091F8048082F818800EF1010E5FFA8EFE70
:10AED000B9E781F802C021690846B0E7A82191705E
:10AEE0002069BE460279B0E7774663E78170DEE706
:10AEF0001021A023D170013BFDD12269937803F08A
:10AF0000F7037746937055E723691B79C5E700BFC0
:10AF1000949FFF1F0148FFF71FBD00BFE090FF1F78
:10AF20000148FFF719BD00BF4C91FF1F704700BFDC
:10AF300038B5144C037801225B000546204684F89E
:10AF40003B3084F85E2084F85D20FFF78BFC2046C0
:10AF50000021FFF747FE0B4C2978012320461A46B3
:10AF6000FFF7CAFE0128F6D194F8383094F839205A
:10AF70009A4205D9E218013384F83830107E38BD82
:10AF8000FF2038BDE090FF1F38B51B4C037801222D
:10AF90005B000546204684F83B3084F85E2084F848
:10AFA0005D20FFF75FFC20460021FFF71BFE124CDF
:10AFB0002978204601230222FFF79EFE0228F6D1BF
:10AFC00094F8382094F839108A420FD2531CDBB21F
:10AFD000A018994284F83830007E0AD923440232FE
:10AFE0001B7E84F8382040EA032038BD4FF6FF70FE
:10AFF00038BD40F47F4038BDE090FF1F0C2901D9D7
:10B00000002070470231490001F0FE01FFF7BCBF8C
:10B0100070B50C4C0378164601255B00204684F879
:10B020003B3084F85E5084F85D50FFF71BFC3146DE
:10B030002046FFF717FC29462046BDE87040FFF781
:10B04000D1BD00BFE090FF1FF8B505460F4616467C
:10B05000412421463A462846FFF7DAFF611C0234B4
:10B06000C9B232462846E4B2FFF7D2FF592CF0D1DC
:10B07000F8BD00BF38B504460D463548FFF706FC5D
:10B080006322802120462570FFF7C2FF012002F0D5
:10B09000C9FC204600225E21FFF7BAFF20465D2151
:10B0A000FFF746FF242801D0002038BD20460622A5
:10B0B0000C21FFF7C9FF204601222B21FFF7A8FF33
:10B0C000204601222C21FFF7A3FF20460E222D212E
:10B0D000FFF79EFF204600222E21FFF799FF204612
:10B0E00001222F21FFF794FF204605223021FFF790
:10B0F0008FFF204601223121FFF78AFF20460022E0
:10B100003221FFF785FF204600223321FFF780FF21
:10B11000204600223421FFF77BFF20460022352104
:10B12000FFF776FF204600225B21FFF771FF2046E4
:10B1300010225C21FFF76CFF204620225D21FFF7E3
:10B1400067FF20468F225E21FFF762FF012038BD96
:10B15000E090FF1F10B4047F4160022CC26002D057
:10B1600010BC01F0D7BB836810BC184790E80C00F6
:10B17000F0B41C6859682568164F174E29432160A2
:10B18000164D17491760D66015611160417A154A4E
:10B190005C180A3194F8244053F8215002EBC401A2
:10B1A00049680D60017A5C1803EB8101247ECD694A
:10B1B00002EBC40149680D60817A581803EB8103E2
:10B1C00090F83000596B02EBC002F0BC5368196074
:10B1D000704700BF01401F000110003801100078C7
:10B1E00000001F80F4410100704700BFF0B50C1E45
:10B1F000BDF8146034DBB0F906701919B942C4BF48
:10B200003B1B1BB2002BA6461CDD002A1146B8BF13
:10B21000D11D02F00705CC10826A012007FB04E172
:10B22000A840012E0A44C0B21ED00CD3022E09D170
:10B23000013B12FA83F3013A12F8011F41409A428E
:10B240001170F9D1F0BDC043013B12FA83F3C0B2D3
:10B25000013A12F8011F014093421170F9D1F0BD7B
:10B2600023441BB20024C6E7013B12FA83F3013AE0
:10B2700012F8011F01439A421170F9D1F0BD00BFCD
:10B28000F8B50D1E0EDB14461F46064601F03AFBCC
:10B29000A84207DD002C05DB304601F037FBA04259
:10B2A00001DCF8BDF8BD304601F02AFB022853D07E
:10B2B00003284BD0012806D16540F3886C406540D7
:10B2C000013B5D1B2DB2012F03D02AD3022F14D0D6
:10B2D000F8BD002C2246B6F90630B06AB8BFE21DB0
:10B2E00042F3CF0202FB035504F00704435D012142
:10B2F00001FA04F41C434455F8BD002C2246B6F96B
:10B300000630B06AB8BFE21D42F3CF0202FB03551C
:10B3100004F00704435D012101FA04F45C40445544
:10B32000F8BD002C2246B6F90630B06AB8BFE21D5F
:10B3300042F3CF0202FB035504F00704435D0121F1
:10B3400001FA04F423EA04044455F8BD3389013BAF
:10B35000591B25460CB2B6E7F18832890139013A0A
:10B360004D1B141B2DB224B2ADE700BF2DE9F041F7
:10B37000079E9DF91880089D04461F4600F0C0FFF7
:10B380000D4B0E480E4984F83380FF22002F08BF72
:10B390001F4684F82F20002384F8302084F83120C1
:10B3A00084F832202060A665E565676261652362E6
:10B3B000A3622046BDE8F081E090FF1F4C370100FA
:10B3C0000110013810B50446806A034B236008B1B0
:10B3D00005F076FB204610BD4C370100F8B5436AF6
:10B3E000DBB190F82C200125AA4083F83B2083F89C
:10B3F0005E5083F85D500446406A03680E461B6841
:10B4000000219847606A036831461B6898472946BF
:10B41000606ABDE8F840FFF7E5BBC26BC56C136816
:10B42000046A23EA050313604CB122684FF000431D
:10B43000D3625163D36A002BFCDA936BF8BD836B44
:10B44000466B0825802410E03768426C3A4332602E
:10B450001F68826C3A431A601A68876C013D22EAC1
:10B4600007024FEA54041A6007D02142ECD1326837
:10B47000476C22EA07023260EAE7F8BD70B504467D
:10B48000406A0D4600282BD0A16DFFF749FA002D28
:10B4900020460CBFA621A721FFF7A0FF606A20B1BC
:10B4A000E16DBDE87040FFF73BBA216C226D086882
:10B4B000236A02430A6093B1DA7A82B1D00703D5D6
:10B4C000224A99691160DA7A910703D5204AD9692D
:10B4D0001160DA7A520702D51E4A1B6A136070BDEA
:10B4E000236A002B2BD0D97A626DE1B172B6D97A7A
:10B4F000CE0706D51848D9680668314099610160C1
:10B50000D97A880706D51548196906683140D96186
:10B510000160D97A4E0705D511485969066831404E
:10B520001962016062B61B68D968914207D00D4864
:10B5300018600D49DA6042F0804018611960226C91
:10B54000216D136823EA01031360A0E700E100E026
:10B5500004E100E008E100E080E100E084E100E0D7
:10B5600088E100E001403F0000003F80436A2DE990
:10B57000F04105460E469046002B3ED090F82C1028
:10B580000124A14083F83B1083F85E4083F85D40BE
:10B59000406A036800211B6808F1FF379847FFB233
:10B5A000B8F1000F23D03744A046013E686A16F870
:10B5B000011F03681B6898470134B742E4B216D0F4
:10B5C000202CF3D10121686AFFF70CFB95F82C20A1
:10B5D0006B6A520083F83B2083F85E8083F85D80BD
:10B5E000686A036800211B6898470124DEE7686ADF
:10B5F0000121BDE8F041FFF7F5BAC26BC16C1368D9
:10B6000023EA010306EB080413604FF00048A6424A
:10B610000ED02B6A16F801EB63B11A68C2F82C80C1
:10B62000C2F834E0D36A002BFCDAA642936BF0D167
:10B63000BDE8F081AB6BD5F834C008208021DCF880
:10B6400000206F6C1EEA010F14BF3A43BA43CCF8D6
:10B6500000201A68AF6C3A431A601A68AF6C013860
:10B6600022EA07024FEA51011A60E8D1CFE700BF92
:10B6700070B50446406A0D46002828D0A16DFFF73A
:10B680004FF920462946FFF7A9FE606A20B1E16D17
:10B69000BDE87040FFF744B9216C226D0868236A49
:10B6A00002430A6093B1DA7A82B1D00703D5234A04
:10B6B00099691160DA7A910703D5214AD969116035
:10B6C000DA7A520702D51F4A1B6A136070BD236ADB
:10B6D000002B2BD0D97A626DE1B172B6D97ACE0740
:10B6E00006D51948D9680668314099610160D97A50
:10B6F000880706D51548196906683140D961016087
:10B70000D97A4E0705D51248596906683140196241
:10B71000016062B61B68D968914207D00D48186075
:10B720000D49DA6042F0804018611960226C216D89
:10B73000136823EA01031360A3E700BF00E100E000
:10B7400004E100E008E100E080E100E084E100E0E5
:10B7500088E100E001403F0000003F802DE9F0411A
:10B76000044686B0806A9DF830801E460F46154616
:10B77000B4F90830002800F04281DA1D48BF03F117
:10B780000E02B4F90630D21003FB02F2002105F0DC
:10B79000BBFCB4F90820202A00F39280B4F906100B
:10B7A000A34B0120203A733902EBD27201EBD17125
:10B7B0004FF0200E029073208DE8014042F34F02BB
:10B7C00041F34F01204600F051FE606A84F82D706D
:10B7D000002800F04D81002D40F08A80B4F9083037
:10B7E000202B14BF3D253C2584F82C50B8F1000FC8
:10B7F00040F0858006B394F93300002818DBC0B20E
:10B80000012102F0E7F8012194F8330002F0CEF8AC
:10B81000012002F007F9002194F8330002F0C6F885
:10B820000A2002F0FFF8012194F8330002F0BEF87C
:10B83000606A002800F08280A16DFFF771F8042291
:10B840007C492046FFF792FE217A0139C9B2204691
:10B85000FFF7C4FD784904222046FFF787FE94F9DC
:10B860002D30012B14BF142110212046FFF7B6FD07
:10B87000042272492046FFF779FEB4F90630802B86
:10B8800000F09280602B00F0A680D9212046FFF7BF
:10B89000A5FD94F92D30012B14BFF1212221204662
:10B8A000FFF79CFD204606226549FFF75FFE606AB0
:10B8B00050B3E16DFFF734F8012006B0BDE8F08128
:10B8C000B4F906105F4B0120403A52394FF0400E58
:10B8D000029002EBD272522001EBD1718DE801404F
:10B8E00042F34F0241F34F01204600F0BFFD6CE7E9
:10B8F0006DB284F82C50B8F1000F3FF47BAFFEF727
:10B90000C5FF002E94D076E7216C226D0868236A6B
:10B9100002430A6073B1DA7A62B1D00703D54A4AAA
:10B9200099691160DA7A91077CD4520702D5474AA7
:10B930001B6A1360012006B0BDE8F081236A002B6A
:10B940002BD0D97A626DE1B172B6D97ACF0706D51C
:10B950003F48D9680568294099610160D97A8E0706
:10B9600006D53C48196905682940D9610160D97A32
:10B970004D0705D5384859690568294019620160A5
:10B9800062B61B68D968914207D0344818603449C0
:10B99000DA6042F0804018611960226C216D1368F2
:10B9A00023EA010313604AE7B4F90830202B00F0C2
:10B9B0008680402B7FF469AF2A4920460322FFF797
:10B9C000D5FD94F92D30012B14BFCF219F212046A6
:10B9D000FFF704FD59E7B4F90830102B7FF455AF99
:10B9E000214920460322FFF7C1FD94F92D30012B98
:10B9F00014BFAF2110212046FFF7F0FC45E7DA1D08
:10BA000048BF03F10E02B4F90630D21003FB02F274
:10BA10001046059205F04CF8A06200283FF44DAFA7
:10BA2000059AB3E6114AD9691160DA7A7DE700BF59
:10BA3000A437010084390100883901008C390100E4
:10BA4000903901009839010000E100E008E100E0D0
:10BA500080E100E084E100E088E100E001403F0097
:10BA600000003F80A0370100583C010004E100E0E5
:10BA7000012194F83100244F01F0ACFF94F832001A
:10BA8000012101F0A7FF94F9312094F9323057F8E1
:10BA90003220E26357F83330206A23640125E564DD
:10BAA00025651A682A431A6078B1B8F1000F3FF48F
:10BAB00028AFFFF75BFB002E3FF4BAAE9BE60422F3
:10BAC00012492046FFF752FDDFE6294694F82F0081
:10BAD00001F080FF294694F8300001F07BFF94F9D3
:10BAE0002F2094F9303057F83220626357F8333002
:10BAF0006564A5641A68A36322F001021A60002E2F
:10BB00003FF496AE77E600BFF44101009C37010098
:10BB1000B0F90820D31D48BF02F10E03B0F906208A
:10BB2000806ADB1002FB03F2002105F0EDBA00BFD2
:10BB3000F0B50029BDF814502EDBB0F90660B14213
:10BB40002ADA002A59DBB0F9087014461C44BC42BA
:10BB5000C4BFBB1A1BB2002B1EDDD2B2D408D0F872
:10BB600028E016FB041112F00702DBB20EEB010411
:10BB700021D0C2F10807FAB2374F9342BF5C0CD212
:10BB8000C3EB020CFF2646FA0CF6012D07EA060766
:10BB90003FD005D3022D36D0F0BD012D39D030D2A3
:10BBA0001EF8016026EA07070EF801709342F3D3EE
:10BBB000B0F906100C449A1AD2B2072A10D9022DF5
:10BBC00036D0002D14BFFF26002613462670083BF2
:10BBD000B0F90610DBB2072B0C44F7D802F00702CD
:10BBE000002AD9D01D4B012D9B5C1DD017D3022DEF
:10BBF000D2D1227853402370F0BD13441BB20022EF
:10BC0000A1E7022D25D11EF8016077400EF80170E2
:10BC1000CCE71EF8016037430EF80170C6E72278C2
:10BC200022EA03032370F0BD227813432370F0BD92
:10BC300011462378DB4323700839B0F90630C9B2C6
:10BC400007291C44F5D812F00702A5D0034B9B5CD2
:10BC5000CFE73444AFE700BF3C3701002C37010089
:10BC600070B4C47DBDF80C50022C18D0032C1FD02A
:10BC7000012C0BD0002A03DBB0F90840944201DC10
:10BC800070BC7047039570BCFFF7B0BAC4880395C9
:10BC9000013CA41A0A4621B270BCFFF749BF0689CD
:10BCA000C488013E641AB21AE41A12B221B2E1E762
:10BCB00004890395E41A641A114622B270BCFFF796
:10BCC00037BF00BF70B4C57DBDF80C60022D1AD01F
:10BCD000032D12D0012D03D0039670BCFFF728BFAF
:10BCE000C488E41AA41A0A4621B2002A03DBB0F978
:10BCF0000840944213DC70BC70470489013C641A0C
:10BD0000114622B2F1E7C48805890396013CAD1AB9
:10BD1000ED1A621A11B22AB270BCFFF709BF03967E
:10BD200070BCFFF763BA00BF2DE9F8430446406AD0
:10BD3000002863D0A16DFEF7F3FD0522744920466B
:10BD4000FFF714FCA1790139C9B22046FFF746FB81
:10BD5000B4F90820E588A66AD31D48BF02F10E0396
:10BD6000DB10626A15FB03F51FFA85F8002A7BD009
:10BD700094F82C300125AB4082F83B3082F85E50BD
:10BD800082F85D50606A036840211B6808F1FF3744
:10BD90009847BFB2B8F1000F23D03744A846013E00
:10BDA000606A16F8011F03681B6898470135B7429F
:10BDB000EDB216D0202DF3D10121606AFEF712FFFB
:10BDC00094F82C20636A520083F83B2083F85E804D
:10BDD00083F85D80606A036840211B6898470125ED
:10BDE000DEE70121606AFEF7FDFE606A002800F0D0
:10BDF0008D80E16DBDE8F843FEF792BD236A002B0C
:10BE00002BD0D97A626DE1B172B6D97ACE0706D558
:10BE10004048D9680568294099610160D97A8D0741
:10BE200006D53D48196905682940D9610160D97A6C
:10BE3000480705D5394859690568294019620160E4
:10BE400062B61B68D968914207D0354818603549F9
:10BE5000DA6042F0804018611960226C216D13682D
:10BE600023EA0103136068E7E26BE36C1168276A59
:10BE70000B4306EB080913604FF0004E4E450DD002
:10BE800016F801CB2FB33A68C2F82CE0C2F834C0E0
:10BE9000D36A002BFCDA4E45936BF1D1226C236DF3
:10BEA00011680B43136097B1FB7A83B1D90703D5AF
:10BEB0001D4BBA691A60FB7A9A0703D51B4BFA69C6
:10BEC0001A60FB7A5B0702D5194B3A6A1A60BDE823
:10BED000F883A36BD4F8348008208021D8F80020A0
:10BEE000656C1CEA010F14BF2A43AA43C8F800205E
:10BEF0001A68A56C2A431A601A68A56C013822EAF0
:10BF000005024FEA51011A60E8D1B7E7276AC5E791
:10BF10003437010080E100E084E100E088E100E0E6
:10BF200001403F0000003F8000E100E004E100E04C
:10BF300008E100E02DE9F04F85B09946BDF9387071
:10BF4000BDF83CA0BB1AC1EB090B002BB8BF5B428C
:10BF5000BBF1000FB8BFCBF1000B5B450D46164699
:10BF60000093804648DC4D453A4633464CDC194642
:10BF700013460A46C5EB09019B1A89B2002B0CB285
:10BF8000B8BF5B4204EBD474BE42ACBF4FF0FF328B
:10BF900001224D45039102924FEA640429DC9BB2D1
:10BFA00001930DE0D8F80070BF69B847019BE41A0F
:10BFB000A3B21CB20135002C2DB211DBA94518DB50
:10BFC000009B5B452A46534631464046EADCD8F89A
:10BFD000002053469769294632464046B847E5E770
:10BFE000029A1644039AA94502EB030436B224B21E
:10BFF000E6DA05B0BDE8F08F4A462B46B94635462D
:10C000004D4517461E46B2DD304629463E464D4652
:10C0100007468946AEE700BF10B404682469A44609
:10C0200010BC604730B40468BDF808500295A46B9A
:10C03000A44630BC604700BF30B40468BDF8085067
:10C040000295E46BA44630BC604700BF70B404683E
:10C05000BDF90C60BDF8105003960495246CA446FD
:10C0600070BC6047704700BF10B582B0B0F90C20BB
:10C0700001910168009200220C6CB0F90A3011465F
:10C08000A04702B010BD00BF704700BF01F0030120
:10C090000129C17506D0032904D0C28803894281D1
:10C0A000838170470289C38842818381704700BFC2
:10C0B0002DE9F0410568134E6F6986B0B74204461A
:10C0C000BDF8308010D1013B13441BB20093CDF872
:10C0D00004800B46AD6A2046A8472368DB6AB3425A
:10C0E0000AD106B0BDE8F081059304920391B847E8
:10C0F00003A925680EC9E6E7204606B0BDE8F04171
:10C10000184700BF65C000002DE9F0410568124ED8
:10C110006F6986B0B7420446BDF830800FD1013B4D
:10C12000CDF804800B4400921BB2AD6A2046A847AC
:10C130002368DB6AB3420AD106B0BDE8F0810593FB
:10C1400004920391B84703A925680EC9E7E7204682
:10C1500006B0BDE8F041184765C000002DE9F04F7A
:10C160000568DFF858B06F6985B05F450646BDF9D0
:10C170003890BDF83CA00C46904615D11F19BC4222
:10C180000CDACDF800A0214601342D6A4B46424618
:10C19000304624B2A847BC423568F2DBEB6A5B4507
:10C1A00007D105B0BDE8F08F0393B8473568039B0E
:10C1B000E4E7304605B0BDE8F04F184765C0000021
:10C1C0002DE9F04387B099420546BDF93840BDF8E6
:10C1D0003C6025D0A24212D00768DFF88080D7F8F3
:10C1E0001490C14532D18DE850002846BC6AA04762
:10C1F0002B68DB6A434524D107B0BDE8F083994240
:10C2000002DD08461946034628680E96C46B0133C2
:10C210005B1A1BB22846A44607B0BDE8F04360474E
:10C22000A24202DD134622461C4628680E96631C75
:10C23000846B9B1A1BB22846A44607B0BDE8F043A6
:10C240006047284607B0BDE8F043184705930492BD
:10C250000391C84703A92F680EC9C4E765C0000051
:10C260002DE9F04FD0F800E0DFF89090DEF814B040
:10C2700083B0CB450446BDF93080BDF834A00D46EF
:10C2800017461E4631D1CDF800A0DEF824B029466D
:10C2900033463A462046D8472368CDF800A008F137
:10C2A000FF323A44D3F824B0294612B2334620462E
:10C2B000D8472368CDF800A02946D3F820B03A46E5
:10C2C00043462046D8472068CDF800A0711E294477
:10C2D0004346056A09B23A462046A8472368DB6A06
:10C2E0004B4506D103B0BDE8F08FD847D4F800E045
:10C2F000C9E7204603B0BDE8F04F184765C000000D
:10C30000F0B4002401264FF6FF75094F0760047151
:10C31000C475C48104824476C461867506768582BC
:10C320004582C180028141818281F0BC704700BF9B
:10C33000643C01002DE9F04F85B00668BDF844501B
:10C34000BDF93880CDF8008004460195D6F848B094
:10C350000392BDF93C60BDF9407089469A46D847C2
:10C3600023680195009742465146D3F848802046FD
:10C370003346C0472068039B0E930F95856C4B4650
:10C380003A4631462046AC4605B0BDE8F04F60471E
:10C390002DE9F04F87B01746BDF940400091254682
:10C3A000E91D059344BF2B4603F10E010268BDF859
:10C3B000486053690294C91003912B49BDF9444068
:10C3C00001968B42824645D1002C3CDD029B3C44C9
:10C3D0005E1EB6B24FF0000923B2049301364D46FB
:10C3E000029B002B28DD059B002403EB090806E0D7
:10C3F000EDB22B0604F1010411D4A6421CD0A1B267
:10C4000011F0070F23B24FEA4505F1D1002BB8BF59
:10C410000733DB10013418F803502B06EDD5009BD1
:10C42000D2F818B019443A4609B2019B5046D84791
:10C43000A642DAF80020E2D1039B01379944049B1D
:10C440003FB2BB42CCD1D36A074A934206D107B070
:10C45000BDE8F08F9847DAF80020B5E7504607B0FE
:10C46000BDE8F04F184700BF65C0000070B4BDF9CB
:10C470000C60BDF91050BDF8144003960495059466
:10C4800070BCFFF785BF00BF2DE9F04F93B0904619
:10C490000591C1691090BDF870000790BDF87490C7
:10C4A0009DF878A00493002900F0CD800A7A0AC98B
:10C4B000894604998A1AD2B203EBC203BAF1010F7A
:10C4C000DA780B9293F905201E8893F802B00F9248
:10C4D00093F9064079D913B2099323B20C93109BB8
:10C4E0001A68A94B1193194653698B4240F0A680F4
:10C4F0000B9B002B55D01FFA88F300210D93C846E3
:10C500002344DDF8409006910E930F460C46BBF194
:10C51000000F3FD0BDF818100C9B03971FFA8AF04C
:10C52000CB1813FB00F304900E9801440D980344BC
:10C5300009B21BB20A910893002505E00135EBB260
:10C5400064009B45E4B222D9039B2B44590703D1D5
:10C55000731C18F806409EB22306EFD5099BBDF860
:10C560001000E91811FB00F10598BAF1010F0FFA5C
:10C570008AF301441CD0079801900093D26909B254
:10C5800017464846089AB847D9F80020D6E7039FCF
:10C590005F44FFB2069B0B9901330693DBB29942CD
:10C5A000B5D8D36A119A934243D113B0BDE8F08F46
:10C5B0000F9B191893690A9A29441F4609B2079BD1
:10C5C0004846B847D9F80020B8E700230C930993F0
:10C5D00085E70A9A0D9B0132013B52B213F0FF032B
:10C5E0000A920D936FD1DDF81890079BDDF83C801F
:10C5F000DDF820A04B4517D0BAF1010F00F0C8803C
:10C600000B9A109DCDF804900BEB8B014FEACB03F6
:10C610000A4400931146DEF81C405346424609B2D4
:10C620002846A047D5F800E0DEF82C30119A934256
:10C63000BBD0109813B0BDE8F04F1847109D2846A6
:10C6400098472A6854E7109A0598B2F90A3083424D
:10C65000ABDDB2F90C304345A7DD062313FB0A031B
:10C66000002BA2DD08EBCA03002B9EDD537E2BB905
:10C67000049BAF2B02D90133DBB20493109BD3F898
:10C6800000E0414B11931A46DEF81430934240F01B
:10C690008E801FFA88F30E9308339BB2BDF81420E6
:10C6A000059305230D9300230A93CDF83C800FFAE0
:10C6B0008AF3DDF84080CDF818900B921FFA8AFBC0
:10C6C000CDF820A099460A9ABDF810000B9C0E9D4B
:10C6D0000523194611FB00232C481146C75C03971C
:10C6E00002FB0B4214FA81F312B21BB209920C93B3
:10C6F0002C462E461CE0089B0999012B2AB24B467A
:10C7000040462DD0079F0197CDF80090DEF81CA081
:10C71000D047D8F800E0039B5B0801340393059BE6
:10C72000A4B25D445E44A342ADB2B6B23FF451AF91
:10C73000039BD807DFD4079B069A9342EBD0089B54
:10C74000012B16D0069B0193CDF80090DEF81CA0BB
:10C7500009994B4632B24046D047D8F800E0DAE7B4
:10C76000DEF818A0079B0C9922B2D047D8F800E059
:10C77000D1E7DEF818A00C991346404622B2D04704
:10C78000D8F800E0C7E700BF65C00000B43C010076
:10C790000B99109DCDF800900531DEF8204009B2CC
:10C7A000424608232846A047D5F800E03CE7109C05
:10C7B00020469847D4F800E06BE700BFF0B5C369A6
:10C7C00085B004462BB30A2968D00D294AD01A7ABD
:10C7D000914247D3587A884244D35D688A1A05EB60
:10C7E000C205AA78002A50D0E87800284DD0207ED3
:10C7F00000283AD095F905E0B4F90E00A67DB4F909
:10C800000A70724406FB0202BA4262DCB4F91020DC
:10C8100030E00A2956D00D2924D0027E002A4BD0C0
:10C82000B0F90E00A57DB4F90A60062212FB0502DC
:10C83000B2423EDD228AE38102EBC50212B2184603
:10C840002282A78A668A02950B468DE8C0000146BF
:10C850002046FFF719FEA37DE28903EB430302EBB9
:10C860004303E381012005B0F0BDA67DB4F90E00BD
:10C87000B4F91020B4F814E0678A02960B468DE8EC
:10C88000804001462046FFF7FFFD2979E389A27D1C
:10C89000012001FB0233E38105B0F0BD0022C2811B
:10C8A0009A7A817D038A01FB02330382012005B05D
:10C8B000F0BDB4F91020C4E7857DB4F91020B0F9BB
:10C8C0000E00BEE7028A817DC38102EBC1030382B1
:10C8D000C8E70020E0819B7A228A03FB062212B27D
:10C8E0002282C7E7C1810282704700BF002908BFCA
:10C8F00001218175704700BF81824182704700BF6E
:10C90000C07D7047B0F90A00704700BFB0F90C0055
:10C91000704700BF10B4EFF3108272B6437F33B993
:10C92000017F012907D003290FD00123437702B9E2
:10C9300062B610BC7047124C2168A1B11149436125
:10C940000B68836108605861EFE70F4C216881B183
:10C950000E4943610B688361086058610C4B4FF0CE
:10C9600080511960E1E7074B4161816120601860E7
:10C97000DBE7064B4161816120601860EEE700BF94
:10C98000809FFF1F7C9FFF1F709FFF1F749FFF1FD3
:10C9900004ED00E070B5EFF3108272B60C4C206825
:10C9A00080B10C4E00254369236073B19D6102B9CB
:10C9B00062B6457783689847EFF3108272B62068B5
:10C9C0000028F0D102B962B670BD3360EFE700BF56
:10C9D000709FFF1F749FFF1FFFF7DCBF184A30B422
:10C9E0001468002C27D0036821688B420ED2CB1A22
:10C9F00000218460C1602360E06010600223037541
:10CA000030BC704711688B42144608D3A2685B1A89
:10CA10000360002AF6D18260C460A060EEE7D268AD
:10CA2000C2608460E060C568CB1A0222A8602360FF
:10CA3000027530BC70478460C4601060DEE700BFE0
:10CA4000789FFF1FF8B5224E34682CB32368002B63
:10CA50003AD1204F1D4604E03468ECB12368002B26
:10CA600032D1A36803B1DD602069336003682575A6
:10CA70001B68BB4221D1037F4560022BC46020D0DC
:10CA8000FFF748FF6368002BE6D023602046FFF7DE
:10CA9000A5FF3468002CE1D1EFF3108372B60E4A83
:10CAA00000211068116003B962B628B18468FFF7ED
:10CAB00095FF20460028F9D1F8BD2246002198476D
:10CAC000E0E783689847DDE7013B2360E4E700BFC8
:10CAD000789FFF1F55B10000889FFF1F024A13680F
:10CAE00001331360FFF7AEBF949FFF1F704700BF75
:10CAF0000368F0B4FBB1002501249D60DC601B4C91
:10CB00001A601C44241104F144056A1103269200A2
:10CB10009E60174F0679174B47F8241002F16042C8
:10CB200002F5614205F01F05012000FA05F5E65403
:10CB30001560F0BC7047104C236843F40003236079
:10CB400000BF0E4B0E4DA4F58734A4F59E7401264C
:10CB50001E60234604609C68002CD0D01033AB428A
:10CB60000360F8D1002303601846E2E7008FFCBFA2
:10CB7000B891FF1F44E400E03C8004400070034093
:10CB8000407103400168A9B10B4BF0B40B441B1179
:10CB90000A4E0B4F0B4D46F8237003F1440202F08E
:10CBA0001F0401235211A340002445F822308C6059
:10CBB0000460F0BC704700BF008FFCBFB891FF1F3E
:10CBC000EDCA000080E100E0024A034B0121116040
:10CBD0001B6818470C710340B891FF1F024A034BB2
:10CBE000012111605B6818471C710340B891FF1F59
:10CBF000024A034B012111609B6818472C710340C6
:10CC0000B891FF1F024A034B01211160DB681847EE
:10CC10003C710340B891FF1FF8B50E4671B17AB16F
:10CC20000746144600253B6816F8011B1B6838466A
:10CC30009847013C0544F6D12846F8BD0846F8BDA2
:10CC40001046F8BD00B5064A036812885B6883B0D9
:10CC500001A9ADF804200222984703B05DF804FB57
:10CC6000B4410100F0B507468BB0002A33D0012A49
:10CC700008BF0A2251B3212400E0F4B2B1FBF2F55F
:10CC800002FB1511C8B2092900F1300198BFC8B2E2
:10CC90000AA988BF3730214488BFC0B201F8240CEC
:10CCA000661E2946002DE8D133B1013CE4B20AAB3F
:10CCB00023442D2203F8242C3B6801AA11195B6838
:10CCC0003846C4F1220298470BB0F0BD30228DF8EF
:10CCD00025202124E8E70368C9B21B6898470BB0F8
:10CCE000F0BD00BF0029BABF49422D2300230A220C
:10CCF000FFF7B8BF374A384913681B06FCD40B68E6
:10CD000013F08003F8D172B634490A78002A5FD054
:10CD1000334A3448F0B4344C176806682568D46840
:10CD20000C303E44143200681268304F35442C44B5
:10CD300020440244C2F34E022D4E2E482E4D2F4C5D
:10CD400042F400423A60376806682D682C4A24682D
:10CD50000C303E44006812682A4F35442C4420446D
:10CD60000244C2F34E02284E2848294D294C42F471
:10CD700000423A60376806682D68274A24680C30FC
:10CD80003E4400681268254F35442C442044024438
:10CD9000C2F34E02224E2348234D244C42F400425B
:10CDA0003A60376806682D68214A24680C303E4492
:10CDB0000068126835442C4420440244C2F34E02F9
:10CDC0001C4842F4004202600B7062B6F0BC70472F
:10CDD00062B6704724B0034024B00B408D9FFF1F04
:10CDE00038B003403CB0034040B003402CB0034097
:10CDF00058B003405CB0034060B0034064B00340EF
:10CE00006CB0034030B0034038B00B403CB00B4036
:10CE100040B00B4044B00B404CB00B402CB00B402A
:10CE200058B00B405CB00B4060B00B4064B00B409E
:10CE30006CB00B4030B00B4030B42948294A2A4B23
:10CE40002A4D6024E121047011701B78284C082BB6
:10CE500030D00A2B2748284937D00C2B0CBF35225D
:10CE60003D2212232A60236002600B60234B244979
:10CE70001B78244ABBB101230B601360224B23496A
:10CE80001B78234A012B26D9042B0FD9082B1ED936
:10CE9000102B94BF862387230B6013601D4B012248
:10CEA0001A7030BC70470B601360E7E784230B6097
:10CEB0001360F3E700F58E200F4908300122132399
:10CEC0002A60236002600B60D0E73922F7E78523F0
:10CED0000B601360E2E780230B601360DEE700BFA6
:10CEE0000040074001400740C891FF1F08B00340C1
:10CEF0000CB0034008B00B400CB00B40909FFF1FDC
:10CF000020B0034020B00B40C991FF1F24B0034064
:10CF100024B00B408D9FFF1F0C2830B417D910236D
:10CF2000984228BF18461C46104A114D1178181A0D
:10CF30008C42287018D00F4913700B7823B10E491A
:10CF40000E4A00230B60136030BCFFF775BF0A2840
:10CF500002D90C231C46E7E7082802D90A231C46FD
:10CF6000E2E708231C46DFE730BC7047C891FF1F8B
:10CF70008C9FFF1F8D9FFF1F24B0034024B00B40E8
:10CF800028282FD8334B2DE9F0411E5CFF2E2BD0E3
:10CF9000314B1B78002B2AD132062CD472B62F4D80
:10CFA0002F4C2F46012326602B7062B672B6236881
:10CFB0001B060CD43B781BB9F4E72B78002BF1D07F
:10CFC00062B602F09BF972B623681806F5D5254BB8
:10CFD0001B6800222A7062B6234A107843FA00F0D8
:10CFE000BDE8F081002070470020BDE8F081FFF728
:10CFF00081FE3206D2D572B61C4DDFF87C801C4C07
:10D0000006F04007FFB206F03F06D8F80030DFB167
:10D0100023F01003C8F8003001232660134A2B7058
:10D0200062B672B6236819060CD413781BB9ECE704
:10D030002B78002BE9D062B602F060F972B6236853
:10D040001B06F5D50B4BC3E743F01003C8F80030BF
:10D05000E2E700BFB84101008D9FFF1F8F9FFF1FB8
:10D0600000B0034010B003408C9FFF1F8E9FFF1F36
:10D0700000B00B4010B00B400CB00B400A4A0B49FB
:10D08000136843F4805313600B7843B9084BC022F4
:10D090001A70084B80F30C0000B218807047044BE4
:10D0A00080221A70F5E700BF2C800440909FFF1F7C
:10D0B00021C00C4000C00C40F0B51B4B1B4E596802
:10D0C00018689A68DB6885B06C460FC43378990796
:10D0D0001DD5174A174C1378174913F0700318BF62
:10D0E0001370164A164B8027177000263320032230
:10D0F00026706D4608701A7072B6043C45F0010542
:10D100002046A84762B6237813F0700309D10D4B6F
:10D11000064901E0013B02D00A78D207FAD505B0F2
:10D12000F0BD237005B0F0BDE441010001000240F4
:10D1300000000240040002400B00024007000240D1
:10D140000A000240410D0300B0F5006F0AD210B58D
:10D15000094B1B78DB07044606D504F1A050007884
:10D16000C0B210BD00207047FFF7A6FF04F1A05029
:10D170000078C0B210BD00BF01000240B0F5006FE2
:10D1800017D238B50F4B1B78DA070D46044611D578
:10D1900004F1A0500378AB420AD00B4A137813F085
:10D1A000700318BF1370074A05701378DB07FCD5AE
:10D1B00038BD7047FFF780FF04F1A0500378AB4201
:10D1C000EBD1F5E7010002400000024008B5F4F79A
:10D1D00037FDF5F72FF902F091F8FAE7844641EAB6
:10D1E000000313F003036DD1403A41D351F8043BDF
:10D1F00040F8043B51F8043B40F8043B51F8043B31
:10D2000040F8043B51F8043B40F8043B51F8043B20
:10D2100040F8043B51F8043B40F8043B51F8043B10
:10D2200040F8043B51F8043B40F8043B51F8043B00
:10D2300040F8043B51F8043B40F8043B51F8043BF0
:10D2400040F8043B51F8043B40F8043B51F8043BE0
:10D2500040F8043B51F8043B40F8043B51F8043BD0
:10D2600040F8043B51F8043B40F8043B403ABDD23F
:10D27000303211D351F8043B40F8043B51F8043BE1
:10D2800040F8043B51F8043B40F8043B51F8043BA0
:10D2900040F8043B103AEDD20C3205D351F8043B70
:10D2A00040F8043B043AF9D2043208D0D2071CBF3C
:10D2B00011F8013B00F8013B01D30B880380604665
:10D2C000704700BF082A13D38B078DD010F00303DB
:10D2D0008AD0C3F10403D21ADB071CBF11F8013B4B
:10D2E00000F8013B80D331F8023B20F8023B7BE79A
:10D2F000043AD9D3013A11F8013B00F8013BF9D2C5
:10D300000B7803704B7843708B788370604670475E
:10D3100008B5104C08E0236859050DD423681A0598
:10D320000FD42368DB0411D423685803F3D500F02D
:10D330008DFE23685905F1D502F044F823681A05DB
:10D34000EFD502F0D5F82368DB04EDD500F0F0FC52
:10D35000EAE700BF3480044008B5FFF7D9FF00BFFB
:10D36000014B10221A80704700200540704700BF13
:10D37000094908B50B6830B16A461844A2F58052D5
:10D38000904202D20860184608BD03F063FB0C23EC
:10D3900003604FF0FF3008BDCC91FF1FFEE700BFD8
:10D3A000EFF3138070B9EFF310836BB9EFF30582DD
:10D3B0005AB94FF48070EFF311832BB1984228BF14
:10D3C000184670474FF0FF3070470F2A01D81846B3
:10D3D000F1E7014BD05CEEE7F0E300E0F0B44D1E66
:10D3E0002E46002400E00134B0FBF2F302FB1300F0
:10D3F000092800F130078ABF3730F8B2C0B206F80A
:10D40000010F1846002BEED10A1953704CB1107859
:10D4100015F8016F28700133E01A834202F80169A0
:10D42000F5DB0846F0BC7047704700BF10B40F4BE7
:10D4300053F8302092F880422CB1012369B182F870
:10D44000803010BC704703EBC0035B681A6841B9B9
:10D4500022F002021A6010BC704782F8003110BC42
:10D46000704742F003021A6010BC7047F44101009B
:10D470001C4A02EBC00301295B6811D004291BD0B0
:10D4800052F83000002280F8802229B1022920D0F1
:10D49000032922D01A6070474FF480721A607047D7
:10D4A00052F830004FF4A27280F880121A601A68A5
:10D4B00022F020021A60704752F830104FF4A27226
:10D4C000012081F880021A601A6842F020021A6076
:10D4D000704740F203121A6070474FF481721A606D
:10D4E000704700BFF4410100212848D8F8B5042A4C
:10D4F00044D8DFE802F0484B4E0345004FF41026B5
:10D500002B4B03EBC0030D465C68216811F4E0610E
:10D5100048D0284B284A2949C3F89C2104F14042AD
:10D520002748C3F8A411A2F59221264FC3F8A00101
:10D530007C292548C3F8A871C3F8AC012CD9A2F501
:10D5400094237C2B2AD9A2F596237C2B28D9A2F5EB
:10D5500098237C2B29D9A2F59A227C2A27D81B480C
:10D5600072B6236823F4702343F08072C4F38401FD
:10D570001643236040F82150266062B6F8BD70471C
:10D580004FF43026BCE74FF40026B9E74FF44026AD
:10D59000B6E74FF42026B3E70D48E1E70D48DFE793
:10D5A0000D48DDE7FFF764FFB3E70C48D8E7F8BDA7
:10D5B000F44101000082FF1FF188FF1F9988FF1FBF
:10D5C000C588FF1F6D88FF1F4188FF1FA892FF1F9E
:10D5D000D091FF1F0892FF1F5892FF1F8892FF1FD4
:10D5E0001A4B03EBC00010B4426802F14043A3F5AC
:10D5F00092217C2923D9A3F594217C290DD9A3F567
:10D6000096217C291FD9A3F598217C2919D9A3F546
:10D610009A237C2B11D80E4C00E00E4C72B6136886
:10D620000D4823F08773C2F3840123F4803343F061
:10D630008073136044F8210062B610BC7047074C39
:10D64000ECE7074CEAE7074CE8E700BFF4410100CC
:10D65000A892FF1F0892FF1F29D40000D091FF1F3E
:10D660008892FF1F5892FF1F30B4054B054D064CA2
:10D67000002210211A602A602060196030BC7047B7
:10D6800014D0034004D0034000D00340282838B50C
:10D690002ED0002904464FDD5F4B1B78012505FA8B
:10D6A00003F28A4202D8212837D938BD0338C2B2E2
:10D6B000012A3AD9202C4AD0192C48D0574A12684E
:10D6C00002FB011222FA03F31D2800F29B80DFE81F
:10D6D00000F0928B847D9999766F9999999999998F
:10D6E00099999968615A53994C9999999999994539
:10D6F000494B1B780B2B08D90C2B1CBF0C3B194139
:10D700000846BDE83840FFF7B9BCC3F10C039940A7
:10D710000846BDE83840FFF7B1BC2946FFF786FE52
:10D720002946BDE83840FFF7A3BE3D4A126802FB18
:10D73000011222FA03F3C7E72128B6D80021FFF728
:10D7400075FE20460121BDE83840FFF791BE354AFD
:10D75000126802FB011222FA03F3B5E73249334A99
:10D760000B604FF45173136038BD3149314A0B607F
:10D770004FF45173136038BD2F49304A0B6040F2AB
:10D780004443136038BD2E492E4A0B6040F2444397
:10D79000136038BD2C492D4A0B6040F2444313609E
:10D7A00038BD2B492B4A0B6040F24443136038BD0F
:10D7B00029492A4A0B6040F24443136038BD284986
:10D7C000284A0B6040F24443136038BD2649274A7B
:10D7D0000B6040F24443136038BD2549254A0B6075
:10D7E00040F24443136038BD2349244A0B604FF490
:10D7F0005173136038BD2249224A0B604FF45173B4
:10D80000136038BD212C3FF650AF7F29D4BF0021D3
:10D810000121204693E700BFB092FF1F088003401C
:10D820000890034008800B4010800B4048A0044043
:10D8300018800B404CA004401880034008B00440FE
:10D840001080034004B004404080034018C00440EE
:10D850003880034014C004402880034010B00440C6
:10D86000208003400CB004403080034010C00440CE
:10D87000488003401CC0044018900340349004408A
:10D88000109003403090044038B1102828BF102079
:10D89000044AC3B2107813707047024A012310780B
:10D8A00013707047B092FF1F2DE9F8430E46804673
:10D8B0003249334D304603F053F847F6122300281F
:10D8C0001ABF1D464FF002094FF00109002425FA46
:10D8D00004F002F04FFE4FF05E51074602F0A2FE48
:10D8E0000146304603F050F830B90134072CEED130
:10D8F000E80902F03FFE07463146384602F046FF8F
:10D900004FF07C5102F084FD03F078F84FF6FF727F
:10D910009042A8F1030328BF1046012B29D9B8F182
:10D92000170F17D8174B23FA08F303F0010383F0FE
:10D93000010223B9B8F1190F0FD0BDE8F883124BDB
:10D94000124D13491A6044EAC9042A6008601C6039
:10D95000BDE8F883B8F1200FECD10E4B0E4D0F4906
:10D96000002244EAC9041A602A6008601C60BDE80D
:10D97000F8830B4B0B4D0C49F2E700BF001BB7407F
:10D98000006CDC026006F00000800340048003406D
:10D990000880034000800B4004800B4008800B404F
:10D9A000009003400490034008900340212801D8D0
:10D9B000FFF73CBD704700BF212806D8044B53F841
:10D9C000303093F80002C0B270470020704700BFAB
:10D9D000F4410100212801D8FFF74ABD704700BF7C
:10D9E00072B60C490C4B0D4A1B680868126862B687
:10D9F000520102D5322B88BF01300949C3F5BB3330
:10DA00004FF47A72FF33A1FB031302FB00F000EB2B
:10DA100093107047949FFF1F18E000E004ED00E0B2
:10DA2000ABAAAAAA2DE9F843054672B6204F214BAE
:10DA3000214A1B683C68126862B6520102D5322B3B
:10DA400088BF013495B3C3F5BB331C4EDFF8649037
:10DA5000DFF86480FF334FF47A72A6FB031302FBF6
:10DA600004F404EB931472B6D9F800103A68D8F8AD
:10DA700000E062B6C1F5BB33FF33A6FB03031EF023
:10DA8000806FC4EB93134FF47A7002D0322988BFB1
:10DA9000013200FB0233B3F57A7F04D3013D05D098
:10DAA00004F57A74DFE701F029FCDCE7BDE8F883D0
:10DAB000949FFF1F18E000E004ED00E0ABAAAAAAC3
:10DAC000F8B52D4B2D49DFF8D0E0DFF8D0C02C4E53
:10DAD0002C4D2D4C2D4A2E4F4FF4000018604FF066
:10DAE000807018604FF0007018604FF08060186010
:10DAF0004FF0006018600020086028234BF6FF718B
:10DB0000CCF80010CEF80030336013602B60236037
:10DB10003B60B3629362092245F8242CC4F8D80F05
:10DB200005F57F65C7F8D41F07F5FF2707F5FA67E6
:10DB3000C6F8F83F2B6006F5FF26C4F8D42F05F58C
:10DB4000FD2504F5FF24386006F2F47611483160B3
:10DB500005F5FF6504F5FD642B6023600260FFF7A7
:10DB60006BF91920FFF75EFF00F0B6FF40F21310CB
:10DB7000BDE8F840FFF756BF08E100E0048003402D
:10DB800014800340248003402C8003401C80034009
:10DB90003480034000800B400C8003400880034029
:10DBA0002DE9F84F214B1B6807460BB101221A7073
:10DBB000DFF888901E4D99F80040DFF884801D4EF4
:10DBC0000134272C8ABF4FF0000A5FFA84FA5446CA
:10DBD000AB462B78A34216D1FFF7E2FB40281FDCAF
:10DBE00033791B06F5D59BF800300133272B86BF10
:10DBF00000221346DAB218F80330DBB2F3712A7050
:10DC00002B78A342E8D00C490A4BFFB208F8047005
:10DC10000120AC22087089F800A0DA70BDE8F88F06
:10DC2000FF28D6DD01F06AFBD3E700BF0CA0FF1F81
:10DC300009A0FF1F00C0064008A0FF1F10A0FF1F83
:10DC4000A09FFF1F1C4BDFF894C01A681B49F0B55A
:10DC500042F480521A4D1A60DFF884E0194F1A4ED0
:10DC60001A4C00238CF800304FF451722B701F288F
:10DC700040F213358EF800303B70337025600A6037
:10DC800012D819460124124A124D117012485470CC
:10DC900000212C27402693724FF4003491701174A8
:10DCA000D7702E700460F0BDC0F34431C0F3471448
:10DCB00000F01F03E7E700BF348004400CC00440BD
:10DCC0009D9FFF1F09A0FF1F08A0FF1F08C0044061
:10DCD00000C0064031E400E004E100E09C9FFF1F2B
:10DCE00010A0FF1F034B1B68DB0401D5FFF758BFD3
:10DCF000704700BF3480044010B5044C237823B132
:10DD000001F0FCFA2378002BFAD110BD08A0FF1F08
:10DD1000054A064B10781B78C0B2DBB2984238BF78
:10DD20004030C01A704700BF9C9FFF1F9D9FFF1F80
:10DD300030B42B4B1A7994061FD52A48DA79037828
:10DD4000294901333F2B0978C8BF00238B42D2B247
:10DD500003D0264CD9B2E2540170254A116861B152
:10DD6000244A1278D2B2934236BFC2F140029B1AC3
:10DD70009B18272BC4BF01230B70194AD378DBB241
:10DD8000180611D45A060DD5154B1B795B0609D51B
:10DD9000194B1A491B6800220A7003B11A70104B04
:10DDA0002C22DA7030BC704711790906EAD5144983
:10DDB00010480C780178C9B28C420DD04A1C272A31
:10DDC00084BF00210A460F4D054C98BFD1B2AA5C12
:10DDD000D2B2E2710170D5E76C21D170D2E700BFF9
:10DDE00000C006409C9FFF1F9D9FFF1FC89FFF1FF5
:10DDF000989FFF1F09A0FF1F0CA0FF1F08A0FF1F77
:10DE000010A0FF1FA09FFF1F21282FD8184B195CBF
:10DE1000FF292BD0174B184ADFF870C003EBC00066
:10DE2000F0B54368DFF868E0144F154D154E002437
:10DE30001C60DEF80030012043F020038840CEF85B
:10DE4000003014604FF4A07338602E60C2F800C038
:10DE5000013BFDD113689B05FCD42023013BFDD180
:10DE6000094B09B233F8110080B2F0BD00207047B1
:10DE700004430100F44101000050044008500440F4
:10DE800004500440000002030051044080014A0095
:10DE900038800440431E032B14D872B60A4951F847
:10DEA000230068B170B4094C058834F81320466823
:10DEB00041F82360521B24F8132062B670BC7047EF
:10DEC00062B67047002070476CA0FF1FB0A2FF1F12
:10DED000013803280BD872B6074B53F8203043B1F2
:10DEE00000205B680130002BFBD162B67047002038
:10DEF00070471846F9E700BFC0A0FF1F30B472B6E4
:10DF00002B4A13781D0706D52A4B196A002936D0EB
:10DF1000996A002941D053781C0706D5254B196C06
:10DF200000293ED0996C002939D09378190705D57E
:10DF3000204B196E002936D0996E89B1D3781B0712
:10DF400007D51C4BD3F880207AB3D3F88820112151
:10DF50003AB162B6184B00221A7030BC00F04ABECB
:10DF60000D21154C154D227843F8315003EBC103B8
:10DF70000830013A5860227062B630BC7047042203
:10DF80000D4C0F4D217843F8325003EBC20308309B
:10DF90004A1E5860227062B6EFE70521E1E70921C9
:10DFA000DFE70822ECE70C22EAE71022E8E700BFEF
:10DFB000284301000080FF1FE9A0FF1FC8004000A8
:10DFC00088004000431E032B1DD81B4A400140F02F
:10DFD000100030B4104472B6184CE25C032A1BD80F
:10DFE000DFE802F00212151703220D88E25410F048
:10DFF000080F14BFC823882343EA05430831036090
:10E00000416062B630BC704708300222EDE705225D
:10E01000EBE708300422E8E7094A52F8230038B158
:10E02000084A52F82300416042F8231062B6E9E73B
:10E0300042F82310034AF7E70080FF1FF8A0FF1FF4
:10E04000C0A0FF1FD0A0FF1F00BE70472DE9F04FFA
:10E05000DFF818B3DFF818A387B044E0AD4F4FEAFC
:10E06000930807EBC809013ED9F8042003F0080320
:10E07000F6B2A2F1080003F0FF04002B40F001818A
:10E0800057F838301B0C99B222F8081C002B00F00E
:10E09000EF80A14B22F8064C42F8044C53F826209E
:10E0A000002A00F0CF819D4D55F8263058609C4CD9
:10E0B00045F8260034F81630194424F8161000F0FC
:10E0C00079FD002800F0C281964A974B19F0080F9D
:10E0D00000F1080018BF1346C9F8040047F83830AB
:10E0E00008238BF800309BF80040E4B265071CD58C
:10E0F0008E4B1B78B3B18E490A7802F0FF0322B130
:10E10000013BDBB20B7003B900BE8A490A7802F00A
:10E11000FF032AB1013BDBB20B70002B00F06881DA
:10E1200000F066FE04238BF8003004F0080303F0CF
:10E13000FF02002B00F0C9809AF80030DBB21E0904
:10E140008CD19A08DFF8CC9159F8321009EBC20053
:10E15000C1F38301013940680C2900F28580DFE8B2
:10E1600001F07A7A838383838383468383830700E2
:10E170000168714D4068714F714E6860296088B2C6
:10E1800040F281610024674B49F832304FF0010EB4
:10E1900088423C60C9F81040C9F8184086F800E091
:10E1A0005C4A00F2E780B0F5D06F80F01B82B0F5DA
:10E1B000817F00F0D98100F26981802800F02A82F5
:10E1C000822840F0D781A98801F07F01042900F25C
:10E1D000D1815C485C4A890008441470547001780D
:10E1E0008C0740F1608382F800E0022173E1534F15
:10E1F0003A682AB3554B524E5548198834780578F9
:10E2000040298E4645F0020828BF4FF0400E002CF2
:10E2100084F001043470CEEB01010CBF8824C824C3
:10E2200009EBC80689B285F0010544EA0E44726024
:10E23000198049F8384072440570002965D03A6069
:10E240003D4B1A88B2F5A06F0ED100219A78597013
:10E25000404B1A7008E038493F4C0D68A54200F069
:10E260009880304949F832103C4A0123137037E74F
:10E270002C4A2D4B19F0080F18BF134647F83830B9
:10E280002EE700F0B7FC364A364952F82630002B0C
:10E2900000F0E38058688C5D42F8260003F1080224
:10E2A000C9F80420032C05D8DFE804F02C02292645
:10E2B00002228A551A8819F0080F0CBF8823C82338
:10E2C00043EA024347F838300AE7E00700F1938059
:10E2D000210600F1D180A20706D5234A23491378ED
:10E2E0000220DBB213700870E30602D51F4B102228
:10E2F0001A7007B0BDE8F08F04228A55DAE70522CC
:10E300008A55D7E703228A55D4E7BEF1400F18BFDC
:10E31000002294E70080FF1F6CA0FF1F18A0FF1FC2
:10E32000B0A2FF1FC800400088004000F4A0FF1FFB
:10E330007DA0FF1F68A1FF1FE0A0FF1F14A0FF1F0B
:10E340007CA0FF1FC0200740ECA0FF1F28A0FF1FDC
:10E35000E8A0FF1F982007402109000394200740F0
:10E36000C0A0FF1FF8A0FF1F8820074080200740A3
:10E3700090200740B0F5106F00F07C8140F2A38040
:10E3800040F62112904240F07B82A54A012313708F
:10E390006AE74C68A3498C427FF463AF0178A929EE
:10E3A0007FF45FAF417845297FF45BAF8178C22964
:10E3B0007FF457AFC1786B297FF453AF9A489B4ED7
:10E3C0000178347881F00105002C41F002010570DC
:10E3D0000CBF8820C82084F0010449F8310009EB03
:10E3E000C10193483470002505244D60047038E75E
:10E3F00000F064FF94E68F4B89488B491A614FF017
:10E40000020E80F800E08C4F0A708C491960996008
:10E410008B4E8C4D8C4C9A610D213970FF213170DF
:10E42000DFF84CE229702270884D894A8EF800107E
:10E430009F27012406F8047C5D600470DA6007B051
:10E44000BDE8F08F43F82600824D30E6824A47F857
:10E45000380013780133137042E68B5D032B00F212
:10E46000BA8001A252F823F0E1E00000E1E00000F0
:10E47000C1E40000BBE400006F49724B80220D2014
:10E4800008701A70A2077FF52FAF26E740F202321C
:10E49000904240F0ED81AA8802F07F02042A69D8F8
:10E4A0006D88002D66D16449CDF804E092001144D6
:10E4B0000A7842F002020A70C1E101238B550FE68F
:10E4C00000238B550CE6B0F5086F53D16349644ABD
:10E4D000097811707146ED888D4280F0E8825248CB
:10E4E0000478402DAE4644F0020C28BF4FF0400E99
:10E4F00002EB0E0309EBCC01029301234A604FEAC1
:10E500000E48CEEB050101930025C82242EA08031C
:10E5100084F0010249F83C3035700270DFF814C114
:10E52000424BDFF8048149BBBEF1400F7FF42DAFB1
:10E5300042F0020C09EBCC03029ADFF8F8E05A60D3
:10E540008DBB0D0445F088059DF804304EF83C5015
:10E550000A4433700470134640297FF416AF00213B
:10E56000404A3B60118010E7AA8802F07F02042A2B
:10E5700040F28B81304A0F23137006E74029D7D928
:10E5800042F002020CEBC200029E4660BDB19DF853
:10E59000045035481D703346403988F800404033F8
:10E5A0004CF83200DCE79DF8043033700D04029B18
:10E5B000047045F0C8050B444EF83C50CCE79DF87C
:10E5C00004501D70029B1D4888F8004040394033BC
:10E5D0004CF83200C4E719F0080F0CBF02230323E4
:10E5E0008B557DE521494A68002AC3D06C88B5F86F
:10E5F00004E003E00C314A68002ABBD00B88A34238
:10E60000F8D14B887345F5D1240A032C0CBF11783F
:10E61000098960E7124A0221147054705BE700BF59
:10E620009420074001000400E8A0FF1F7CA0FF1F0A
:10E630007DA0FF1F0080FF1FC02007408800400012
:10E640008820074080200740982007402CA0FF1F0B
:10E6500080A0FF1F18A0FF1FE9A0FF1FF4A0FF1F4D
:10E66000ECA0FF1F28A0FF1FC80040002C430100A2
:10E670008C200740B248116AAC7804700C0600F197
:10E680009881D9F82820AF49100600F1DB81D9F82C
:10E690003020AC49120600F1D081D9F83820A949C0
:10E6A000130600F1C581D9F84020A649150600F1EE
:10E6B000BA81D9F84820A349140600F1AF81D9F8EE
:10E6C0005020A049100600F1A481D9F858209D4996
:10E6D000120600F19981D9F860209A49130600F1D9
:10E6E0008E81D9F868209749150600F18381D9F801
:10E6F00070209449140600F17881D9F87820914966
:10E70000100600F16D81D9F880208E49120600F1C3
:10E710006181D9F888208B49130600F15581D9F819
:10E7200090208849150600F14981D9F8982085493B
:10E73000140600F1FF808448844A85490190854889
:10E74000854D864C049700230596029580460F461A
:10E7500016461D460394306828B1446800F04AFA12
:10E760002046002CF9D100233360029B38681A46FA
:10E77000002342F8253028B1446800F03BFA2046D7
:10E78000002CF9D100223A60019A98F80030114625
:10E79000002241F8042B039A0191023B4FF0000143
:10E7A00022F81510032B07D8DFE803F05D025D02A5
:10E7B0004FF0010388F800300135042D06F10406FE
:10E7C00007F1040708F10108C5D1654C654D2278B1
:10E7D000654B049F059E0021100729701A7000F1F7
:10E7E0009280624962780A700021C9F83010C9F835
:10E7F00038101107DFF84C816ED4A2785C49DFF83D
:10E8000044810A7000211207C9F85010C9F8581045
:10E810004BD4E27857494B4C0A7013074FF0000174
:10E82000C9F87010C9F8781000F1AE803378019300
:10E83000002283F00105C9F89020C9F89820002132
:10E84000029188468E460A464B48047844F0020CF2
:10E8500009EBCC030393019B002B039B5A600CBF75
:10E860008822C82252E64FF0000388F80030A3E760
:10E87000B0F5A06F7FF47EAE012300250193DEE7A3
:10E8800040F621229042F7D074E66D88002D7FF487
:10E8900071AE3A49CDF804E0920011440A7822F0B2
:10E8A00002020A70CBE7022115E600F083F9002886
:10E8B00000F0EB800830324AC8F86400C8F86020E5
:10E8C00000F078F9002800F0DA8008302D4AC9F805
:10E8D0006C00C9F868209CE700F06CF9002800F093
:10E8E000E0800830264AC8F84400C8F8402000F00C
:10E8F00061F9002800F0CF800830224AC9F84C00A6
:10E90000C9F8482079E700F055F9002800F0A58003
:10E9100008301B4AC9F82400C9F8202000F04AF941
:10E92000002800F094800830164AC9F82C00C9F875
:10E93000282056E7D1F89C00083800F05BF9FAE689
:10E94000F4A0FF1F0080FF1FD0A0FF1F6CA0FF1FBF
:10E95000C0A0FF1FF8A0FF1F18A0FF1FB0A2FF1F3D
:10E9600028430100E9A0FF1FC4200740C82007403A
:10E97000CC200740D0200740E8A0FF1FC020074060
:10E9800088004000C800400000F014F9002870D052
:10E9900008304F4AC4F88400C4F8802000F00AF917
:10E9A000002860D008304B4AC9F88C00C9F888208C
:10E9B0003CE7506A083800F01DF962E6D1F894008F
:10E9C000083800F017F9B0E6D1F88C00083800F0EC
:10E9D00011F9A4E6D1F88400083800F00BF998E6A4
:10E9E000C86F083800F006F98DE6486F083800F067
:10E9F00001F982E6C86E083800F0FCF877E6486E48
:10EA0000083800F0F7F86CE6C86D083800F0F2F846
:10EA100061E6486D083800F0EDF856E6C86C083835
:10EA200000F0E8F84BE6486C083800F0E3F840E600
:10EA3000C86B083800F0DEF835E6486B083800F09F
:10EA4000D9F82AE6C86A083800F0D4F81FE62A7810
:10EA5000C9F8280001322A70C3E62A78C9F82000D4
:10EA600001322A705AE72A78C9F8880001322A70E0
:10EA7000DCE62A78C4F8800001322A708EE72A7812
:10EA8000C9F8680001322A70C3E62A78C8F8600025
:10EA900001322A7014E72A78C9F8480001322A7036
:10EAA000ABE62A78C8F8400001322A701FE74029F7
:10EAB0008E4628BF4FF0400E02EB0E030293012357
:10EAC000CEEB01014FEA0E4800250193BCE600BFE2
:10EAD00088004000C8004000F8B500F08FFD294BC9
:10EAE00029482A4C2A4F2B4DDFF8BCC0DFF8BCE088
:10EAF000294E00221A605A609A60DA601A615A61DF
:10EB00009A61DA611A625A629A62DA621A635A6325
:10EB10009A63DA631A645A649A64DA641A655A6505
:10EB20009A65DA651A665A669A66DA661A675A67E5
:10EB30009A67DA67C3F880200168C3F8842041F43B
:10EB400080210160C3F307212170C3F307401349FB
:10EB500038701B0E2B70FF238CF80030104D8EF890
:10EB6000003010480B700123337084F86420702645
:10EB70004FF40074102207F82C3C2E70046081F8CA
:10EB8000F820F8BD0080FF1F348004409C2007401F
:10EB9000B0200740B42007409420074010200740D1
:10EBA00049E400E008E100E08020074088200740B9
:10EBB000704700BF72B60D480268B2FA82F30F2B9D
:10EBC00010DC4FF00041D94022EA0102026062B637
:10EBD000074803EBC303DB00C2180021C1501046F5
:10EBE0005160704762B60020704700BFB492FF1FAB
:10EBF000BC83FF1F0D4B0E4AC31AA2FB03231B0944
:10EC00000F2B0CD80B4A127852B972B60A484FF043
:10EC10000041026821FA03F31A43026062B67047AA
:10EC2000064A1278002AF0D0FFF768B9BC83FF1FAC
:10EC3000398EE338E9A0FF1FB492FF1FF4A0FF1F35
:10EC400038B50E4B0E4C1B68218805468BB1B1F5CB
:10EC5000917F05D20B4A4B1C55549BB2238038BD83
:10EC60000022084898470021064A55540123238072
:10EC700038BDB1F5917FEDD338BD00BF20A1FF1F96
:10EC8000BAA2FF1FC0A2FF1F2DE9F843214E224F59
:10EC90003168012380463B70B1B1204D4B8801EBB8
:10ECA0008302013300240F2BC2F808802C7004D893
:10ECB0004B8000233B70BDE8F88340230B8003208A
:10ECC000FFF780F93460F4E7DFF8549099F80030EA
:10ECD000002BF0D0114D45F6215408E0013C12D034
:10ECE0002B7883B900F00AFB99F800307BB1032040
:10ECF000FFF7EEF80528F1D8FFF75CFF014630601A
:10ED00000028EBD0CAE701232B70BDE8F883BDE8EB
:10ED1000F88300BF3CA1FF1F10A1FF1F40A1FF1FF0
:10ED2000F4A0FF1F1201F8B5D5B2A1B3012943D059
:10ED30004378044600781B0643EA004040F47040E4
:10ED400045F004068F1E3043FFF79EFF022F04F1AB
:10ED5000020314D9053414F8023C14F8032C14F8F7
:10ED6000010C1B0443EA0223334343EA0060033FE0
:10ED7000FFF78AFF022F234604F10304EBD8022F8A
:10ED800023D0012F0DD045F4774040F00500BDE8B9
:10ED9000F840FFF779BF14482843BDE8F840FFF773
:10EDA00073BF187845F4770545F0060545EA00205D
:10EDB000BDE8F840FFF768BF03780C4845EA034513
:10EDC0002843BDE8F840FFF75FBF1A78587845F050
:10EDD000774545F0070545EA022545EA0040BDE8CC
:10EDE000F840FFF751BF00BF06F0F70007F000F74B
:10EDF00038B5084B1C7824B9074D296809B14B88F0
:10EE000003B938BD9B000B800320FFF7DBF82C60B3
:10EE100038BD00BF10A1FF1F3CA1FF1F2DE9F0412D
:10EE2000AD4E33680746002B00F092801D885A884B
:10EE3000910803EB81010432AA428C6842D25A80C5
:10EE400004F00F064FEA1428A449A6F1080208F0BE
:10EE50000F00C4F30313062A00F101050B701AD941
:10EE6000B31E012B5FFA88F04ED9052E48D0042E30
:10EE700000F0A481731F022B7FD90F2E0ED1F7282B
:10EE800042D8F02802D0964B1B883BB1FFF7D8FE42
:10EE90000020BDE8F08127B1BD4202D00020BDE8CE
:10EEA000F081082EC4F3033300F08780092E11D0BF
:10EEB0000A2E40F094800A2BF0D18A4B8A4A1B68B4
:10EEC000A02181E01846FFF795FE0420FEF7E2FF3F
:10EED0003060B5E7092BE1D1270E00F07B81834B31
:10EEE000814A1B689021C4F307461170EDB2FCB251
:10EEF000002B00F09D80224631462846984797E037
:10EF0000F02843D9F72841D0F1380E28C6D801A3FC
:10EF100053F820F0CBF00000AFF000009DF00000AF
:10EF20009DEE00009DEE00008FF000009DEE0000C1
:10EF30006FF100009DEE000039F1000053F1000078
:10EF400077F000009DEE00005FF0000043F000004D
:10EF5000674B1B78002BA1D00420FEF79BFF0346D4
:10EF6000306000289AD00588002D7FF460AFFFF74D
:10EF700041FE35602846BDE8F081FFF761FEC4F32D
:10EF80000740FFF75DFE072E02D1200EFFF758FE67
:10EF9000534B584A198858481468584D524A0170C2
:10EFA00000270E0AF0201F802E7010700CB3012273
:10EFB0005348A0470120BDE8F081082B7FF46EAFD5
:10EFC000504B494A1B688021C4F307461170EDB2CB
:10EFD000240E6BB3284622463146984728E00B2E74
:10EFE00011D10B2B7FF45AAF474B3F4A1B68B0211E
:10EFF000EAE7464B1B68002B00F0FB80404898472F
:10F000000120BDE8F0810C2E40F000810C2B7FF434
:10F0100045AF3F4B344A1B68C0211170EDB2C4F3B9
:10F020000746002B00F0C88028463146240E98473A
:10F030003849314A314B0D7016701C700120BDE803
:10F04000F081354B1B68002B00F0D6809847C4F345
:10F050000746254BEDB2240E83F80080E8E72F4BDE
:10F060001B68002BF2D12E4B1B68A3B1FE209847E2
:10F07000C4F30746EDE72B4B1B68002BE6D1284B6A
:10F080001B6843B1FC209847C4F30746E1E7264BD1
:10F090001B68002BDAD1C4F30746DAE7234B1B6861
:10F0A000C4F30746002BD4D030469847D1E7204B15
:10F0B0001A68002AEFD0260C630C06F07F0003F4D8
:10F0C0007E531843F6B29047C3E71A4B1B68C4F34C
:10F0D0000746002BE8D1BCE748A1FF1FBEA2FF1FD7
:10F0E000BAA2FF1F24A1FF1FB8A2FF1F58A1FF1F34
:10F0F000F4A0FF1F20A1FF1FBCA2FF1FBDA2FF1F86
:10F10000C0A2FF1F50A1FF1F54A1FF1F38A1FF1F66
:10F1100014A1FF1FBFA2FF1F00A1FF1F04A1FF1F1B
:10F1200008A1FF1F44A1FF1F34A1FF1F4CA1FF1F17
:10F130001CA1FF1F30A1FF1F3F4B1B68002B85D177
:10F140003E4B1B68002BA6D0FA209847C4F3074615
:10F150007FE73B4B1B68002B7FF478AF374B1B6876
:10F16000002B98D0FB209847C4F3074671E7354B36
:10F170001B68002B7FF46AAF304B1B68002B8AD0D2
:10F18000F8209847C4F3074663E70E2B7FF486AE5A
:10F190002D4A2E4B1268E0211970002A47D0260C08
:10F1A000610C06F07F0301F47E511943EDB2A1F525
:10F1B000005128469047F6B2240E39E7FFF740FD8C
:10F1C000C4F30740FFF73CFD200EFFF739FD002098
:10F1D000BDE8F0811E4B1D4A1B6880211170EDB205
:10F1E000C4F3074683B1314628463A4698473C4621
:10F1F0001EE70120BDE8F081104B1B68002B3FF497
:10F200004AAFFF20984746E71C4611E70D2EBCD1B8
:10F210000D2B7FF443AE0F4B0C4A1B68D0211170AD
:10F22000EDB2C4F30746002B7FF4FEAEC4E7C4F38F
:10F230000746EDB2240EFBE62CA1FF1F08A1FF1F1D
:10F240000CA1FF1FFCA0FF1F18A1FF1FB8A2FF1FEA
:10F2500050A1FF1F28A1FF1F38B5164D2868E0B147
:10F2600001884488A14213DD03191B7A83B104F19C
:10F270000803C2180C1B002302E012F8011F21B181
:10F280000133A342F9D1204638BD1C46204638BD83
:10F29000FFF7B0FC0020286038BD074B1B780BB986
:10F2A000002038BD0220FEF7F5FD28600028D7D1E8
:10F2B000F6E700BF64A1FF1FF4A0FF1F0D4B1B78F2
:10F2C000BBB910B50C4C216803F0FF024B883F2BF3
:10F2D00007DC07330B4401F1470003F8012F834299
:10F2E000FBD140230B800120FEF76CFE002323603E
:10F2F00010BD70475CA1FF1F60A1FF1F38B5224CF5
:10F30000237803B138BD01232370FFF7A5FF70BB3D
:10F3100000F048F840BB00F0DBF810BBFEF7F8FC4B
:10F32000E0B900232370EFF30583002BEAD1EFF35C
:10F33000108172B6154B1868E0B1154C2278CAB925
:10F3400045691D6001232370C5B1AA6101B962B688
:10F3500000254577836898472570D3E700F020F8AB
:10F36000DFE700F01BF8D9E700F016F8D3E7FFF766
:10F370001FFCCDE70029C5D162B638BD054B1D6025
:10F380000029E5D1E3E700BF69A1FF1F809FFF1FB0
:10F39000849FFF1F7C9FFF1F704700BF704700BF07
:10F3A000704700BF054A064B10781B78C0B2DBB22D
:10F3B000984238BF4030C01A704700BF70A1FF1F8D
:10F3C00071A1FF1FF0B4384B1A7912F0300F2CD016
:10F3D00072B6997D01F0FF0200293DD062B6334F2D
:10F3E000334938780D78334E1C46C0B2EDB2431C19
:10F3F000402BE17928BF0023AB4202F1FF32C9B2B2
:10F400001CBFF154184612F0FF02F0D12A4B1B68C2
:10F41000C2B23A704BB1A84236BFC5F14005401B9D
:10F4200040192728C4BF01221A701F49CA78D2B2D6
:10F43000150616D452060DD51B4B1B795B0609D554
:10F440001E4B1F491B6800220A7003B11A70164B2D
:10F450003C22DA70F0BC70474022D9795A7462B607
:10F46000E3E70B791C06E5D5164B174E1C7833786D
:10F47000E4B2DBB29C420ED0144D01E0A3420AD0AC
:10F480000133402B28BF00230879E85CC0B2C87163
:10F49000087D0728F2D9DBB2034933700B791806CF
:10F4A00044BF7C23CB70C5E700A0064070A1FF1FBE
:10F4B00071A1FF1FB4A1FF1F6CA1FF1FF8A1FF1FC7
:10F4C000F4A1FF1FFCA1FF1FF5A1FF1F74A1FF1FE7
:10F4D000054A064B10781B78C0B2DBB2984238BFA1
:10F4E0004030C01A704700BF70A2FF1F05A2FF1F67
:10F4F000F0B4384B1A7912F0300F2CD072B6997DD7
:10F5000001F0FF0200293DD062B6334F334938780D
:10F510000D78334E1C46C0B2EDB2431C402BE1794E
:10F5200028BF0023AB4202F1FF32C9B21CBFF15425
:10F53000184612F0FF02F0D12A4B1B68C2B23A7093
:10F540004BB1A84236BFC5F14005401B40192728E2
:10F55000C4BF01221A701F49CA78D2B2150616D448
:10F5600052060DD51B4B1B795B0609D51E4B1F4957
:10F570001B6800220A7003B11A70164B3C22DA7025
:10F58000F0BC70474022D9795A7462B6E3E70B7930
:10F590001C06E5D5164B174E1C783378E4B2DBB267
:10F5A0009C420ED0144D01E0A3420AD00133282B17
:10F5B00028BF00230879E85CC0B2C871087D07281D
:10F5C000F2D9DBB2034933700B79180644BF7C23B0
:10F5D000CB70C5E700B0064070A2FF1F05A2FF1F59
:10F5E00030A2FF1F00A2FF1F74A2FF1F04A2FF1F73
:10F5F00078A2FF1F71A2FF1F08A2FF1F70B584B081
:10F6000072B6194B194D1A48702241260F248021D9
:10F610001A702E701A460470197013781B06FCD5E8
:10F62000144B186862B6144B144C984298BF00EB08
:10F63000800001A998BF40000A22FDF7CFFE01A972
:10F640002046002311F8012B01333AB10A2B20F890
:10F65000022FF7D11623237004B070BD5B00DBB21C
:10F66000237004B070BD00BF0000024007000240DC
:10F6700006000240080002407F9698008093FF1F1A
:10F680002DE9F043DFF8EC808BB006460F4600F022
:10F6900073F898F90030013304460D4637D03046F0
:10F6A000394600F0DFF9002831D02BA3D3E900233D
:10F6B0003046394600F026FE814668BB28A3D3E9D0
:10F6C00000233046394600F0FFFD00B398F90030C2
:10F6D000254ACDF82090042400200021022BCDE9FA
:10F6E0000467CDE9026700940192CDE906012CD0B0
:10F6F000684600F0BDF940B3089B1BB101F0AAF9C0
:10F70000089B0360DDE906010BB0BDE8F0832046ED
:10F7100029460BB0BDE8F083134A98F900300192F6
:10F7200003210022CDE90467CDE902670091089228
:10F730002BB90E4B4FF06042CDE90623D8E70C49B8
:10F740000020022BCDE90601D2D101F083F922235A
:10F750000360D1E7AFF30080EF39FAFE422E864016
:10F7600051302DD5104987C098430100FFFFEF4766
:10F770000000F07F9693FF1F2DE9F04FB04F21F06E
:10F780000042BA4283B00C464FEAD17605460DD905
:10F79000AC4FBA4225D9C1F31303034340F0EF80C5
:10F7A0000EB10020014603B0BDE8F08FA64B9A428F
:10F7B00000F2CC80A54B9A4200F2DE808AA3D3E906
:10F7C000002300F05DF90022A14B00F09BFD002812
:10F7D00000F005812846214600229D4B00F050F99B
:10F7E000E1E783A3D3E9002300F08CFD002840F07B
:10F7F000CB802846214680A3D3E9002300F064FD96
:10F800000028CED1934B284603EBC60821467CA3A3
:10F81000D3E9002300F0E6FAD8E9002300F030F93C
:10F8200000F07AFD804600F077FA77A3D3E9002351
:10F8300006460F4600F0D6FA02460B4628462146F9
:10F8400000F01CF972A3D3E90023CDE90001304692
:10F85000394600F0C7FA82468B4652465B46DDE9E0
:10F86000000100F00BF905460C462A4623462846BF
:10F87000214600F0B7FA68A3D3E9002306460F46F5
:10F8800000F0B0FA66A3D3E9002300F0F7F832469F
:10F890003B4600F0A7FA64A3D3E9002300F0F0F898
:10F8A00032463B4600F09EFA61A3D3E9002300F004
:10F8B000E5F832463B4600F095FA5FA3D3E9002312
:10F8C00000F0DEF832463B4600F08CFA02460B466A
:10F8D0002846214600F0D2F806460F462846214623
:10F8E00032463B46B8F1000F56D000F07BFA324664
:10F8F00004460D463B4600204FF0804100F0BEF824
:10F9000002460B462046294600F096FB02460B466F
:10F910005046594600F0B2F8DDE9002300F0AEF899
:10F920000B4602464A49002000F0A8F86FF47F73A6
:10F9300098454FDA08F57A7801EB085100224FF02C
:10F94000B87300F04FFA03B0BDE8F08F424B9A4213
:10F950003FF658AF414BF4002344D3E9002300F0B5
:10F960008DF83F4BC6F101081C44CDE90001D4E9F4
:10F9700000ABC6EB080870E74FF0000875E70246D9
:10F980000B4600F07DF80EE717A3D3E900231046DD
:10F99000194600F027FA06E700F024FA0022804614
:10F9A00089464FF080433046394600F067F80246FA
:10F9B0000B464046494600F03FFB2A46234600F0EE
:10F9C0005DF802460B460020214900F057F803B0CD
:10F9D000BDE8F08F01EB085103B0BDE8F08F804621
:10F9E00043E700BFAFF300809C7500883CE4377E9E
:10F9F000EF39FAFE422E864051302DD5104987C08E
:10FA0000FE822B654715F73F0000E0FE422EE63FE1
:10FA1000763C7935EF39EA3DD0A4BE726937663E4F
:10FA2000F16BD2C541BDBB3E2CDE25AF6A56113FFE
:10FA300093BDBE166CC1663F3E5555555555C53FE5
:10FA4000412E8640FFFFEF7F422ED63FFFFF2F3E25
:10FA50000000F03FA0430100B1A2F03FC04301000D
:10FA6000B043010041F0004101F58010C00F704724
:10FA70000020704781F0004102E000BF83F00043A6
:10FA800030B54FEA41044FEA430594EA050F08BF39
:10FA900090EA020F1FBF54EA000C55EA020C7FEAFD
:10FAA000645C7FEA655C00F0E2804FEA5454D4EB7A
:10FAB0005555B8BF6D420CDD2C4480EA020281EA44
:10FAC000030382EA000083EA010180EA020281EA7C
:10FAD0000303362D88BF30BD11F0004F4FEA0131CE
:10FAE0004FF4801C4CEA113102D0404261EB4101DD
:10FAF00013F0004F4FEA03334CEA133302D0524263
:10FB000063EB430394EA050F00F0A780A4F101041E
:10FB1000D5F1200E0DDB02FA0EFC22FA05F2801858
:10FB200041F1000103FA0EF2801843FA05F359413E
:10FB30000EE0A5F120050EF1200E012A03FA0EFCBD
:10FB400028BF4CF0020C43FA05F3C01851EBE371E7
:10FB500001F0004507D54FF0000EDCF1000C7EEB04
:10FB600000006EEB0101B1F5801F1BD3B1F5001F42
:10FB70000CD349085FEA30004FEA3C0C04F1010461
:10FB80004FEA445212F5800F80F09A80BCF1004F8A
:10FB900008BF5FEA500C50F1000041EB045141EA0C
:10FBA000050130BD5FEA4C0C404141EB010111F40D
:10FBB000801FA4F10104E9D191F0000F04BF0146B8
:10FBC0000020B1FA81F308BF2033A3F10B03B3F196
:10FBD00020020CDA0C3208DD02F1140CC2F10C0226
:10FBE00001FA0CF021FA02F10CE002F11402D8BF84
:10FBF000C2F1200C01FA02F120FA0CFCDCBF41EA50
:10FC00000C019040E41AA2BF01EB0451294330BD1E
:10FC10006FEA04041F3C1CDA0C340EDC04F11404FB
:10FC2000C4F1200220FA04F001FA02F340EA0300D2
:10FC300021FA04F345EA030130BDC4F10C04C4F118
:10FC4000200220FA02F001FA04F340EA03002946F8
:10FC500030BD21FA04F0294630BD94F0000F83F442
:10FC6000801306BF81F480110134013D4EE77FEA25
:10FC7000645C18BF7FEA655C29D094EA050F08BF71
:10FC800090EA020F05D054EA000C04BF1946104652
:10FC900030BD91EA030F1EBF0021002030BD5FEA96
:10FCA000545C05D14000494128BF41F0004130BDBE
:10FCB00014F580043CBF01F5801130BD01F0004512
:10FCC00045F0FE4141F470014FF0000030BD7FEA85
:10FCD000645C1ABF194610467FEA655C1CBF0B4680
:10FCE000024650EA013406BF52EA033591EA030F97
:10FCF00041F4002130BD00BF90F0000F04BF00218F
:10FD0000704730B54FF4806404F132044FF00005C1
:10FD10004FF0000150E700BF90F0000F04BF00213A
:10FD2000704730B54FF4806404F1320410F00045A0
:10FD300048BF40424FF000013EE700BF42004FEA9B
:10FD4000E2014FEA31014FEA02701FBF12F07F4318
:10FD500093F07F4F81F06051704792F0000F14BF15
:10FD600093F07F4F704730B54FF4607401F0004559
:10FD700021F0004120E700BF50EA010208BF7047B0
:10FD800030B54FF000050AE050EA010208BF7047A5
:10FD900030B511F0004502D5404261EB41014FF40E
:10FDA000806404F132045FEA915C3FF4DCAE4FF012
:10FDB00003025FEADC0C18BF03325FEADC0C18BFF9
:10FDC000033202EBDC02C2F1200300FA03FC20FA4A
:10FDD00002F001FA03FE40EA0E0021FA02F1144497
:10FDE000C1E600BF70B54FF0FF0C4CF4E06C1CEAAC
:10FDF00011541DBF1CEA135594EA0C0F95EA0C0F21
:10FE000000F0DEF82C4481EA030621EA4C5123EA93
:10FE10004C5350EA013518BF52EA033541F48011C2
:10FE200043F4801338D0A0FB02CE4FF00005E1FB75
:10FE300002E506F00042E0FB03E54FF00006E1FBBF
:10FE400003569CF0000F18BF4EF0010EA4F1FF0402
:10FE5000B6F5007F64F5407404D25FEA4E0E6D4142
:10FE600046EB060642EAC62141EA55514FEAC52053
:10FE700040EA5E504FEACE2EB4F1FD0C88BFBCF5CF
:10FE8000E06F1ED8BEF1004F08BF5FEA500E50F180
:10FE9000000041EB045170BD06F0004646EA010146
:10FEA00040EA020081EA0301B4EB5C04C2BFD4EB78
:10FEB0000C0541EA045170BD41F480114FF0000E71
:10FEC000013C00F3AB8014F1360FDEBF002001F0DF
:10FED000004170BDC4F10004203C35DA0C341BDC59
:10FEE00004F11404C4F1200500FA05F320FA04F02B
:10FEF00001FA05F240EA020001F0004221F000415F
:10FF000010EBD37021FA04F642EB06015EEA430ED1
:10FF100008BF20EAD37070BDC4F10C04C4F1200501
:10FF200000FA04F320FA05F001FA04F240EA0200B4
:10FF300001F0004110EBD37041F100015EEA430E85
:10FF400008BF20EAD37070BDC4F1200500FA05F2A5
:10FF50004EEA020E20FA04F301FA05F243EA020324
:10FF600021FA04F001F0004121FA04F220EA020033
:10FF700000EBD3705EEA430E08BF20EAD37070BD79
:10FF800094F0000F0FD101F00046400041EB010159
:10FF900011F4801F08BF013CF7D041EA060195F03B
:10FFA000000F18BF704703F00046520043EB0303F5
:10FFB00013F4801F08BF013DF7D043EA06037047E2
:10FFC00094EA0C0F0CEA135518BF95EA0C0F0CD0ED
:10FFD00050EA410618BF52EA4306D1D181EA030133
:10FFE00001F000414FF0000070BD50EA410606BF2D
:10FFF0001046194652EA430619D094EA0C0F02D172
:020000021000EC
:1000000050EA013613D195EA0C0F05D152EA0336B6
:100010001CBF104619460AD181EA030101F00041D4
:1000200041F0FE4141F470014FF0000070BD41F01D
:10003000FE4141F4780170BD70B54FF0FF0C4CF4F7
:10004000E06C1CEA11541DBF1CEA135594EA0C0F16
:1000500095EA0C0F00F0A7F8A4EB050481EA030E63
:1000600052EA03354FEA013100F088804FEA03334A
:100070004FF0805545EA131343EA12634FEA022218
:1000800045EA111545EA10654FEA00260EF00041D9
:100090009D4208BF964244F1FD0404F5407402D22B
:1000A0005B084FEA3202B61A65EB03055B084FEABC
:1000B00032024FF480104FF4002CB6EB020E75EBB9
:1000C000030E22BFB61A754640EA0C005B084FEAE1
:1000D0003202B6EB020E75EB030E22BFB61A75465E
:1000E00040EA5C005B084FEA3202B6EB020E75EBA9
:1000F000030E22BFB61A754640EA9C005B084FEA21
:100100003202B6EB020E75EB030E22BFB61A75462D
:1001100040EADC0055EA060E18D04FEA051545EA1C
:1001200016754FEA06164FEAC30343EA52734FEAC5
:10013000C2025FEA1C1CC0D111F4801F0BD141EA3E
:1001400000014FF000004FF0004CB6E711F4801FA3
:1001500004BF01430020B4F1FD0C88BFBCF5E06F83
:100160003FF6AFAEB5EB030C04BFB6EB020C5FEA93
:10017000500C50F1000041EB045170BD0EF0004EE8
:100180004EEA113114EB5C04C2BFD4EB0C0541EA1A
:10019000045170BD41F480114FF0000E013C90E617
:1001A00045EA060E8DE60CEA135594EA0C0F08BFDB
:1001B00095EA0C0F3FF43BAF94EA0C0F0AD150EADA
:1001C00001347FF434AF95EA0C0F7FF425AF10466D
:1001D00019462CE795EA0C0F06D152EA03353FF495
:1001E000FDAE1046194622E750EA410618BF52EA12
:1001F00043067FF4C5AE50EA41047FF40DAF52EAE6
:1002000043057FF4EBAE12E74FF0FF3C06E000BF82
:100210004FF0010C02E000BF4FF0010C4DF804CD8F
:100220004FEA410C7FEA6C5C4FEA430C18BF7FEA4F
:100230006C5C1BD001B050EA410C0CBF52EA430C7D
:1002400091EA030F02BF90EA020F0020704710F1FD
:10025000000F91EA030F58BF994208BF90422CBF8C
:10026000D8176FEAE37040F0010070474FEA410C85
:100270007FEA6C5C02D150EA013C07D14FEA430CA3
:100280007FEA6C5CD6D152EA033CD3D05DF8040B14
:10029000704700BF8446104662468C461946634646
:1002A00000E000BF01B5FFF7B7FF002848BF10F11D
:1002B000000F01BD4DF808EDFFF7F4FF0CBF012062
:1002C00000205DF808FB00BF4DF808EDFFF7EAFFDE
:1002D00034BF012000205DF808FB00BF4DF808ED99
:1002E000FFF7E0FF94BF012000205DF808FB00BF8E
:1002F0004DF808EDFFF7CEFF94BF012000205DF818
:1003000008FB00BF4DF808EDFFF7C4FF34BF012024
:1003100000205DF808FB00BF4FEA410212F5001211
:1003200015D211D56FF47873B3EB625212D94FEA3C
:10033000C12343F0004343EA505311F0004F23FA26
:1003400002F018BF404270474FF00000704750EA7B
:10035000013005D111F0004008BF6FF00040704738
:100360004FF00000704700BF4FEA4102B2F1E04396
:1003700024BFB3F5001CDCF1FE5C0DD901F0004C8C
:100380004FEAC0024CEA5070B2F1004F40EB8300DC
:1003900008BF20F00100704711F0804F21D113F108
:1003A0003872BCBF01F00040704741F480114FEA41
:1003B0005252C2F11802C2F1200C10FA0CF320FACA
:1003C00002F018BF40F001004FEAC1234FEAD323E7
:1003D00003FA0CFC40EA0C0023FA02F34FEA430351
:1003E000CCE77FEA625307D150EA01331EBF4FF0DA
:1003F000FE4040F44000704701F0004040F0FE40F5
:1004000040F40000704700BF80F0004002E000BFF1
:1004100081F0004142001FBF5FEA410392EA030FEF
:100420007FEA226C7FEA236C6AD04FEA1262D2EB39
:100430001363C1BFD218414048404140B8BF5B423E
:10044000192B88BF704710F0004F40F4000020F0D7
:100450007F4018BF404211F0004F41F4000121F0ED
:100460007F4118BF494292EA030F3FD0A2F1010237
:1004700041FA03FC10EB0C00C3F1200301FA03F175
:1004800000F0004302D5494260EB4000B0F5000F98
:1004900013D3B0F1807F06D340084FEA310102F157
:1004A0000102FE2A51D2B1F1004F40EBC25008BF09
:1004B00020F0010040EA03007047490040EB0000D3
:1004C00010F4000FA2F10102EDD1B0FA80FCACF102
:1004D000080CB2EB0C0200FA0CF0AABF00EBC25001
:1004E00052421843BCBFD0401843704792F0000FEF
:1004F00081F4000106BF80F400000132013BB5E742
:100500004FEA41037FEA226C18BF7FEA236C21D0B7
:1005100092EA030F04D092F0000F08BF084670471C
:1005200090EA010F1CBF0020704712F07F4F04D1EA
:10053000400028BF40F00040704712F100723CBFFD
:1005400000F50000704700F0004343F0FE4040F427
:10055000000070477FEA226216BF08467FEA2363E5
:100560000146420206BF5FEA412390EA010F40F4D0
:10057000800070474FF0000304E000BF10F000431C
:1005800048BF40425FEA000C08BF704743F0964303
:1005900001464FF000001CE050EA010208BF70471E
:1005A0004FF000030AE000BF50EA010208BF7047A5
:1005B00011F0004302D5404261EB41015FEA010CBA
:1005C00002BF84460146002043F0B64308BFA3F1B2
:1005D0008053A3F50003BCFA8CF2083AA3EBC25394
:1005E00010DB01FA02FC634400FA02FCC2F12002B3
:1005F000BCF1004F20FA02F243EB020008BF20F0EA
:100600000100704702F1200201FA02FCC2F120024F
:1006100050EA4C0021FA02F243EB020008BF20EA44
:10062000DC7070474FF0FF0C1CEAD0521EBF1CEA72
:10063000D15392EA0C0F93EA0C0F6FD01A4480EA60
:10064000010C400218BF5FEA41211ED04FF0006349
:1006500043EA501043EA5111A0FB01310CF0004075
:10066000B1F5000F3EBF490041EAD3715B0040EA9B
:10067000010062F17F02FD2A1DD8B3F1004F40EB6B
:10068000C25008BF20F00100704790F0000F0CF03E
:10069000004C08BF49024CEA502040EA51207F3A02
:1006A000C2BFD2F1FF0340EAC250704740F40000DD
:1006B0004FF00003013A5DDC12F1190FDCBF00F0CE
:1006C00000407047C2F10002410021FA02F1C2F17C
:1006D000200200FA02FC5FEA310040F1000053EA18
:1006E0004C0308BF20EADC70704792F0000F00F066
:1006F000004C02BF400010F4000F013AF9D040EA6C
:100700000C0093F0000F01F0004C02BF490011F4FF
:10071000000F013BF9D041EA0C018FE70CEAD153FD
:1007200092EA0C0F18BF93EA0C0F0AD030F0004C7D
:1007300018BF31F0004CD8D180EA010000F0004031
:10074000704790F0000F17BF90F0004F084691F0EF
:10075000000F91F0004F14D092EA0C0F01D1420229
:100760000FD193EA0C0F03D14B0218BF084608D1F2
:1007700080EA010000F0004040F0FE4040F400003C
:10078000704740F0FE4040F4400070474FF0FF0CCF
:100790001CEAD0521EBF1CEAD15392EA0C0F93EA16
:1007A0000C0F69D0A2EB030280EA010C49024FEA68
:1007B000402037D04FF0805343EA111143EA101321
:1007C0000CF000408B4238BF5B0042F17D024FF4D9
:1007D000000C8B4224BF5B1A40EA0C00B3EB510FB4
:1007E00024BFA3EB510340EA5C00B3EB910F24BF9D
:1007F000A3EB910340EA9C00B3EBD10F24BFA3EB22
:10080000D10340EADC001B0118BF5FEA1C1CE0D1E9
:10081000FD2A3FF650AF8B4240EBC25008BF20F09C
:10082000010070470CF0004C4CEA50207F32C2BFF0
:10083000D2F1FF0340EAC250704740F400004FF08D
:100840000003013A37E792F0000F00F0004C02BFBE
:10085000400010F4000F013AF9D040EA0C0093F088
:10086000000F01F0004C02BF490011F4000F013BE2
:10087000F9D041EA0C0195E70CEAD15392EA0C0F4A
:1008800008D142027FF47DAF93EA0C0F7FF470AF82
:10089000084676E793EA0C0F04D14B023FF44CAFC5
:1008A00008466EE730F0004C18BF31F0004CCAD15A
:1008B00030F000427FF45CAF31F000437FF43CAF96
:1008C0005FE700BF4FF0FF3C06E000BF4FF0010CB8
:1008D00002E000BF4FF0010C4DF804CD4FEA40029A
:1008E0004FEA41037FEA226C18BF7FEA236C11D0E4
:1008F00001B052EA530C18BF90EA010F58BFB2EB97
:10090000030088BFC81738BF6FEAE17018BF40F016
:10091000010070477FEA226C02D15FEA402C05D1CA
:100920007FEA236CE4D15FEA412CE1D05DF8040B4F
:10093000704700BF844608466146FFE70FB5FFF7E2
:10094000C9FF002848BF10F1000F0FBD4DF808ED9A
:10095000FFF7F4FF0CBF012000205DF808FB00BF8B
:100960004DF808EDFFF7EAFF34BF012000205DF8E5
:1009700008FB00BF4DF808EDFFF7E0FF94BF012032
:1009800000205DF808FB00BF4DF808EDFFF7D2FF2F
:1009900094BF012000205DF808FB00BF4DF808ED72
:1009A000FFF7C8FF34BF012000205DF808FB00BF3F
:1009B0004FEA4002B2F1FE4F0FD34FF09E03B3EB6C
:1009C00012620DD94FEA002343F0004310F0004FAC
:1009D00023FA02F018BF404270474FF00000704702
:1009E00012F1610F01D1420205D110F0004008BFA1
:1009F0006FF0004070474FF00000704742000ED289
:100A0000B2F1FE4F0BD34FF09E03B3EB126209D449
:100A10004FEA002343F0004323FA02F070474FF0FF
:100A20000000704712F1610F01D1420202D14FF074
:100A3000FF3070474FF00000704700BF0B46014683
:100A4000184600F001B800BF13460A4601460220CE
:100A500000F0A8BE014B1868704700BFC097FF1F89
:100A600070B50F4E0F4D761BB61018BF002405D081
:100A7000013455F8043B9847A642F9D10A4E0B4D74
:100A8000761B03F0A7FCB61018BF002406D0013473
:100A900055F8043B9847A642F9D170BD70BD00BF20
:100AA000E0430100E0430100F4430100E0430100A2
:100AB000024B0146186800F00BB800BFC097FF1F3B
:100AC000024B0146186800F031BF00BFC097FF1FFE
:100AD0002DE9F04F01F10B05162D83B0064640F2CB
:100AE0009F8035F0070500F1BF80A94200F2BC806D
:100AF00000F058FBB5F5FC7FC0F09C826B0A00F05B
:100B0000BA80042B00F28381A80900F1390E4FEA64
:100B10004E033830C44F07EB8303A3F108015C6830
:100B2000A14207D1ACE0002A80F2AC80E468A14287
:100B300000F0A680636823F003035A1B0F2AF2DD3E
:100B4000B9493C6901F1080E744500F0B38163684E
:100B500023F003035A1B0F2A00F39981002AC1F8DE
:100B600014E0C1F810E080F29E80B3F5007F80F0C1
:100B70006781DB0803F1010C01229B1002FA03F3E9
:100B80004A6851F83C80C4F8088001EBCC091A434C
:100B9000A9F10803E3604A6041F83C40C8F80C4002
:100BA000831001249C40944200F28A80144206D1B2
:100BB00020F003006400144200F10400FAD007EBB7
:100BC000C009CC468046DCF80C108C4507D173E197
:100BD000002A80F28181C9688C4500F06D814B68E4
:100BE00023F003035A1B0F2AF2DD0C46D1F80CC088
:100BF00054F8088F4B1945F001054D6042F0010192
:100C0000C8F80CC03046CCF808807B613B61C3F863
:100C10000CE0C3F808E059609A5000F0C5FA1FE0F4
:100C2000102921D800F0BEFA1025062302207E4F9D
:100C300007EB8303A3F108025C68944200F045814E
:100C40006368E168A56823F00303234430465A68CB
:100C5000E96042F001028D605A6000F0A5FA0834A4
:100C6000204603B0BDE8F08F00240C2320463360FB
:100C700003B0BDE8F08F80234FF0400E3F2049E7DE
:100C800070465DE72344E1685A68A56842F00102B6
:100C9000E96030468D605A6000F086FA08342046DC
:100CA00003B0BDE8F08F234430465A6842F0010299
:100CB0005A6000F079FA0834204603B0BDE8F08F9E
:100CC000BC68636823F00308A84504D3C5EB080398
:100CD0000F2B00F38C80554BDFF860911A68D9F820
:100CE000003001332A4404EB080A00F0608102F569
:100CF00080520F3222F47F6222F00F0211463046FA
:100D0000019200F04BFCB0F1FF3F8346019A00F0E6
:100D10005881824500F2FC80454B1968DA45114440
:100D2000196000F05381D9F80000DFF810E10130BC
:100D30001BBFCAEB0B0A5144CEF800B019601BF080
:100D4000070100F01781C1F10800C1F5805183440B
:100D500008315A44C2F30B02C2EB0109494630463E
:100D6000019300F01BFC431C019B00F03F81CBEB87
:100D700000024A4442F001021968C7F808B0494429
:100D8000BC42CBF804201960DFF8A49016D0B8F16B
:100D90000F0F40F2FD806268A8F10C0323F00703F7
:100DA000E01802F001024FF0050E1A430F2B6260AB
:100DB000C0F804E0C0F808E000F21C811D4BBC68DC
:100DC0001A68914288BF19601B4B1A689142626889
:100DD00088BF196022F003029542A2EB050301D8F7
:100DE0000F2B04DC304600F0DFF9002438E76219ED
:100DF00043F0010345F0010565603046BA60536079
:100E000000F0D2F90834204603B0BDE8F08F142B6F
:100E100071D9542B00F2A480280B00F16F0E4FEA19
:100E20004E036E3076E600BFC497FF1F84A2FF1FFB
:100E300088A2FF1F80A2FF1F7CA2FF1FD09BFF1F65
:100E40005A0A042A5ED9142A00F2B38002F15C0126
:100E500049005B3207EB810C57F82110DFF8DC8189
:100E6000ACF1080C8C4500F088804A6822F003023F
:100E7000934202D289688C45F7D1D1F80CC07A68C8
:100E8000C4F80CC0A160CCF80840CC6088E66319B7
:100E900042F0010745F00105656030464B610B618A
:100EA000C3F80CE0C3F808E05F609A50083400F023
:100EB0007BF9D5E64A6873E608F1010818F0030FDC
:100EC0000CF1080C7FF47FAE30E0DC68A34208BF71
:100ED00002303FF435AEB3E60B440C465A68C9689D
:100EE00054F8085F42F001025A603046E9608D60B4
:100EF00000F05AF9B4E603F15C0E03F15B004FEA2F
:100F00004E0307E69A0902F1390149003832A1E798
:100F1000BC424A4B3FF400AF9C68626822F0030277
:100F20005AE759F80839994540F0828010F0030FCC
:100F300000F1FF30F5D17B6823EA04037B60640095
:100F40009C423FF6BDAE002C3FF4BAAE1C42404678
:100F50007FF435AE64001C4200F10400FAD02EE6A6
:100F6000B3F5AA7F18D8E80B00F1780E4FEA4E03CC
:100F70007730CFE54FF48051EBE60121D8F804300B
:100F8000921001FA02F21A43C8F80420614677E78A
:100F90000123CBF8043025E740F25452934220D885
:100FA000A80C00F17D0E4FEA4E037C30B2E5103202
:100FB000A4E6542A26D81A0B02F16F0149006E32BA
:100FC00048E7BC68626822F0030205E7CAF30B0039
:100FD00000287FF4A8AE4244BB6842F001025A6088
:100FE000ECE6FE234FF07F0E7E2093E501224FF0CA
:100FF0000009C1E604F10801304600F097FCD9F879
:101000000010DBE6B2F5AA7F05D8DA0B02F1780111
:10101000490077321EE740F254518A4205D89A0CB3
:1010200002F17D0149007C3214E7FE217E2211E7A6
:101030007B6884E7E808431C5B00F8E5C497FF1F62
:101040008842F0B50DD98B1898420AD28118002A2F
:1010500051D09A1A13F8014D01F8014D9342F9D17C
:10106000F0BD0F2A48D941EA00039B0746D100F1A1
:10107000100401F11003154653F8106C44F8106C7D
:1010800053F80C6C44F80C6C53F8086C44F8086C7A
:10109000103D53F8046C44F8046C0F2D03F1100359
:1010A00004F11004E8D8A2F1100323F00F0302F0BA
:1010B0000F0E1033BEF1030F1944034421D91E1F34
:1010C0000D467446043C55F8047B46F8047F032C17
:1010D000F8D8AEF1040424F003040434234421447A
:1010E00002F0030262B1013B0A4411F8014B03F81C
:1010F000014F8A42F9D1F0BD0346F3E70346F2E718
:10110000F0BD7246EEE700BF70B4840746D0541EAF
:10111000002A41D0CDB2034602E0621EE4B3144679
:1011200003F8015B9A07F8D1032C2ED9CDB245EA1A
:1011300005250F2C45EA054519D903F1100226466D
:10114000103E0F2E42F8105C42F80C5C42F8085C2E
:1011500042F8045C02F11002F2D8A4F1100222F06D
:101160000F0204F00F041032032C13440DD91E4655
:101170002246043A032A46F8045BFAD8221F22F0DA
:1011800003020432134404F003042CB1C9B21C441A
:1011900003F8011BA342FBD170BC70471446034601
:1011A000C2E700BF704700BF704700BF024B0A464E
:1011B0000146186800F002B8C097FF1F2DE9F04FF4
:1011C000174683B0002900F0C1800E46814607F122
:1011D0000B05FFF7E7FF56F804EC162D2EF003047D
:1011E000A6F1080840D810221546AF4241D89442D3
:1011F00075DAC94B996808EB04008842416800F031
:10120000D98021F0010303445B68DB077DD51EF024
:10121000010F35D039464846FFF75AFC0746E0B182
:1012200056F8043C23F001034344A0F108029A421B
:1012300000F04481221F242A00F23181132A00F297
:1012400004810346324611681960516859609268FA
:101250009A603146484600F069FB4846FFF7A4FF14
:10126000384603B0BDE8F08F25F00705002D2A466B
:10127000BBDA0C230020C9F8003003B0BDE8F08FC2
:1012800056F8083CC3EB080ADAF8043023F0030CE4
:1012900004EB0C039342BDDB5746DAF80C1057F809
:1012A000080F221F242AC160886000F21781132AC8
:1012B00040F212813168CAF808107168CAF80C103F
:1012C0001B2A00F22B8108360AF1100231681160E6
:1012D00071685160B16891603E461C46D046631B00
:1012E0000F2B1DD8D8F8043003F0010323434444E6
:1012F000C8F80430636843F0010363604846FFF7B1
:1013000053FF304603B0BDE8F08F21F003012144C4
:10131000914221DBC36882680C46D3609A60DEE7A5
:10132000D8F8042008EB050102F00102154343F050
:1013300001020B44C8F804504A605A6842F00102A6
:1013400008315A60484600F0F1FAD7E7114603B079
:10135000BDE8F04FFFF7BCBB1EF0010F7FF45AAFA2
:1013600056F8083CC3EB080ADAF8043023F0030C03
:1013700001EB0C0E96458BDBC36882685746D36041
:101380009A6057F8081FDAF80C30CB60221F242A25
:10139000996000F29980132A62D93368CAF808303C
:1013A0007368CAF80C301B2A00F2A08008360AF1D4
:1013B000100356E021F0030BA34405F11000834510
:1013C00059DA1EF0010F7FF425AF56F8081CC1EB67
:1013D000080ADAF8041021F0030CE34458453FF7FB
:1013E00057AF5746DAF80C1057F8080F221F242A77
:1013F000C160886000F2B480132A40F2A580316891
:10140000CAF808107168CAF80C101B2A00F2AF80E5
:1014100008360AF110023168116071685160B168D4
:1014200091600AEB0501C5EB0B0242F001029960E5
:101430004A60DAF8043003F001031D434846CAF855
:101440000450FFF7B1FE38465CE733680360736809
:1014500043601B2A27D800F1080306F10802F2E6D0
:101460003B4632681A6072685A60B2689A603E46BB
:101470007446D04633E708EB0501C5EB0B0B4BF088
:10148000010299604A6056F8043C03F001031D43D1
:10149000484646F8045CFFF787FE304632E731469F
:1014A000FFF7CEFDD5E6B3688360F368C360242AF6
:1014B00028D000F1100306F11002C4E650F8043CF5
:1014C00023F003031C440AE7314638467446D046ED
:1014D000FFF7B6FD3E4602E73A46F7E631463846A4
:1014E0001C46D046FFF7ACFD3E46F8E6B368CAF8A6
:1014F0001030F368CAF81430242A1BD010360AF1D1
:101500001803AEE7336903617369436106F118029A
:1015100000F1180397E600BFC497FF1FB168CAF82F
:101520001010F168CAF81410242A0FD010360AF1EE
:101530001802CBE63369CAF818307369CAF81C3050
:1015400018360AF120038CE73A4664E73269CAF894
:1015500018207269CAF81C2018360AF12002B5E674
:10156000314638460193FFF76BFD019B59E7B1689F
:10157000CAF81010F168CAF81410242A03D01036E3
:101580000AF1180247E73269CAF818207269CAF8E6
:101590001C2018360AF120023DE700BF38B5074C81
:1015A0000023054608462360FBF7E2FE431C00D0FB
:1015B00038BD2368002BFBD02B6038BDE4A3FF1F90
:1015C00090F800F06DE9024520F007016FF0000C83
:1015D00010F0070491F820F040F049804FF000042B
:1015E0006FF00700D1E9002391F840F000F1080006
:1015F00082FA4CF2A4FA8CF283FA4CF3A2FA8CF33E
:101600004BBBD1E9022382FA4CF200F10800A4FAA4
:101610008CF283FA4CF3A2FA8CF3E3B9D1E90423F8
:1016200082FA4CF200F10800A4FA8CF283FA4CF32F
:10163000A2FA8CF37BB9D1E9062301F1200182FAE9
:101640004CF200F10800A4FA8CF283FA4CF3A2FAEF
:101650008CF3002BC6D0002A04BF04301A4612BAFD
:10166000B2FA82F2FDE8024500EBD2007047D1E900
:10167000002304F00305C4F100004FEAC50514F08F
:10168000040F91F840F00CFA05F562EA05021CBF60
:1016900063EA050362464FF00004A9E7002A41D03F
:1016A00040EA010313F00303F0B425D1032A23D940
:1016B00004680D68AC421FD1043A35D0A4F101355D
:1016C00025EA040414F0803F31D1071D0D1D0DE003
:1016D00057F8043B0E68A3F10134B34224EA030433
:1016E0000AD1043A20D014F0803F23D1032A29469E
:1016F000384605F10405EBD803780C789C4202F1DA
:10170000FF320CD182B114B916E06AB17BB110F886
:10171000013F11F8014FA34202F1FF32F5D0181B2F
:10172000F0BC7047104670471046F0BC7047184632
:10173000F0BC70470020F3E72046F1E740EA0103E0
:101740009B0770B42BD1032A29D90C4603462146A6
:1017500054F8046BA6F1013525EA060515F0803F23
:1017600006D1043A032A43F8046B2146EFD8A2B10C
:101770000C781C70013A013301313CB16AB111F8A7
:10178000014B03F8014B013A002CF7D12AB11A445E
:10179000002103F8011B9A42FBD170BC704703463D
:1017A000E5E700BF2DE9F047254C2568D5F848410D
:1017B0000646884692469946C4B360681F2817DCDF
:1017C000431C76B104EB80050122C5F888A0D4F84B
:1017D000881182401143022EC4F88811C5F808917F
:1017E0001ED00230636044F820800020BDE8F087FE
:1017F000144B03B34FF4C870FFF75AF90446D0B145
:10180000D5F84831002780E88800C5F848413846B7
:101810000123C4F88871C4F88C71002EE1D0D1E79F
:10182000D4F88C110A43C4F88C21DAE705F5A674C4
:10183000C5F84841C1E74FF0FF30BDE8F08700BF71
:10184000D0430100B10A0100024B13B1024800F07D
:1018500005B8704700000000691801000023014628
:101860001A461846FFF79EBF38B5074D074C2C1B8C
:10187000A41005D0013C55F8043D9847002CF9D13F
:10188000BDE8384002F0B6BD0000000000000000D6
:10189000F8B5234F0C460646FFF784FCBB685D682D
:1018A00025F00305291B01F6EF7121F47F6121F07A
:1018B0000F01A1F58054B4F5805F07DB00213046AD
:1018C000FFF76CFEBB682B44984204D03046FFF70C
:1018D0006BFC0020F8BD61423046FFF75FFE01302F
:1018E0000DD0104BBA6819682D1B45F00105304624
:1018F000091B55601960FFF757FC0120F8BD002156
:101900003046FFF74BFEBA68831A0F2BDEDD064C1C
:101910000449246843F00103001B53600860D5E7C5
:10192000C497FF1F88A2FF1FD09BFF1F002945D02F
:101930002DE9F0410D468046FFF734FC55F8047C54
:101940006A4927F00103A5F10804E2188E6850687F
:10195000B24220F0030062D0FE0750600BD455F86D
:10196000087CE41B01F1080EA56875453B446FD067
:10197000E768EF60BD6015186D68ED0742D543F06C
:1019800001026260E350B3F5007F18D2DB085A1CF5
:101990004D6851F83270A76001209B1000FA03F3E4
:1019A00001EBC2001D430838E0604D6041F8324051
:1019B000FC604046BDE8F041FFF7F6BB70475A0AAD
:1019C000042A53D89A0902F139077F0002F1380539
:1019D00001EB870051F827204449083890424DD048
:1019E000516821F003018B4202D292689042F7D1F4
:1019F000D068E060A2608460D4604046BDE8F041F9
:101A0000FFF7D2BB95683A4FBD4203443FD0D06840
:101A1000E86043F0010285606260E350B3E7FF07CE
:101A2000034407D455F8082CA41A1344A068E268AC
:101A3000C26090602F4A126843F0010093426060D8
:101A40008C60B6D32C4B40461968FFF721FFB0E7F6
:101A500011184968C90744D49168D268CA60034420
:101A600043F0010091606060E350A2E7142A17D8A8
:101A700002F15C077F0002F15B05A9E7AA104B6841
:101A8000012505FA02F213434B600246B1E743F029
:101A900001024C610C61E560A5606260E35088E77B
:101AA000542A06D81A0B02F16F077F0002F16E0567
:101AB0008EE7B2F5AA7F06D8DA0B02F178077F002D
:101AC00002F1770584E740F25450824206D89A0C1E
:101AD00002F17D077F0002F17C0579E7FE277E2574
:101AE00076E743F001026260E35062E7C497FF1FAC
:101AF000CC97FF1FCC9BFF1F84A2FF1F000078051F
:101B00003408540B800C3C0F5C12E015FA19141EBB
:101B10006022AC265C2B0C30BC34023AFF3FFFFF46
:101B200000000000070000000C0000001000000092
:101B300013000000180000001C000000000000005E
:101B4000070000000C00000010000000130000005F
:101B50001600000018000000000000000700000050
:101B60000C00000013000000180000001F0000001F
:101B700024000000000000000C000000180000001D
:101B800024000000300000003C000000480000007D
:101B9000FBFFFFFFF7FFFFFFF4FFFFFFFBFFFFFF70
:101BA000F7FFFFFFF4FFFFFFFBFFFFFFF7FFFFFF64
:101BB000F4FFFFFFFDFFFFFFF8FFFFFFF4FFFFFF54
:101BC000FDFFFFFFF8FFFFFFF4FFFFFFFDFFFFFF3B
:101BD000F8FFFFFFF4FFFFFFFBFFFFFFF7FFFFFF33
:101BE000F4FFFFFFFBFFFFFFF7FFFFFFF4FFFFFF27
:101BF000FBFFFFFFF8FFFFFFF4FFFFFFFCFFFFFF0E
:101C0000F9FFFFFFF4FFFFFFFDFFFFFFF8FFFFFFFE
